:020000040000FA
:100000000020040000000000C0220000C022000008
:10001000C0220000C0220000C0220000C022000058
:10002000C0220000C0220000C0220000C022000048
:10003000C0220000C0220000C0220000C022000038
:10004000C0220000C0220000C0220000C022000028
:10005000C0220000C0220000C022000082C20000B6
:10006000C0220000C0220000C0220000C022000008
:10007000C0220000C0220000C0220000C0220000F8
:10008000C0220000C0220000C0220000C0220000E8
:10009000C0220000C0220000C0220000C0220000D8
:1000A000C0220000C0220000C0220000C0220000C8
:1000B000C0220000C0220000C0220000C0220000B8
:1000C000C0220000C0220000C0220000C0220000A8
:1000D000C0220000C0220000C0220000C022000098
:1000E000C0220000C0220000C0220000C022000088
:1000F000C0220000C0220000C0220000C022000078
:10010000C0220000C0220000C0220000C022000067
:10011000C0220000C0220000C0220000C022000057
:10012000C0220000C0220000C0220000C022000047
:10013000C0220000C0220000C0220000C022000037
:10014000C0220000C0220000C0220000C022000027
:10015000C0220000C0220000C0220000C022000017
:10016000C0220000C0220000C0220000C022000007
:10017000C0220000C0220000C0220000C0220000F7
:10018000CABF0000C0220000C0220000C022000040
:10019000C0220000C0220000C0220000C0220000D7
:1001A000FFFFFF00FFFFFF00FFFFFF00FFFFFF005B
:1001B000FFFFFF00FFFFFF00FFFFFF00FFFFFF004B
:1001C000FFFFFF00FFFFFF00FFFFFF00FFFFFF003B
:1001D000FFFFFF00FFFFFF00FFFFFF00FFFFFF002B
:1001E000FFFFFF00FFFFFF00FFFFFF00FFFFFF001B
:1001F000FFFFFF00FFFFFF00FFFFFF00FFFFFF000B
:10020000FFFFFF00FFFFFF00C0220000C022000030
:10021000C0220000C0220000C0220000C022000056
:10022000C0220000C0220000C0220000C022000046
:10023000C0220000C0220000C0220000C022000036
:10024000C0220000C0220000C0220000C022000026
:10400000CF5123000E7F24000E0188000000000025
:10401000000020000000E00002003200000120004B
:10402000200288000C000700E0C32A0001002000E5
:1040300011000700000020000000E0000200320034
:104040000000020000000000A0BF0200000000000D
:104050000040DA000000FE004440A900E05D2000BE
:104060000000E0000300320000002000A0018800F2
:104070004440A800000006009101880080007800FC
:104080000000EB0015003700E280400032A0B400D1
:104090009101BA00E280400032A0B4009102BA005F
:1040A000E280400032A0B4000002EB00472BDE00AB
:1040B000F507B200602CE10004003A000059EB0063
:1040C0008301E900FDFF3E00040037006128E100A4
:1040D000010032000082EB000B00070011C3BA00A0
:1040E0001101BA000604E00003003A000200E000FB
:1040F000E5FF3A0000000600F607B20096018800CE
:1041000082007800F5FF37003159BA008301E900D9
:104110000C0032002159BA008301E9000800320086
:104120000400E00003003A00E280400032A0B40046
:10413000F5FF370011D9BA008301E900FAFF3A0010
:104140008100E800E180400032A0B40000000600D9
:10415000069D040000000000129D04000000000005
:104160000C9D040000000000009D04000000000001
:10417000729D040000000000967004000000000022
:104180001E710400000000008075040000000000A3
:10419000E2740400000000002C7104000000000024
:1041A0008E70040000000000F870040000000000A1
:1041B00088710400000000009076040000000000F8
:1041C00000710400000000002677040000000000D9
:1041D0005E76040000000000267604000000000067
:1041E0004C73040000000000B870040000000000E0
:1041F00022750400000000009C7004000000000014
:10420000F6720400000000006C9F04000000000033
:1042100034980400000000005098040000000000E2
:1042200028450400000000008CC3040000000000CA
:104230007CC30400000000006CC304000000000008
:104240005CC30400000000004CC304000000000038
:1042500032C304000000000044C30400000000005A
:104260003EC30400000000003C9004000000000079
:10427000F68F040000000000EE8F04000000000034
:104280001A900400000000000E90040000000000DE
:104290000690040000000000FE8F040000000000F3
:1042A000FA8F0400000000000491040000000000E8
:1042B000269004000000000034900400000000007C
:1042C000366B040000000000486B04000000000092
:1042D000E06804000000000098680400000000008E
:1042E000586B040000000000146D04000000000082
:1042F0006669040000000000BE6D040000000000BC
:10430000326B040000000000BE6B040000000000DF
:10431000E6680400000000001E7A040000000000AF
:10432000D4790400000000009E7A04000000000020
:104330002E7B040000000000AC7C040000000000A4
:10434000AC78040000000000907B04000000000036
:1043500042790400000000005479040000000000CD
:1043600080780400000000007E600400000000006F
:104370005E600400000000009E6004000000000079
:104380008A630400000000009C6304000000000039
:1043900054650400000000002E61040000000000CD
:1043A00042630400000000007A6304000000000083
:1043B000C862040000000000BA60040000000000B1
:1043C0007EB104000000000092B104000000000073
:1043D00078B104000000000074B104000000000087
:1043E000C0B1040000000000BAB1040000000000E9
:1043F000D2B1040000000000CCB1040000000000B5
:10440000B2B1040000000000C6B1040000000000CA
:10441000A6B1040000000000C4B3040000000000C6
:1044200008B204000000000088B204000000000090
:104430009AB2040000000000D8B10400000000009F
:10444000B2B804000000000082B8040000000000C0
:10445000E2B804000000000072B804000000000090
:104460006CB80400000000002CB90400000000003B
:1044700032B904000000000038B904000000000058
:104480003EB90400000000001EB904000000000056
:1044900026B904000000000012B90400000000006A
:1044A00080B904000000000046BA040000000000CB
:1044B0005EBA04000000000044B9040000000000DF
:1044C0003CB00400000000006AB1040000000000DD
:1044D0001CB1040000000000F6AE04000000000063
:1044E00054AF0400000000003EB6040000000000CD
:1044F0004AB604000000000016B7040000000000E7
:104500005CB704000000000056B604000000000084
:104510005CB60400000000005E63040000000000C0
:1045200094B6040000000000EA93040000000000BC
:104530000C94040000000000D2940400000000006D
:104540001E940400000000003C96040000000000DF
:104550004093040000000000DE930400000000000F
:10456000E493040000000000C09604000000000076
:10457000A0C30400000000009CC304000000000071
:104580000040DA000000FE0003F0A200889FBE0099
:104590008A9FBE008C1F780059010700600133001C
:1045A0006450E1004F0032006420E100520032000C
:1045B00003826C0007003B000905D0000306D00011
:1045C000820F54000C065D00020039000200320028
:1045D00089017800030678008582550004003D00BB
:1045E0000003FD008103FD008502EA008B85420087
:1045F000840F720002003B0060001000E080180091
:104600006011B8000005EB007A28E1000A003900CB
:1046100006007800C75DDD00F707B20087807500EF
:104620002D003700828171000A0178006105600069
:104630008180D1000080D3008502E900F9FF3B00B2
:10464000060440008784480002003B006004140018
:10465000E0841C000988A300070032008A817100F1
:1046600082817100610164008904D1000884D30053
:104670008B05E800170037000978A30013003A0003
:104680000B00E000130034008B05E900080444002F
:1046900089844C000A4474000978A3000D003A0094
:1046A0000B00E000070034008B05E900080444001B
:1046B00089844C0001003A000B0020000978A30017
:1046C000F7FF32000001EB00020037008281710029
:1046D0000A017800CF0007000CF0A70001F0A0004D
:1046E000180137006420E10002003A00838F6C005B
:1046F000180133000801BE000200BE00110137009E
:10470000889FBE008A9FBE008C1F7800FC000700B7
:104710000301330003866C006450E1002E00320078
:104720006420E100330032006150E1002F003200CC
:104730006120E1003100320085855500EB07B000B3
:104740000900200008042000050037000804440088
:1047500089844C000A0031000603430087834B0024
:104760000001530081815B00F8FF33000203BE00AB
:104770000800A0000804440089844C00F6FF3900BA
:10478000C639DD00830173000100320013002000F0
:104790008904D1000884D3000998A30005003200E1
:1047A0000800A7000300A0008904D1000884D300FA
:1047B0008B05E8008904D1000884D3000001EB00D8
:1047C0000281D2009300070001F0A1000CF0A700C5
:1047D00001F0A000DB0037006420E100DD003200C2
:1047E0000801BE000200BE00F7FF37006120E100B3
:1047F000D80032006000B800F3FF3700000020004E
:1048000001F82700F0FF3700839F68000100E000F7
:1048100002003D0060001000E08018000300E0008E
:1048200002003D0060011100E08119000001070055
:104830004F00E00002003B0060001000E080180024
:10484000000006001400200014023700F4FF2F00BF
:10485000120237000003BE00940007006011B80088
:104860000470A70007F0A10007F8A30017003A00A2
:104870006509B1000D0032000D00350086022000F0
:104880000628E10003003500030028006000B8009E
:10489000020005000000400081804800020149003C
:1048A000838149008502E900FAFF3A000000060012
:1048B000F88F4200050034008100D1000080D30051
:1048C0008502E800FCFF3A00000006006011B80015
:1048D0008000EB00000005000001BE00730007002F
:1048E0000470A70003F0A10003F8A30013003A002E
:1048F0006509B10010003200090035006928E100A7
:104900000200350001002800000005000000400002
:10491000818048008502E900FCFF3A0000000600A3
:10492000F88F4200050035008100D1000080D300DF
:104930008502E800FCFF3A00000006008000EB0062
:10494000000005004F89DE0082017800EE0137008B
:10495000889FBE008A9FBE00008270000402710022
:1049600004827100260032000004BE000200BE0076
:104970006011B8006B092000950220000182CF0071
:104980000A0039000541B1000082CF00070039005C
:104990000541B1000982CF00040039000541B10092
:1049A0000882CF00010039000541B10005425200E4
:1049B000120032000A003B00828171006101640034
:1049C0008100D1000080D3008984D3000884D30003
:1049D0008B05E8000442E800F7FF3A0007003700C3
:1049E0000804440089844C0000004800818048008D
:1049F0008B05E9000442E900F9FF3A0005000700D1
:104A00004F05BE004F04BE00000006006011B80054
:104A1000CFFF370081002000618055000B003D0072
:104A20000B00200061FE2F000100E1001D0034009A
:104A300082817100610164008904D1000884D3007F
:104A40000000E800FAFF3A007100200061006400F5
:104A5000030070000200600009003200610444009D
:104A6000E0844C000988A500050032008B05E800B1
:104A70006808E10002003A008904D1000884D300EC
:104A8000F20F20000258E10005003D00C75DDD0087
:104A9000F907B20089807500080078000000060060
:104AA0000BF827008B00780000000500C70ADE0025
:104AB000F107B200F50FB20008003200E1CF42006A
:104AC000020032000170A00024000500810F700078
:104AD000010032000408050044000500810F700049
:104AE00002003A00140005008502E90000004000C1
:104AF00081C04800FCFF3B000170A00024000500BD
:104B00000004BE00E9FF07000003BE000405BE006C
:104B10000200BE00E5FF0700844F7500000006009C
:104B20000200BE006450E100050036006420E10090
:104B3000020036000968A30001003A000800BE0028
:104B40000160A0004F0678004F05BE004F04BE0074
:104B500000000600F0FF2F00F1FF2700F9FF3700EB
:104B6000889FBE008A9FBE008C1F7800E4FF07006C
:104B7000EBFF330003866C006450E1002400320038
:104B80006420E100270032006150E1002200320081
:104B90006120E100210032008B854200EB07B1006B
:104BA0000134B800003AB8000804420089844A0081
:104BB000013AB8000030B8008880400009014A007E
:104BC00004003300000040008180480002014900D9
:104BD0008B05E900C909DD00830170000100320086
:104BE00013002000C814DE004814DD004709DE0071
:104BF0001200B200C808DE000884700085FF0700BC
:104C000001F0A1000CF0A70001F0A000CDFF3700DB
:104C10006120E100CFFF32000801BE000200BE00AB
:104C2000F7FF37006150E100FCFF3A00C9FF370091
:104C30006022B800060220000000D0008180D2006F
:104C40000482D2008582D2000000A000020252003D
:104C500083825A00030031000202420083824A002C
:104C60000000A1000603E900F3FF3A00000006007F
:104C7000EFFF07000400BE0000000600020AB900B2
:104C8000001BB9000200B80081004200810043000F
:104C900000000600889FBE008A9FBE0030044200CC
:104CA000B0844A0030054B0090854B006000B10095
:104CB0000898BE000A90BE000440E10005C8E1006B
:104CC00006D0E10007D8E100020031006800400092
:104CD0001008E8004F05BE004F04BE0000000600AB
:104CE000889FBE008A9FBE003004BE002005BE0023
:104CF0000418540005985C0006185D0007985D00D4
:104D0000110020000440E10005C8E10006D0E100E8
:104D100007D8E100010039008000EB001088100086
:104D20004F05BE004F04BE00000006001200FA004E
:104D3000889FBE008A9FBE008C9FBE00E0B79F0088
:104D4000F1B79F0082BF9F0093BF9F000605BE0082
:104D50000404BE000000EB00D0B79F00C0B79F0066
:104D6000B0B79F00A0B79F0090B79F000006EB0070
:104D70005FB19700CFB09700820141003FB097002C
:104D80000200E00004003D00370007007E8057006D
:104D9000C0FF070003003700330007007E80570084
:104DA000CFFF0700DFB697000D00E0000C003500D4
:104DB0006FB29700FFB297000FBB97009FBB9700A1
:104DC00010002000010020006011B80000027200F5
:104DD0008182720002037300838373001B0007004B
:104DE0000C06E80001042000810F5600E0FF3A00A5
:104DF0000D00E00004003D000802BE000A03BE00F2
:104E00007E805700A3FF07005FA897000000E00026
:104E100005003A001FB29700AFB297003FB397006A
:104E2000CFB39700090007006FB09700FFB097005D
:104E30000FB997009FB997004F06BE004F05BE00FF
:104E40004F04BE000080FA000000060001000700C9
:104E500000000600A4B79F00B5B79F00C6B79F002B
:104E6000D7B79F00000006004F09DE008281710065
:104E7000B3B79F004F01DE00818040008280700048
:104E8000A1B79F008FB097004F09DE0000004000DF
:104E90000200700090B79F007FA897004F01DE00CE
:104EA000818040008280700081B79F000D00070064
:104EB0004F3ADE000000400004007000F0AF9F0099
:104EC000080007000402420085824A0006034B00E6
:104ED00087834B00DFFF07000802BE000A03BE0005
:104EE000000006002FB29700BFB297004FB39700A3
:104EF000DFB3970000000600881F7800180020002C
:104F0000881F780089FF07008F87E9004F04780029
:104F100000000600801FEB0084FF07008F87E90078
:104F200000000600889FBE008A9FBE00E00F500070
:104F3000E08F5800E00F5900E08F59000C003D0051
:104F40006044B8006055B8000000540081805C00E7
:104F500002015D0083815D0018002000150007003C
:104F600008003D00180007000004EB0005003700B2
:104F70000004EB000F00070002003D0012000700D4
:104F800018002000DCFF07000800E00006003200E7
:104F90006022B8006033B8000000520081805A00DF
:104FA00002015B0083815B004F05BE004F04BE0021
:104FB00000000600E00F5200E08F5A00E00F5B0097
:104FC000E08F5B00000006006044B8006055B80048
:104FD0000402540085825C0006035D0087835D0047
:104FE00000000600889FBE008A9FBE008C1F7800CC
:104FF000E00F5000E08F5800E00F5900E08F59009B
:105000000D003D006044B8006055B8000000540039
:1050100081805C0002015D0083815D001C00200036
:105020000820E10009A8E1000AB0E1000BB8E100A6
:105030000D003D00080037000006EB00E00F5200B5
:10504000E08F5A00E00F5B00E08F5B0006003D0040
:105050006044B8006055B8000402540085825C00CA
:1050600006035D0087835D00AAFF07000C00E000D7
:10507000060032006022B8006033B8000000520021
:1050800081805A0002015B0083815B004F0678003B
:105090004F05BE004F04BE0000000600889FBE0002
:1050A0008A9FBE00841F780095FE07004F0078009D
:1050B00011003300F0FF2F00838F6C0006003B00CF
:1050C000040565000A00A7000800370009F0A600E3
:1050D0001000200008003700820F5400838F5C000E
:1050E000030039001000200001003E0000002000F5
:1050F00009F0A7000000EA004F05BE004F04BE0003
:105100000000E00000000600881F7800030478001B
:105110000300E00007003D0060001000E080180080
:1051200060011900E081190002003B0001F02D0030
:105130000300370006FE070008F0A70001F0A000FA
:105140004F0478000000060080017800020037005C
:10515000B15978000201E9000200E000FCFF3A00CA
:10516000000006000D0A0000280000007800000082
:10517000293E000000080000200800000000000098
:105180002E20000000200000004300006C7500008D
:10519000746300006820000064690000736500000B
:1051A0006E67000061670000656400002121000057
:1051B00021000000546F000020660000696E0000AE
:1051C00069730000682000007365000074750000BA
:1051D000702C0000207300007461000072740000E5
:1051E0002075000070200000746800006520000039
:1051F000706F00007765000072200000737500007A
:10520000707000006C69000065730000207700007A
:105210006974000068200000636F00006D6D00007D
:10522000616E00006420000027570000270D000079
:105230000A00000042750000732000005069000061
:1052400072610000746500002076000034000000E8
:10525000436F00006D6D0000756E00006974000002
:105260007920000046690000726D0000776100003F
:105270007265000020760000372E0000302000000C
:105280002D200000676F00006F2E0000676C00008B
:105290002F670000437A0000516E00005720000085
:1052A0000020000028320000344600004A3200008E
:1052B0003536000047420000313000003620000043
:1052C000004100003300000041350000005500009F
:1052D0004E4B0000002900000049000009000000BA
:1052E0004F09000000480000090000004C090000C0
:1052F0000043000046470000303A00002000000054
:1053000056700000753D0000355600002C2000004E
:1053100000560000707500003D3300005633000059
:105320002C200000004500006E7400006572000033
:10533000207200006177000020760000616C0000A0
:1053400075650000206600006F72000020420000BA
:105350005247000000570000617200006E690000B3
:105360006E6700003A200000616C0000726500006A
:10537000616400007920000061200000766F000069
:105380006C74000061670000652000006F6E000013
:1053900020560000707500006C6C000075700000F5
:1053A00020700000696E0000003E0000001B00003D
:1053B0005B440000001B00005B0000004400000094
:1053C0001B5B0000430000001B5B0000324B000031
:1053D0000D000000430000001B5B00003244000091
:1053E00000570000617200006E6900006E670000E7
:1053F0003A2000006E6F0000207600006F6C000005
:105400007461000067650000206F00006E200000DE
:1054100056700000756C00006C7500007020000074
:10542000706900006E000000203D000020000000B8
:105430005245000053450000540D00000A000000D2
:10544000436C000075740000636800002065000074
:105450006E670000616700006564000021210000A4
:105460002100000056520000454700002074000053
:105470006F6F0000206C00006F7700002C20000090
:105480006973000020740000686500007265000008
:105490002061000020730000686F0000727400003B
:1054A0003F0000002E2000003C000000002E000005
:1054B000003A0000200000003157000030310000A9
:1054C000005E0000BCE20000613F0000DD830000E0
:1054D000C29C00007E200000A3FD00001F410000D0
:1054E0009DC30000217F0000FCA20000401E0000C0
:1054F0005F010000E3BD00003E60000082DC0000B0
:10550000237D00009FC10000421C0000FEA000009F
:10551000E1BF00005D03000080DE00003C6200008F
:10552000BEE00000025C0000DF810000633D00007F
:105530007C220000C09E00001D430000A1FF00006F
:1055400046180000FAA40000277900009BC500005F
:1055500084DA000038660000E5BB0000590700004F
:10556000DB85000067390000BAE40000065800003F
:1055700019470000A5FB000078260000C49A00002F
:10558000653B0000D9870000045A0000B8E600001F
:10559000A7F900001B450000C69800007A2400000F
:1055A000F8A60000441A000099C70000257B0000FF
:1055B0003A64000086D800005B050000E7B90000EF
:1055C0008CD20000306E0000EDB30000510F0000DF
:1055D0004E100000F2AC00002F71000093CD0000CF
:1055E000114F0000ADF30000702E0000CC920000BF
:1055F000D38D00006F310000B2EC00000E500000AF
:10560000AFF10000134D0000CE900000722C00009E
:105610006D330000D18F00000C520000B0EE00008E
:10562000326C00008ED00000530D0000EFB100007E
:10563000F0AE00004C12000091CF00002D7300006E
:10564000CA94000076280000ABF50000174900005E
:1056500008560000B4EA000069370000D58B00004E
:1056600057090000EBB50000366800008AD400003E
:1056700095CB000029770000F4AA0000481600002E
:10568000E9B70000550B000088D60000346A00001E
:105690002B75000097C900004A140000F6A800000E
:1056A000742A0000C8960000154B0000A9F70000FE
:1056B000B6E800000A540000D78900006B350000EE
:1056C0005245000054550000524E000000000000FA
:1056D000525500004E0000004C4900005354000099
:1056E00000450000584900005400000044450000F7
:1056F00042550000470000004E45000057000000E2
:105700004C450000540000004946000000540000D1
:10571000484500004E000000454C00005345000085
:10572000004700004F5400004F000000474F0000AA
:105730005355000042000000524500004D0000009B
:1057400050520000494E000054000000494E000035
:105750005055000054000000464F00005200000069
:10576000544F0000004E0000455800005400000057
:105770005245000041440000004400004154000034
:1057800041000000535400004152000054520000F8
:105790000053000054410000525400000053000028
:1057A000544F00005052000000530000544F0000BE
:1057B00050000000534500004E440000005200001D
:1057C00045430000454900005645000000430000E5
:1057D0004C4B000000440000415400000042000017
:1057E00049540000524500004144000000410000BF
:1057F000444300000041000055580000504900009B
:105800004E000000505300005500000050550000AD
:105810004C4C00005550000000440000454C000076
:1058200041590000004100005558000000460000AA
:10583000524500005100000044550000545900003A
:10584000004D000041430000524F000000450000A1
:105850004E440000000000001201000000020000A1
:105860000200000000080000D804000000FB000057
:105870000200000001020000030100000902000014
:1058800043000000020100000080000064090000E5
:1058900004000000000100000202000001000000FE
:1058A0000524000000100000010400002402000094
:1058B000020500002406000000010000052400008D
:1058C000010100000107000005810000030A00003B
:1058D000004000000904000001000000020A00006E
:1058E0000000000000070000050200000240000068
:1058F00000000000070500008202000040000000D8
:105900000004000003090000042A00000344000012
:1059100000610000006E00000067000000650000EC
:1059200000720000006F00000075000000730000AE
:10593000002000000050000000720000006F000016
:1059400000740000006F0000007400000079000087
:10595000007000000065000000730000001E0000E1
:1059600003420000007500000073000000200000EA
:10597000005000000069000000720000006100009B
:1059800000740000006500000020000000560000C8
:10599000003400000020000000120000033000006E
:1059A0000030000000300000003000000030000037
:1059B0000030000000300000003100000000000056
:1059C00042610000756400002064000065740000FE
:1059D00065630000746900006F6E000020730000B2
:1059E000656C00006563000074650000642E0000B3
:1059F0002E00000000200000004100005254000072
:105A00003100000014340000040D00008206000084
:105A100040030000A0010000CF0000007F00000054
:105A200067000000440000002200000000000000A9
:105A3000000000002C0100000000000058020000DF
:105A400000000000B0040000000000006009000039
:105A500000000000C01200000000000080250000CF
:105A6000000000004038000000000000004B000073
:105A700000000000807000000000000000960000A0
:105A800000000000C0DA00000000000000E100009B
:105A90000000000000C200000100000000F400004F
:105AA0000100000000E800000300000014340000C2
:105AB000040D00008206000040030000A001000069
:105AC000CF0000006700000044000000220000003A
:105AD0007F000000290000000020000057000000A7
:105AE00020520000004E00006F770000207500007B
:105AF000736900006E670000206F00006E2D0000CB
:105B0000626F0000617200006420000045450000E3
:105B1000505200004F4D0000204900003243000069
:105B2000206900006E74000065720000666100006C
:105B300063650000004F00006E2D0000626F0000E2
:105B400061720000642000004545000050520000D2
:105B50004F4D00002077000072690000746500005E
:105B600020700000726F0000746500006374000014
:105B70002064000069730000616200006C65000031
:105B8000640000004932000043310000009D000025
:105B9000250D0000204800007A0000004672000039
:105BA00065710000756500006E63000069650000A6
:105BB000732000003C200000314800007A200000E3
:105BC00061720000652000006E6F0000742000000C
:105BD00073750000707000006F7200007465000043
:105BE000642E000000000000436F0000756C000090
:105BF000646E000027740000206B000065650000E3
:105C0000702000007570000000000000535000007C
:105C10004931000000000000181C00001D030000B6
:105C20000B1300001B000000181C00001D000000EA
:105C300030300000302C0000003000003000000048
:105C40003062000000300000783000003132000087
:105C50003334000035360000373800003941000089
:105C6000424300004445000046000000314100006E
:105C70004C53000001420000507600003400000048
:105C8000210000000010000000230000000F0000B1
:105C900042400000400500004102000000000000FA
:105CA00029000000007500006E6B00006E6F0000A0
:105CB000776E0000206D00006F640000650000003A
:105CC0005049000043310000000000004242000043
:105CD000494F0000310000005853000056310000C9
:105CE000000000000808000008080000080000008C
:105CF0000000000052410000573100000000000089
:105D00004E4F0000454D0000530000000000000011
:105D1000000000002900000000000000000000005A
:105D20001398810003007800F00FB20002202300D6
:105D300062407800F1CCB30081404000E8CF5000D1
:105D400013003E000000FB000003B1001100200022
:105D5000060037006A02B90000FD2F000400400071
:105D60000201FB00020040008100E80003814000C6
:105D7000F20FB200042023006441790004CDB30087
:105D800004424100E94F5200F2FF36006000370044
:105D900001C3B300814F500059003A008300E8006E
:105DA000F10FB20062C1780021C6B300814F5100EB
:105DB00003003A000000EB0021002000090037003A
:105DC00021C4B300814F51000F003A00F9FF3700A2
:105DD000000040000003B1000201FB00020040008F
:105DE0008100E80003814000F20FB200042023008C
:105DF0006441790004CDB30004424100E14F5200F8
:105E0000F3FF36004200370081C7B300814F5100D5
:105E100003003A000000EB002100200010003700D2
:105E200081C5B300814F51001E003A00F9FF3700D1
:105E30004400DD00E9CF520002003E000003B10043
:105E4000040037000254A0000520230082727A006B
:105E50007005B1000201FB00020040008100E80073
:105E600003824000F40FB2000220230062417A0056
:105E700005CDB30085424100E9CF5200ECFF36006A
:105E8000F6CBB30006434100E54F5300E8FF360070
:105E9000F6C9B30006434100E54F5300E4FF360066
:105EA0001B003700004251000000EB0011002000F1
:105EB000E94F520016003E000200FB000003B10053
:105EC000060037006A02B90000FD2F000400400000
:105ED0000201FB00020040008100E8000381400055
:105EE000F20FB200042023006441790004CDB30016
:105EF00004424100E94F5200F2FF3600040037002F
:105F000011C0B300403023000148780000000500B4
:105F10001298810082804000F10FB2001198890030
:105F200000000600129881008200E800F10FB20024
:105F300000202300E0C1780010002000A1C3B300BE
:105F400081CF510008003A000280E800F00FB20053
:105F50001098890072FF0700119881008100E90004
:105F6000F10FB2001198890000000600129881001C
:105F70008200E800F10FB20000202300E0C17800A9
:105F80000000EB00B1C3B30081CF510008003A001C
:105F90000280E800F00FB2001098890060FF07004F
:105FA000119881008100E900F10FB2001198890079
:105FB00000000600119881008100E800F10FB20096
:105FC0000020230060C1780080C7B300804F5100DB
:105FD00002003A00119889001000050040C6B30085
:105FE000804F510002003A001198890020000500FE
:105FF00020C6B300804F510002003A00119889007A
:10600000300005000040EB0073C7B300834F510020
:1060100002003A001198890040C0B3000000060059
:1060200010988100020037000000E800F00FB20075
:10603000012023006141780001C2B300814F51006B
:10604000F9FF32001098890000000600E887470039
:10605000889FBE008A9FBE008C9FBE008E1F780066
:106060000004BE000205BE00208B2A00C8A4020066
:10607000000000000800E00004003D00608B2A00E2
:10608000C8A40200000000000300370008407800A8
:106090009AA3020000000000808B2A00C8A402001E
:1060A000000000000007EB000006EB002D003700A9
:1060B0000C00E000050032000C06E900B08B2A005D
:1060C000C8A4020000000000260037000E00E00017
:1060D00021003200B08B2A00C8A40200000000009A
:1060E0000007EB001F0037000C00E0001A003A0028
:1060F0000D4078008CA30200000000001E0020006C
:10610000180037000B00E00043003A0000CDB30058
:1061100000C04600E94F50000F003E00E30F56005C
:106120000500340070C0B3008CA302000000000022
:106130004C0020000B0037000D4078008CA30200BB
:10614000000000008D4078007480570001707E00D0
:106150000C06E8000300370070C0B3008CA30200F7
:106160000000000060A602000000000080467800E9
:10617000EDCF56000D00320005003C00E8CF560080
:10618000CBFF3200EACF5600E0FF3A0007003700AD
:10619000D0C2B30080CF5600D3FF320080C7B30017
:1061A00080CF5600D9FF3A00D6FF3700F08B2A0087
:1061B000AEA40200000000000C00E0001900320054
:1061C000F58057000000EB00040037006A01B900B9
:1061D0005100FB000003B100020040000C06E90082
:1061E000FAFF3B00890F5000060035008A0F50006F
:1061F00004003C000E00E000090032000004EA0048
:1062000008003700B101200060FE20008ABD0200B6
:106210000000000094FF37000084EB00010037000D
:1062200000047800080078004F0778004F06BE0091
:106230004F05BE004F04BE008F00B10000000600F5
:106240001E00FA00889FBE008A9FBE001998810038
:106250008904E900F90FB200180020002700370078
:1062600000202300E0C07C000104E00021003A008F
:106270000905E800FA0FB20060407D000004E0006C
:106280001C003200084078009AA3020000000000C1
:10629000008C2A00C8A40200000000001B0020009F
:1062A000030037008CA30200000000008B05E8000B
:1062B00009804500F00FB200012023006140780002
:1062C0000004E000F7FF3A00080044000A017800EB
:1062D000A1FD2F008F804000823078000804E80084
:1062E000EF0F540008003200F08B2A00AEA4020029
:1062F000000000008904E900F90FB2001098810045
:10630000808F5400D6FF3A00308C2A00AEA40200E1
:106310000000000071002000708220008ABD020091
:1063200000000000130020000801780083007800BE
:106330000000EB0045FF07008000E800E18F5000FF
:106340000700360000004000A1FD2F008F804000B4
:10635000E1027800049881000000EB00090037009A
:10636000F08B2A00AEA40200000000001000200004
:106370001600370084004000F10FB20003F17800EE
:106380000000E80085004000F10FB2000220230069
:10639000E2C178000304E000F6FF3A0001988100B2
:1063A0008100E900F10FB200119889008180E800B6
:1063B00000804000F00FB200009889000000E90062
:1063C000F00FB200037178000000EB004F05BE0033
:1063D0004F04BE000080FA0000000600889FBE0047
:1063E0008A9FBE00109881000000E800F00FB20004
:1063F000109889000AFF070049FE07000000E0002E
:1064000039003A000005EB000A40E8009AA30200B8
:1064100000000000008C2A00C8A402000000000058
:106420000903200009D0B9008002B000C8C62200CC
:1064300008004000AEA40200000000000A05E800C9
:10644000EB0F5500F0FF3A0071012000C07B2000E7
:106450008ABD020000000000403023000048EB002D
:10646000130020000A017800830078000300780000
:10647000F6FE07000005E9000000E800E10F50000B
:1064800003003E00E1002000307D20002F00370097
:1064900080A681000980B9002002B0006800780061
:1064A0000000010074BA0200000000008AA6890002
:1064B00009D0B900FE04400068807C0000000100A3
:1064C000508C2A00AEA40200000000000A00E00088
:1064D00019003200CB02A800A08D2A00AEA4020051
:1064E00000000000140037000004E900EA0F540027
:1064F00014003C000A03200080A681000A80B90035
:106500002002B000C9C62200690078000000010026
:1065100074BA02000000000088A689000AC5B9000C
:106520007E05450069007D00000001000800E000D4
:1065300001003200CB02A80051002000B06520000D
:106540000200370051012000208120008ABD020096
:1065500000000000009881000000E900F00FB20088
:10656000109889004F05BE004F04BE0000000600D1
:10657000F2874700889FBE008A9FBE008C9FBE00A6
:106580008E1F78000004BE0002057800F4B79F005B
:1065900085BF9F0003077800208B2A00C8A4020053
:1065A00000000000E00F5400E08F5C0004003D009C
:1065B000608B2A00C8A4020000000000030037001E
:1065C0000800BE004AA4020000000000808B2A00E0
:1065D000C8A40200000000008005EB000006EB00EC
:1065E0002D0037000C00E000050032000C06E90029
:1065F000B08B2A00C8A4020000000000260037006B
:106600000B00E00021003200B08B2A00C8A4020079
:10661000000000008005EB001F0037000C00E000C8
:106620001A003A000D4078008CA302000000000020
:106630001B002000180037000E00E0004E003A005A
:1066400000CDB30000C04600E94F50000F003E00EF
:10665000E90F56000500340070C0B3008CA302009F
:1066600000000000AC0020000B0037000D40780057
:106670008CA30200000000000D417800FE8057004E
:1066800082707E000C06E8000300370070C0B30083
:106690008CA302000000000060A6020000000000C1
:1066A00080467800EDCF56000D00320005003C001A
:1066B000E8CF5600CBFF3200EACF5600E0FF3A00A9
:1066C00007003700D0C2B30080CF5600D3FF32009E
:1066D00080C7B30080CF5600D9FF3A00D6FF3700FD
:1066E000F08B2A00AEA40200000000000C00E000C5
:1066F00025003200FF8657006000B800090037000F
:10670000A2002000030020003E260200000000003E
:106710005D01FB000203B100CF91DE0000004100EB
:10672000818049000C06E900F5FF3B006151B9008A
:10673000820F5000838F58000A0035007FB1970008
:106740008FB99700820F5000838F580005003C00DE
:106750000B00E0000B00320060041000E084180021
:1067600009003700B101200060FE20008ABD020050
:106770000000000088FF37000084EB008084EB00FD
:10678000010037000004BE000800BE004F0778007B
:106790004F06BE004F05BE004F04BE002F01B100E2
:1067A00000000600881F7800A0912A00AEA4020015
:1067B0000000000080922A00C8A40200000000002F
:1067C000B0C5B3008CA30200000000000004EB0081
:1067D000050037000800E0000300320000C2B300EB
:1067E0008CA30200000000000203200002C1B900D7
:1067F00041C9220001004100C8A4020000000000BD
:106800000804E800EB0F5400F2FF3A00D0C5B300D3
:106810008CA3020000000000F08B2A00AEA402004E
:1068200000000000610020009084200044BD0200B0
:106830000000000090A68100CEA50200000000002C
:1068400071002000F0FD200044BD020000000000A7
:10685000A0A68100CEA502000000000010952A002D
:10686000C8A4020000000000A0A68100E10F5000B3
:1068700003003200E30F500005003A000200370029
:1068800010962A000300370040962A0001003700C6
:1068900070962A00C8A4020000000000B0962A00EA
:1068A000AEA4020000000000E1012000F0842000FE
:1068B0008ABD0200000000004F04780000000600BE
:1068C000D802B60002003200D0962A00010037003C
:1068D00000972A00C8A4040000000000DA02B600F5
:1068E0000200320030972A000100370060972A002A
:1068F000C8A4040000000000A1002000201921000D
:106900008ABD02000000000061052000703A2100ED
:106910008ABD02000000000041022000D03F21009B
:1069200044BD0200000000000003200081A6810099
:106930000088B9004002B000C1C6220061007800A2
:1069400000000100A1002000601B210044BD0200E6
:106950000000000010002000D9FF070000102000F8
:10696000D7FF070000022000D5FF0700000120002C
:10697000D3FF070080002000D1FF07004000200067
:10698000CFFF070020002000CDFF0700F08B2A007A
:10699000AEA40200000000004100200000232100FE
:1069A00044BD02000000000021E3A80020002000F8
:1069B000D0BA020000000000E2A3020000000000C4
:1069C00011002000B037200044BD0200000000008C
:1069D00090C0B3008CA30200000000000000EB0098
:1069E000D0BA020000000000E2A302000000000094
:1069F00011002000B037200044BD0200000000005C
:106A000090C0B3008CA302000000000050002000E2
:106A1000D0BA020000000000E2A302000000000063
:106A200011002000B037200044BD0200000000002B
:106A300090C0B3008CA302000000000010002000F2
:106A4000D0BA020000000000E2A302000000000033
:106A500011002000B037200044BD020000000000FB
:106A600090C0B3008CA302000000000021E3A90045
:106A70001000200099FF07000010200097FF07007A
:106A80000002200095FF07000001200093FF07008F
:106A90008000200091FF0700400020008FFF0700CA
:106AA000200020008DFF0700F08B2A00AEA4040018
:106AB0000000000090972A00C8A402000000000017
:106AC000A17F25001000200078A302000000000034
:106AD000CEA502000000000000C2B3008CA302009B
:106AE0000000000051002000C0A3200044BD0200AF
:106AF00000000000C17F25001000200078A30200E4
:106B000000000000CEA5020000000000610020008F
:106B100010A4200044BD020000000000E17F250019
:106B20001000200078A3020000000000CEA50200A3
:106B300000000000F08B2A00AEA40200000000005C
:106B4000C1002000D08620008ABD020000000000A5
:106B500069FF0700CB22AB000300320011012000C7
:106B60000071200002003700210120001072200077
:106B700044BD020000000000C0C2B3008CA30200AC
:106B80000000000000C2B3008CA30200000000005F
:106B9000E282AB000300320041012000D06B2000F4
:106BA0000200370051012000806A200044BD02002D
:106BB00000000000C0C2B3008CA30200000000006F
:106BC00000C2B3008CA3020000000000E8A2AB00EA
:106BD00003003A0000982A00C8A402000000000048
:106BE000E882AB0003003A0090982A00C8A4020093
:106BF00000000000404B230010407800704060000F
:106C0000030032002102200090872000020037009C
:106C1000E1012000B08920008ABD020000000000D0
:106C2000404B2300104078006840600003003A00A9
:106C3000B1012000908B200002003700C10120002C
:106C4000408D200044BD020000000000C0C2B3001F
:106C50008CA302000000000000C2B3008CA302005D
:106C600000000000B10120000035210044BD0200F9
:106C700000000000304A2300104078009AA3020070
:106C800000000000F08B2A00AEA40200000000000B
:106C9000404B230010407800634060000080FB0000
:106CA000E20F50000A003200E30F50000B003200E8
:106CB000E10F500003003200510120006067200006
:106CC0000800370061012000006620000500370041
:106CD00071012000B0452100020037007101200041
:106CE000204721008ABD02000000000000032000B0
:106CF00081A681000088B9006002B000C1C62200F0
:106D00006100780000000100C1002000D086200052
:106D10008ABD040000000000109881000000E80017
:106D2000F00FB20010988900BDFC0700FCFB0700C3
:106D30000000E900E30F500002003E0070A6890049
:106D40000D003700403023000048EB0021022000F6
:106D5000D08F20008ABD0200000000008001EB00FF
:106D6000420020001100200010002000B7FC0700A6
:106D7000E14C23008008E90021012000F09120006F
:106D80008ABD040000000000881F78001098810070
:106D90000000E800F00FB20010988900A0FC070086
:106DA000DFFB07000040E900E94F500003003E0010
:106DB000C14C2300804878000D003700403023008C
:106DC0000048EB00E10B2000C09520008ABD0200C6
:106DD000000000008001EB00A20020001100200054
:106DE0009000200099FC0700C14C23008048E90076
:106DF0000044EB00C04C230091C0B30090CF1000C2
:106E000010003A0086FC0700C5FB0700004478002C
:106E10000004E0000B003A00413023008048780075
:106E200030992A00AEA40200000000008001EB00AF
:106E3000F2FF27008000EB002002200083FC070007
:106E40000044780041012000A0A120008ABD02007A
:106E50000000000011012000F03321008ABD020073
:106E6000000000004AA60200000000000004E0004C
:106E7000FCFF3200C04C230091C0B30090CF100043
:106E800003003A000840780072A6020000000000EB
:106E900070A602000000000060A6020000000000D2
:106EA00001C2B300814F5000FBFF3A004F0478004D
:106EB0000000060080A681000000E00003003A0008
:106EC000D1012000B068200006003700404B2300AD
:106ED000104078007040600008003A002102200055
:106EE000D0FB20008ABD02000000000011C0B300EA
:106EF000403023000148780000000600E8A2A80006
:106F0000E882A80020002000F6BB0200000000007C
:106F100021E3A80050002000D0BA020000000000C9
:106F200001102000810F500003003600B09A2A00A3
:106F3000AEA402000000000021E3A9001098810027
:106F40000000E800F00FB2001098890034FC070040
:106F500073FB0700413023001104E0000A003200F7
:106F60008048EB0071052000504A21008ABD0200D4
:106F7000000000008001EB00320020001100200022
:106F80001000200031FC0700E20F50000300320027
:106F9000E30F500015003A0006003700E8A2A800F1
:106FA000EA82A900E882A9004100200000C6200072
:106FB00005003700E882A800EAA2A900E8A2A9001B
:106FC00021002000B0C5200044BD020000000000E8
:106FD00091012000C04F210044BD020000000000CC
:106FE000710020005051210008003700E8A2A800DD
:106FF000E882A80091012000C04F210044BD02009A
:107000000000000081002000C05121008ABD040062
:1070100000000000EC874700889FBE008A9FBE00EA
:107020008C9FBE008E1F78000000EB001098890036
:1070300000988900004D23000008EB004030230039
:107040000048EB000000EB00080037000069EB008F
:107050008100E80003022000838F5000FBFF3A000C
:107060000000E800E50F5000050032004501DD009A
:1070700041302300010141008000EB00F3FF3700A5
:107080000000EB00309D890080EF9F008005EB0041
:107090008004EB006066B800DCB79F000007EB00DF
:1070A0000004EB000003200082A681000091B900DB
:1070B00041C9220001004100C8A4020000000000F4
:1070C00000402000614D23001100600004003200E8
:1070D000710020004065200044BD02000000000057
:1070E000509D2A00C8A4020000000000309D8100CD
:1070F0000000E000410032000000E900309D8900FE
:107100000005EB000A0037000198810002202300EF
:1071100000F178008CA30200000000000A05E800DE
:10712000009881000000E800F00FB200009889008C
:10713000309D81004500DD000000450051302300F6
:10714000614078000004E000EFFF3A000000EB002F
:10715000309D890029003700404B23001040780003
:1071600064406000240032000103200082A68100F8
:107170000191B9007A004100CAC622006A00780075
:10718000F1B79F0000000100FFB097000004E0008D
:107190001900320080A681000180B9008102200020
:1071A000808040008A80400001007800C8A402006E
:1071B00000000000509D2A00C8A40200000000004A
:1071C0001A98810000988100800F550007003A004E
:1071D000090037000020230060407D008CA30200DE
:1071E00000000000FA0FB2000A05E80000988100D4
:1071F000800F5500F7FF3A00901680004CA6020061
:10720000000000000004E000D3FF320068A6020086
:1072100000000000804078000104E000030032001C
:107220006EA6020000000000B0FF3700F1B79F001B
:1072300060A602000000000000457800FFB0970043
:10724000E84F5500200032000F003E00E24F55008D
:107250008D00320005003E000A04E000B701320054
:10726000E14F5500BC013A007F013700E54F550062
:107270008C013200E64F550090003200E44F55007B
:10728000B5013A0038003700EE4F5500F1003200EA
:1072900005003E00EA4F550091013200ED4F5500C8
:1072A000AD013A008E013700FB4F5500500032000F
:1072B000F0C7B300804F55002B003200F04F55004F
:1072C000A5013A008400370010988100808F540097
:1072D000E90132000900E90002988100828F540020
:1072E00007003A0080047800F90FB200099889007D
:1072F0000020230001F07C00B08B2A0079FF3700CA
:1073000080047800F90FB200709D2A00C8A4020022
:1073100000000000890078000005EB000E00370037
:107320000101E800E2B79F0002202300EFB19700BF
:1073300062C0790000F178000004E00001003A002A
:1073400000C2B3008CA30200000000000A05E800A0
:10735000EFB09700F10FB20000988100808F5000CD
:10736000EFFF3A001700370000988100808F54002B
:10737000C1013200890078000005EB000E003700E3
:107380000100E800E0B79F000220230080017800A0
:1073900062C0790000F178000004E00001003A00CA
:1073A00000C2B3008CA30200000000000A05E80040
:1073B000EFB09700F10FB20000988100808F50006D
:1073C000EFFF3A008100E900F10FB2000198890057
:1073D000B09D2A00C8A40200000000000A40780006
:1073E0009AA3020000000000E09D2A003DFF370044
:1073F00060A6020000000000B1C5B300814F50003C
:107400003AFF3A0060A602000000000011C4B30079
:10741000814F50003000320007003E00F0C05000A5
:10742000814F50000C003200E3C04000814F5000FB
:107430002EFF3A000E00370031C4B300814F5000D8
:107440001E003200830039008140E800814F500067
:1074500026FF3A000C00370060A602000000000082
:10746000E1C7B300814F500020FF3A00FE00370013
:1074700060A6020000000000E1C7B300814F500089
:107480001AFF3A0007013700E48F56000400340069
:107490001EBD0200000000008006EB0013FF370055
:1074A00010988100808F5400730132008904E90034
:1074B000F90FB200709D2A000AFF37000098810082
:1074C000808F54006C0132008904E800F90FB2008B
:1074D000009E2A0003FF3700129881000205E90090
:1074E000FA0FB200019881008001EB0053003700D1
:1074F0000420230064407D000004E0004D003A00B9
:107500000A00E900F00FB200644278000404E000D1
:10751000480032008301E8008B8F5100450036009F
:107520008B05E800810F510005003A000A00370082
:107530000042EB0084F178008100E900F10FB20015
:1075400003202300828F5000F9FF3A000198890040
:107550000041EB0082F178000198810009003700BA
:1075600002202300624178000204E00003003A0098
:107570000006E800FC0FB200040037000000E9003C
:10758000F00FB200810F5000F5FF3A00409E2A0034
:10759000C8A40200000000000003200082A68100B1
:1075A0000091B90041C9220001004100C8A40200B5
:1075B0000000000000402000614D23001100600029
:1075C00004003200710020004065200044BD02002C
:1075D00000000000509D2A00C8A402000000000026
:1075E0008C0478000C00370061C07C00F1B79F006C
:1075F0008CA302000000000000988100FFB09700FB
:1076000069F078000000E800F00FB20000988900EF
:107610008904E800F90FB200012023008A8F54008A
:10762000F1FF3A00099881000040EB0080F07C00F7
:10763000040037000A05E900FA0FB200810F550077
:10764000ABFF3A0000988100800F5500A7FE3A007A
:1076500009013700139881000305E900FA0FB20011
:10766000019881000001EB00540037000420230042
:1076700064407D000004E0004E003A000A00E9008A
:10768000F00FB200644278000404E00049003200C8
:107690000201E8000B02E900840F510045003A00A6
:1076A00082057800818F510005003A000A003700FA
:1076B0000042EB0004F178008100E900F10FB20014
:1076C00002202300838F5000F9FF3A0001988900BF
:1076D0008041EB0003F17800019881000900370038
:1076E00002202300624178000204E00003003A0017
:1076F0000006E800FC0FB200040037000000E900BB
:10770000F00FB200810F5000F5FF3A00409E2A00B2
:10771000C8A40200000000000003200082A681002F
:107720000091B90041C9220001004100C8A4020033
:107730000000000000402000614D230011006000A7
:1077400004003200710020004065200044BD0200AA
:1077500000000000509D2A00C8A4020000000000A4
:107760008C0478000C00370061C07C00F1B79F00EA
:107770008CA302000000000000988100FFB0970079
:1077800069F078000000E800F00FB200009889006E
:107790008904E800F90FB200012023008A8F540009
:1077A000F1FF3A00099881000040EB0080F07C0076
:1077B000040037000A05E900FA0FB200810F5500F6
:1077C000AAFF3A0000988100800F550047FE3A005A
:1077D000E18F5500A8003A00409E2A00C8A402008C
:1077E000000000000003200082A681000091B90083
:1077F00041C9220001004100C8A4020000000000AD
:1078000000402000614D23001100600004003200A0
:10781000710020004065200044BD0200000000000F
:10782000509D2A00C8A402000000000011988100A9
:1078300009988100040037000041EB0002F07C0051
:107840008904E900F90FB20000202300818F540061
:10785000F9FF3A00099889008040EB0001F07C00B4
:107860008005EB0021FE37001A9881008A8F5400B2
:1078700081003200B09D2A00C8A402000000000070
:107880000A805400F00FB2009AA30200000000002A
:10789000E09D2A00C8A402000000000019988100A1
:1078A00012FE37000A9881008A8F5400720032005D
:1078B000B09D2A00C8A40200000000000900550085
:1078C000F00FB2009AA3020000000000A09E2A0060
:1078D000C8A40200000000000998810003FE3700E0
:1078E000099881008040EB000020230001F07C001B
:1078F0008904E800F90FB20009988900F08B2A008A
:10790000AEA40200000000000E98810010988100D3
:10791000D0B79F00403023000048EB00004020001B
:10792000614D23001100600057003A008005EB0014
:107930008040EB0081EF9F005D0037008D06E8007E
:10794000F48F5600E9FD3A00CEAA020000000000C4
:107950008006EB0085013700019881000100E800F6
:10796000F00FB20012988100820F500042003200E6
:10797000FF4F550040003600E0C7B300804F550070
:107980003D003E00898F50000C003A000A4078000C
:107990008CA3020000000000099881000020230051
:1079A0000AF07C008904E800F90FB2000998890008
:1079B0008040EB0001F07C00CCFD3700B09D2A0038
:1079C000F1B79F00C8A4020000000000FFB09700BC
:1079D00009805000F00FB2009AA3020000000000DE
:1079E000A09E2A00C8A402000000000001988100A7
:1079F0000F00370001004100E2C1780013409800F9
:107A000062C078000004E00007003200F1B79F0078
:107A10008CA3020000000000C09E2A00C8A402003F
:107A200000000000FFB097008100E900F10FB200F4
:107A30000900E900F00FB20002202300808F5000FF
:107A4000ECFF3A000A40780082BF9F008CA302003E
:107A5000000000000FB997000AF17C008904E800DB
:107A6000F90FB200009881000000E800F00FB200AA
:107A7000009889009DFD370070C0B3008CA3020000
:107A80000000000099FD37009A5E0200000000002F
:107A900051002000B06520008ABD020000000000F7
:107AA0008005EB000040EB0080EF9F00E60337000D
:107AB000109881000004EB00012023006141780050
:107AC0000281FB008001EB00E1072000810F5100E3
:107AD000E08F5900B9033E0002600100BB0337008C
:107AE000B6033700B5033700B4033700B3033700DC
:107AF000B2033700B1033700B0033700AF033700DC
:107B0000AE033700B1033700AC033700AB033700D7
:107B1000AE033700A9033700A8033700A7033700D7
:107B2000A6033700A5033700A4033700A3033700DB
:107B3000A2033700A1033700A00337009F033700DB
:107B40009E0337009D0337009C0337009B033700DB
:107B50009A03370099033700980337009B033700D7
:107B60007A03370039023700FC0037000101370083
:107B70009A01370088013700900337001702370059
:107B80008E0337008D0337008C0337008F033700D7
:107B900033033700470337001F03370074023700F1
:107BA000730237007202370071023700700237002B
:107BB0006F0237006E0237006D0237006C0237002B
:107BC0006B0237007D0337007C033700A7013700C5
:107BD000B800370079033700470037000C01370041
:107BE0000201370075033700660037006701370070
:107BF0007203370071033700700337006F033700DB
:107C00006E0337006D0337006E00370073003700D6
:107C10006A033700690337006803370086003700BE
:107C200066033700650337008101370063033700BF
:107C30006203370061033700070137005F03370035
:107C40005E0337005D03370034023700FB02370064
:107C50003D023700250337000A033700570337007A
:107C6000D9003700300037003E0037003E013700B2
:107C70008E0037003200370034003700160037001E
:107C8000200037004D03370046003700580037000A
:107C90002300370049033700250037005E00370016
:107CA00046033700920237005D0137004303370077
:107CB00042033700200037001A0137003F03370026
:107CC0003E0337003D0337001A0237007F003700BC
:107CD000220237009600370059F907000004EB0034
:107CE0000000E00039033A0012988100D2B79F00EB
:107CF0000E9881003503370092BD0200000000009D
:107D000031033700A7FA07000004EB0080A68100CA
:107D10000000E0002D03320066FB07002B03370054
:107D2000AEF907002803370017FC070026033700C9
:107D3000F9FB070024033700EFFA0700220337009E
:107D4000D0820200000000001F03370080A68100DF
:107D50000000E000390132006680020000000000EF
:107D600019033700404B2300C1CFB30010C8600097
:107D700061012000006620008ABD020000000000B2
:107D800011033700414B2300114078000000A00090
:107D90000014A10080487800510120006067200095
:107DA000F5FF3700414B2300114078000000A1008F
:107DB0000014A0008048780071012000B045210027
:107DC000EDFF3700404B23009041780063C87100FD
:107DD0007101200020472100E7FF3700404B2300BE
:107DE0001034A000C1012000408D200004003700A5
:107DF000404B23001034A100B1012000908B2000E3
:107E000044BD020000000000F08B2A00AEA4020076
:107E100000000000EC02370080A681000000E000B6
:107E200006013200E282A900E082A900510120008F
:107E3000806A2000F2FF370080A681000000E00089
:107E4000FE003200404B230010407800704060007C
:107E500004003A0021022000D0FB20008ABD02006D
:107E600000000000E082A800E282A9004101200099
:107E7000D06B200044BD020000000000F08B2A00FF
:107E8000AEA402000000000021E3A8005000200082
:107E9000D0BA020000000000F1042000810F500061
:107EA0009E003E00109F2A009A00370001FC070048
:107EB000C50237000000E800F00FB20010988900FA
:107EC00057F8070096F70700080037000000E800A1
:107ED000F00FB2001098890051F8070090F70700E2
:107EE0000080FB0018BC02000000000000047800C5
:107EF00008007800FAA502000000000040A12A0056
:107F0000C8A4020000000000084078009AA3020004
:107F10000000000040A12A00C8A4020000000000E8
:107F20000840780088A5020000000000B6FF370076
:107F300080A681000000E00005003A0011C0B300F7
:107F40000140780010A10200000000009E023700EE
:107F5000A1012000106D200087FF370080A12A00BA
:107F6000C8A40200000000000004EB000DFA0700A6
:107F7000960237001CBE0200000000000004EB0067
:107F80000004E00091023200A1002000006F2000F8
:107F90008ABD02000000000040062000F6BB02007F
:107FA0000000000074BA0200000000004AA60200AF
:107FB000000000000004E000FCFF320081BF2A0046
:107FC0000140010080023700D6F707000004780066
:107FD00003003700F8850200000000000804E900F3
:107FE0000800E000FBFF3A0078023700CDF70700F9
:107FF0000004780003003700C6850200000000007E
:108000000804E9000800E000FBFF3A006F023700B7
:10801000C4F70700000478000C003700610120005D
:10802000A06F200044BD0200000000002A8602006C
:108030000000000018A6020000000000F08B2A00DB
:10804000AEA40200000000000804E9000800E000FF
:10805000F2FF3A005D02370080A681000000E000D8
:1080600076003200C922A900CB22A80021E3A80093
:1080700020002000F6BB0200000000000000EB0022
:10808000D0BA020000000000011B2000810F500048
:108090001600360020002000D0BA020000000000C8
:1080A000712B2000810F50001000360011012000BC
:1080B0000071200044BD020000000000F08B2A0087
:1080C000AEA40200000000000003200081A6810091
:1080D0000088B9000002B000C1C62200610078002B
:1080E0000000010000A22A000A003700C922A900EE
:1080F000CB22A90020A32A00AEA4020000000000A9
:10810000210120001072200044BD02000000000088
:10811000F08B2A00AEA402000000000021E3A900B9
:108120002902370080A681000000E00043003200F1
:10813000010320000180B9002002B000C1C6220066
:108140006100780000000100508C2A00AEA40200FB
:1081500000000000C922A900CB22A90021012000B3
:108160001072200026FF3700F1002000C0362000EA
:1081700044BD020000000000DEBA02000000000062
:1081800011002000B03720001DFF3700ECBA0200BC
:10819000000000000C02370062F7070000047800BE
:1081A00061002000F073200044BD020000000000C8
:1081B000080078000AA4020000000000210020004E
:1081C000507420008ABD0200000000000800780002
:1081D000CABB020000000000FB01370051F7070096
:1081E0000004780061002000F073200044BD02000C
:1081F00000000000080078000AA40200000000004F
:1082000021002000100021008ABD020000000000B3
:1082100008007800F6BB020000000000EA01370009
:10822000B0A6810000A0A000B0A68900E60137003A
:1082300080A681000000E00003003A00D101200088
:10824000B0682000CCFE37007086020000000000FD
:10825000DD013700E4C3B300844F510001003A0050
:108260008041EB008100E8000200370013C0B3003A
:108270001100200000814000F20FB2000420230012
:10828000644179000204E000F2FF3A00423023002A
:108290000349780023022000838F5000020034003D
:1082A00011C0B300014978000004EB004A302300FC
:1082B0001A04E000C5013A000000E800F00FB20027
:1082C0001098890096F60700000478001098810045
:1082D00080007800F10FB2000220230062C1780014
:1082E000D1C3B300814F51001C003A000804E900DB
:1082F000E40F540036003E000000E800F00FB2002A
:10830000109889004544DD004030230000044400FB
:10831000880078000000EB008068EB000000E800B7
:1083200002022000820F5000FBFF3A0010988100EB
:1083300003003700016C78000000E800F00FB20085
:1083400001202300E1407800E2C3B30082CF500057
:10835000F8FF3A00109889009B0137000800E00000
:1083600013003A005A30230018002000084078001B
:108370009AA302000000000020A52A00C8A4020061
:10838000000000000A007800C8A4020000000000FD
:10839000509D2A00AEA40200000000000804E8007E
:1083A0000A02B000E60F5400F0FF3A0086013700E1
:1083B0000800E900E40F500005003E00F08B2A00A1
:1083C000AEA4020000000000389D89007E01370045
:1083D00010C0B300004D78007B0137000000E800BA
:1083E000F00FB200109889004DF6070000047800E5
:1083F0000BF7070011988100F10FB2000020230055
:10840000E0C0780090C2B30080CF50006B013A000A
:108410000003200081A681000088B9007C00400094
:10842000C1C62200E10078000800780001000100C8
:1084300075FE370024C2B30084CF510001003A001A
:108440008040EB000201E8000200370011C0B300D9
:108450001200200080014100F30FB200042023002D
:10846000E4C179000304E000F2FF3A004030230049
:10847000014878000004EB000104E00053013A00D9
:10848000710020007074200044BD02000000000054
:1084900020C2B3008CA302000000000013003700CC
:1084A000119889008CA30200000000001098810040
:1084B000684078000000FB00414B230091407800A9
:1084C000E8C060000200320018BC0200000000009A
:1084D0000103200082A681000191B900E80041005B
:1084E000C2C62200E28078000100010011988100DC
:1084F0008100E800F10FB2000820230068C0780076
:1085000022C2B300824F5000E5FF3A001198890063
:108510008CA30200000000003BFE37000003200097
:1085200081A681000088B900C2C6220062007800DE
:10853000DE0037000003200081A681000088B9001A
:108540000080E800D70037000003200081A68100EA
:108550000088B90064004000D2003700000320000A
:1085600081A681000088B90066004000CD00370078
:10857000710020007074200044BD02000000000063
:10858000E7F5070000047800109881000000E9007A
:10859000F00FB2001098890062F60700000578001D
:1085A00072F607000000E0004E003200314A23005E
:1085B00080487800F1804000E80F5000020034004D
:1085C0001154A000470037001154A10045003700A6
:1085D000080078003EBB020000000000404B230072
:1085E00002C2B30090406100710050000104E0003D
:1085F00004003A0083C0B30090CF110004003A0099
:108600000A00370001C1B30090CF1000070032000C
:10861000B0C3B3008CA3020000000000304A230066
:10862000104078009AA3020000000000404B230095
:1086300010407800684060000400320008007800B4
:1086400018BC0200000000000004780000032000B5
:1086500081A681000088B90068004000C1C62200E0
:10866000E1007800080078000100010000017800B6
:1086700000C2B30082BF9F008CA302000000000074
:10868000434B230001C4B30013C060001400320048
:1086900061002000E0742000F3B79F0044BD020099
:1086A00000000000FFB197009341780068C06100AE
:1086B0000FB99700040032000200780018BC0200D5
:1086C0000000000000017800020078003EBB0200BC
:1086D0000000000000C2B3008CA3020000000000F4
:1086E0000A05E9000A00E000B9FF3A00C6FD3700BC
:1086F00061002000E074200044BD02000000000082
:108700002CF607000044780006F607000005780004
:1087100016F607000000E00008003200314A23008E
:1087200080487800F1804000E80F500002003400DB
:108730001154A000010037001154A1000804E0000A
:108740002D00320070A6810080EF9F008880FB0022
:10875000E04C23000108E900270037000003200057
:1087600081A681000088B9006A004000C1C62200CD
:108770006100780000000100414B23009140780027
:10878000E8C060000200320018BC020000000000D7
:108790003EBB020000000000404B230002C2B300B9
:1087A00090406100710050000104E00004003A00B4
:1087B00083C0B30090CF110004003A000A003700D4
:1087C00001C1B30090CF100007003200B0C3B30066
:1087D0008CA3020000000000304A23001040780003
:1087E0009AA302000000000000C2B3008CA30200A4
:1087F000000000000A05E9000A00E000D7FF3A0087
:108800000804E00080FD32000FE997000280FB00C1
:1088100070A689007CFD3700810020004075200093
:108820008ABD0200000000000003200081A6810034
:108830000088B9006C0040001A0037008100200059
:10884000C07520008ABD0200000000000003200067
:1088500081A681000088B9006E0040001100370039
:10886000E1002000407620008ABD020000000000E8
:108870000003200081A681000088B900700040003C
:1088800008003700E1002000207720008ABD0200A8
:10889000000000000003200081A681000088B900CC
:1088A00072004000C1C62200610078000000010093
:1088B00045003700C10020003073200044BD020095
:1088C000000000000003200081A681000088B9009C
:1088D00074004000C1C62200610078000000010061
:1088E00018A6020000000000370037008DF50700D1
:1088F00000047800D10020000079200044BD02006F
:1089000000000000080078003EBB020000000000EC
:10891000080037000003200081A681000088B9000C
:1089200076004000C1C6220061007800000001000E
:108930000804E9000800E000F6FF3A00F08B2A0086
:10894000AEA40200000000002000370075F507000B
:1089500000047800A1002000D079200044BD02006E
:10896000000000000E0037000003200081A68100F7
:108970000088B90078004000C1C62200610078007C
:10898000000001000080FB0018A6020000000000AB
:1089900000C2B3008CA30200000000000804E9003C
:1089A0000800E000F0FF3A000101200000782000FC
:1089B0008ABD0200000000000400370011C0B300AF
:1089C00040302300014878000004EB00109881003B
:1089D0000000E800F00FB20010988900403023003A
:1089E0001004E0000F00320051012000707A2000D6
:1089F00044BD02000000000011988100AFE997001B
:108A000003C050009AA30200000000004030230081
:108A10000048EB00F08B2A00AEA40200000000002A
:108A2000180020000098810011988100808F50006C
:108A3000050032000800E0001DFC32001E9889008D
:108A40000E98890097F9370018002000FBFF3700C7
:108A50005752490054452000424954003A20200012
:108A60002A6E650078742000636C6F00636B2000D1
:108A7000285E2900207769006C6C20007573650002
:108A8000207468006973200076616C0075654E0083
:108A90006F2064006576690063652C0020747200A5
:108AA00079202800414C4100524D290020534500B7
:108AB0004152430048206D00616372006F206600E0
:108AC00069727300744144004452450053532000BE
:108AD0004D414300524F200020302E004D61630075
:108AE000726F20006D656E00754D610063726F00DE
:108AF00020202000202031005749520045206100ED
:108B000064647200657373000D0A200020202A003F
:108B10003157490052452000524F4D0020434F002D
:108B20004D4D41004E4420004D414300524F7300D3
:108B30003A0D0A00203531002E52450041442000F4
:108B4000524F4D00202830007833330029202A006E
:108B5000666F7200207369006E676C0065206400A8
:108B60006576690063652000627573000D0A200058
:108B700038352E004D41540043482000524F4D00DF
:108B8000202830007835350029202A00666F6C00D7
:108B90006C6F7700656420006279200036346200D3
:108BA000697420006164640072657300730D0A00CB
:108BB00020323000342E53004B49500020524F00D9
:108BC0004D20280030784300432920002A666F009A
:108BD0006C6C6F00776564002062790020636F0021
:108BE0006D6D61006E640D000A20320033362E0078
:108BF000414C4100524D2000534541005243480032
:108C00002028300078454300290D0A002032340026
:108C1000302E53004541520043482000524F4D0032
:108C2000202830007846300029414C0041524D0048
:108C30002053450041524300482028003078450029
:108C40004329530045415200434820002830780012
:108C50004630290044657600696365002049440078
:108C6000732061007265200061766100696C6100AB
:108C7000626C650020627900204D410043524F0034
:108C80002C20730065652000283029002E524500F5
:108C900041442000524F4D002028300078333300EB
:108CA000293A20004D41540043482000524F4D00C6
:108CB000202830007835350029534B0049502000DA
:108CC000524F4D00202830007843430029556E0054
:108CD0006B6E6F00776E20006D616300726F2C0009
:108CE0002074720079203F00206F7200202830002D
:108CF000292066006F72200068656C007042550084
:108D000053205200455345005420570061726E00B5
:108D1000696E67003A202A0053686F007274200061
:108D20006F7220006E6F200070756C006C2D7500E6
:108D300070202A004E6F200064657600696365002C
:108D4000206465007465630074656400204453000A
:108D500031385300323020004869670068205000E5
:108D600072657300204469006720540068657200D2
:108D70006D445300313842003230200050726F0091
:108D80006720520065732000446967002054680022
:108D900065726D0044533100383232002045630063
:108DA0006F6E2000446967002054680065726D0092
:108DB0004453320034303400204563006F6E72003B
:108DC000616D200074696D00652043006869700062
:108DD000445332003433310020314B0020454500EC
:108DE00050524F004D556E006B6E6F00776E200035
:108DF000646576006963650050574D002064690022
:108E0000736162006C656400314B48007A2D340058
:108E10002C303000304B48007A205000574D46002F
:108E20007265710075656E0063792000696E2000BF
:108E30004B487A002050720065736300616C6500D6
:108E40003A505200323A4400757479002063790038
:108E5000636C650020696E002025200050574D008E
:108E6000206163007469760065455200524F5200DC
:108E70003A205000574D2000616374006976650008
:108E80002C20670020746F00206469007361620009
:108E90006C6541005558200046726500717565008B
:108EA0006E6379003A20410055582000494E500029
:108EB00055542F0048492D005A415500582048006C
:108EC0004947480041555800204C4F0057564F0025
:108ED0004C544D004554450052204D004F44450030
:108EE000564F4C005441470045205000524F42001D
:108EF000453A200056457200726F72002829200002
:108F0000406C69006E653A0020407000676D730028
:108F100070616300653A20006279740065732E0009
:108F2000546F6F00206C6F006E67210053796E00E4
:108F30007461780020657200726F72004E6F2000BD
:108F400045455000524F4D004572610073696E00F7
:108F500067646F006E655300617669006E6720007C
:108F6000746F2000736C6F00742049006E7661008E
:108F70006C69640020736C006F744C006F61640056
:108F8000696E6700206672006F6D2000736C6F0061
:108F90007420450052524F00523A2000636F6D001A
:108FA0006D616E0064206800617320006E6F2000A8
:108FB000656666006563740020686500726541003F
:108FC000434B4E0041434B00493243002053540071
:108FD000415254002042490054493200432053007A
:108FE000544F5000204249005449320043206D0044
:108FF0006F6465003A0D0A0020312E0020536F0087
:1090000066747700617265000D0A2000322E200020
:1090100048617200647761007265530065742000D6
:109020007370650065643A000D0A2000312E20003F
:109030007E354B00487A0D000A2032002E207E003B
:1090400035304B00487A0D000A2033002E207E0078
:10905000313030004B487A000D0A2000342E2000B9
:109060007E343000304B48007A574100524E490060
:109070004E473A00204841005244570041524500B3
:10908000204932004320690073206200726F6B0038
:10909000656E20006F6E20007468690073205000B8
:1090A0004943210020285200455620004133290021
:1090B0005365740020737000656564003A0D0A0002
:1090C00020312E0020313000304B48007A0D0A004C
:1090D00020322E0020343000304B48007A0D0A0038
:1090E00020332E0020314D00487A490032432000C1
:1090F000286D6F0064207300706429003D282000F3
:1091000020302E004D616300726F20006D656E008F
:10911000750D0A0020312E0037626900742061004D
:10912000646472006573730020736500617263008C
:10913000680D0A0020322E004932430020736E0071
:109140006966660065720D000A2033002E436F00C9
:109150006E6E650063742000746F20006F6E2D00CA
:10916000626F61007264200045455000524F4D000F
:109170000D0A2000342E45006E6162006C652000EF
:109180005772690074696E0067207400686520007A
:109190006F6E2D00626F61007264200045455000C3
:1091A000524F4D005365610072636800696E67003D
:1091B00020493200432061006464720065737300CB
:1091C00020737000616365002E2046006F756E008D
:1091D0006420640065766900636573002061740033
:1091E0003A536E0069666600657243006F6D6D00EC
:1091F000616E64006D6F6400653F0D000A312E00E2
:10920000203662002F313400620D0A00322E200019
:1092100034622F003136620044656C0061793F0092
:1092200050494300286D6F00642064006C79290068
:109230003D2843004D44440054416E006F207200AD
:1092400065616400756E6B006E6F77006E206D0057
:109250006F64650028312900206765007420640070
:10926000657649004444650076494400203D20006D
:109270002052650076203D00204E6F00742069006A
:109280006D706C00656D65006E746500642028006B
:109290007965740029506C00656173006520650074
:1092A000786974002050490043207000726F670095
:1092B00072616D006D696E0067206D006F646500FE
:1092C00028424100534943002952650061647900F6
:1092D000612F41002F402000636F6E0074726F0099
:1092E0006C73200041555800207069006E612F009A
:1092F000412F400020636F006E7472006F6C73002A
:1093000020435300207069006E436F006D6D610053
:109310006E6420006E6F7400207573006564200019
:10932000696E20007468690073206D006F646500C9
:1093300050756C006C2D75007020720065736900AB
:1093400073746F00727320004F46460050756C00B6
:109350006C2D7500702072006573690073746F0066
:10936000727320004F4E5300656C66002D746500CB
:1093700073742000696E200048695A00206D6F00E8
:10938000646520006F6E6C007952450053455400AF
:10939000424F4F00544C4F0041444500524155004C
:1093A000582049004E505500542F4800492D5A006E
:1093B0002C205200454144003A2050004F574500B0
:1093C00052205300555050004C49450053204F0047
:1093D0004E504F00574552002053550050504C00FE
:1093E00049455300204F4600464441005441200067
:1093F0005354410054453A00204445004C41590023
:10940000207573005752490054453A0020524500D8
:1094100041443A0020434C004F434B002C20310084
:10942000434C4F00434B2C0020304400415441003A
:10943000204F550054505500542C20003144410019
:10944000544120004F555400505554002C203000FA
:10945000202A7000696E2000697320006E6F77000B
:10946000204869005A434C004F434B0020544900A8
:10947000434B53003A2052004541440020424900EA
:10948000543A200053796E007461780020657200B0
:10949000726F7200206174002063680061722000A6
:1094A000782E200065786900742877006974680058
:1094B0006F75740020636800616E670065296E0037
:1094C0006F206D006F64650020636800616E670047
:1094D00065233A00204E6F0020736F00667477009A
:1094E000617265002072650073657400206F6E0004
:1094F000207634002C2075007365200074686500A8
:1095000020726500736574002062750074746F00CA
:109510006E2E4E006F6E65007869730074656E0084
:1095200074207000726F74006F636F006C2178009C
:109530002E206500786974000D0A49006E7661007E
:109540006C696400206368006F696300652C20000B
:10955000747279002061670061696E0044455600AD
:1095600049443A0068747400703A2F002F64610017
:109570006E676500726F7500737072006F746F00B4
:109580007479700065732E00636F6D002A2D2D00B5
:109590002D2D2D002D2D2D002D2D2A004F70650015
:1095A0006E206400726169006E206F007574700037
:1095B00075747300202848003D4869002D5A2C001E
:1095C000204C3D00474E4400294E6F00726D6100F3
:1095D0006C206F007574700075747300202848004B
:1095E0003D332E0033762C00204C3D00474E440086
:1095F000294D53004220730065743A00204D4F00FE
:10960000535420007369670020626900742066006B
:1096100069727300744C53004220730065743A0001
:10962000204C4500415354002073690067206200BC
:10963000697420006669720073742000426F6F00C5
:10964000746C6F00616465007220760020312E001A
:1096500020484500580D0A0020322E0020444500C5
:10966000430D0A0020332E00204249004E0D0A000F
:1096700020342E00205241005744690073706C0062
:1096800061792000666F72006D617400207365005F
:1096900074566F006C746100676520006D6F6E001A
:1096A00069746F0072733A00203556003A2020002A
:1096B0007C2033002E3356003A2020007C205600B8
:1096C00050554C004C5550003A2053006574200012
:1096D0007365720069616C0020706F007274200005
:1096E0007370650065643A00202862007073290079
:1096F0000D0A2000312E2000333030000D0A2000EA
:10970000322E200031323000300D0A0020332E007E
:109710002032340030300D000A2034002E20340076
:10972000383030000D0A2000352E20003936300048
:10973000300D0A0020362E00203139003230300042
:109740000D0A2000372E20003338340030300D0051
:109750000A2038002E20350037363000300D0A0040
:1097600020392E002031310035323000300D0A0012
:1097700031302E0020496E00707574002043750052
:1097800073746F006D204200415544000D0A310092
:10979000312E2000417574006F2D42006175640008
:1097A000204465007465630074696F006E202800B2
:1097B0004163740069766900747920005265710014
:1097C000756972006564290041646A0075737400EC
:1097D00020796F0075722000746572006D696E00EB
:1097E000616C410072652000796F7500207375000F
:1097F00072653F002043460047313A00204346004F
:1098000047323A00285C2D002F5F5C002D2928008C
:109810005C5F2F002D295300656C65006374200088
:109820006F757400707574002074790070653A006B
:109830000D0A2000312E20004F7065006E2064005C
:10984000726169006E202800483D4800692D5A0069
:109850002C204C003D474E0044290D000A203200C8
:109860002E204E006F726D00616C200028483D0074
:10987000332E3300562C20004C3D47004E44290027
:1098800052325700202873007064200068697A0003
:10989000293D2800202030002E4D610063726F00AA
:1098A000206D65006E750D000A2031002E495300B1
:1098B0004F37380031362D003320410054520D000F
:1098C0000A2032002E4953004F37380031362D0020
:1098D000332070006172730065206F006E6C790038
:1098E00049534F002037380031362D0033204100D6
:1098F000545220002852450053455400206F6E00FA
:1099000020435300290D0A005245530045542000BE
:1099100048494700482C2000434C4F00434B20004F
:10992000544943004B2C200052455300455420001D
:109930004C4F570049534F002037380031362D0027
:109940003320720065706C00792028007573650003
:109950007320630075727200656E7400204C5300B2
:109960004220730065747400696E6700293A200014
:1099700050726F00746F63006F6C3A002073650063
:10998000726961006C3320007769720065322000D3
:10999000776972006552460055756E006B6E6F00F8
:1099A000776E5200656164002074790070653A003A
:1099B00020746F0020656E0064766100726961003A
:1099C000626C6500206C65006E677400684461001D
:1099D00074612000756E690074733A00206E6F0028
:1099E00020696E0064696300617469006F6E4400F1
:1099F0006174610020756E00697420006C656E00F2
:109A0000677468002028620069747300293A200096
:109A100043532000454E4100424C4500444353000F
:109A200020444900534142004C4544005233570002
:109A3000202873007064200063736C002068690044
:109A40007A293D00282029000D0A4400697363002B
:109A50006F6E6E006563740020616E007920640093
:109A600065766900636573000D0A43006F6E6E00D2
:109A7000656374002028410044432000746F200077
:109A80002B332E0033562900437472006C4155006D
:109A9000584D4F00444520004C45440050554C0063
:109AA0004C55500020485000554C4C00555020005B
:109AB0004C5652004547410044432000616E64000B
:109AC0002073750070706C00793556005650550043
:109AD000332E330056414400434275007320680022
:109AE0006967680042757300204869002D5A20009C
:109AF0003042750073204800692D5A0020314D0016
:109B00004F4445002C205600524547002C20610050
:109B10006E64200055534200204C450044732000E1
:109B200073686F00756C640020626500206F6E00C2
:109B300021466F00756E64002020650072726F0010
:109B400072732E004D4F530049434C004B4D49005A
:109B5000534F430053204F004B20460041494C00D7
:109B60005365740020737000656564003A0D0A0047
:109B700020312E00203330004B487A000D0A20009F
:109B8000322E2000313235004B487A000D0A200079
:109B9000332E2000323530004B487A000D0A200069
:109BA000342E2000314D48007A436C006F636B0007
:109BB00020706F006C617200697479003A0D0A00C0
:109BC00020312E00204964006C6520006C6F770006
:109BD000202A640065666100756C74000D0A20001F
:109BE000322E200049646C006520680069676800B7
:109BF0004F7574007075740020636C006F636B00A8
:109C00002065640067653A000D0A2000312E2000AF
:109C100049646C00652074006F2061006374690002
:109C200076650D000A2032002E2041006374690021
:109C300076652000746F200069646C0065202A003E
:109C40006465660061756C0074496E00707574001F
:109C5000207361006D706C00652070006861730096
:109C6000653A0D000A2031002E204D006964640021
:109C70006C6520002A646500666175006C740D00D7
:109C80000A2032002E2045006E6453005049200007
:109C900028737000642063006B702000736B650094
:109CA00020736D0070206300736C200068697A0077
:109CB000293D2800202030002E4D610063726F0086
:109CC000206D65006E750D000A2031002E536E0068
:109CD0006966660020435300206C6F00770D0A0010
:109CE00020322E00536E690066662000616C6C00A5
:109CF000207472006166660069632D0070202D007B
:109D000066202A00427974006573200064726F0037
:109D100070706500642A460041494C0045442C009F
:109D2000204E4F00204441005441440061746100C2
:109D30002062690074732000616E6400207061000D
:109D400072697400793A0D000A2031002E20380023
:109D50002C204E004F4E4500202A640065666100AD
:109D6000756C7400200D0A0020322E0020382C0063
:109D700020455600454E20000D0A2000332E2000BD
:109D8000382C20004F444400200D0A0020342E00BF
:109D900020392C00204E4F004E455300746F700048
:109DA0002062690074733A000D0A2000312E2000F1
:109DB00031202A006465660061756C00740D0A002C
:109DC00020322E00203252006563650069766500FE
:109DD00020706F006C617200697479003A0D0A009E
:109DE00020312E00204964006C65200031202A00BB
:109DF0006465660061756C00740D0A0020322E00E7
:109E0000204964006C652000305541005254200008
:109E10002873700064206200726720006462700022
:109E2000207362002072780070206800697A29002F
:109E30003D28200020302E004D616300726F20000D
:109E40006D656E00750D0A0020312E0054726100A0
:109E50006E737000617265006E742000627269003A
:109E6000646765000D0A2000322E4C00697665009B
:109E7000206D6F006E6974006F720D000A20330050
:109E80002E4272006964670065207700697468007B
:109E900020666C006F772000636F6E0074726F0035
:109EA0006C0A0D0020342E00417574006F204200B2
:109EB00061756400204465007465630074696F0017
:109EC0006E2028004163740069766900747920006F
:109ED0004E656500646564002955410052542000B8
:109EE00062726900646765005265730065742000E2
:109EF000746F200065786900745261007720550006
:109F00004152540020696E00707574005541520032
:109F100054204C00495645002044490053504C0001
:109F200041592C00207D2000544F200053544F00F5
:109F3000504C49005645200044495300504C4100C4
:109F400059205300544F500050454400574152008F
:109F50004E494E00473A200070696E0073206E0033
:109F60006F7420006F7065006E206400726169007C
:109F70006E20280048695A002920520045564900A1
:109F8000443A0D000A496E0076616C006964200055
:109F900063686F00696365002C207400727920008B
:109FA00061676100696E6D0073525300204C4F0071
:109FB000572C2000434F4D004D414E0044204D0092
:109FC0004F4445005253200048494700482C200088
:109FD0004441540041204D004F4445004164640019
:109FE0007265730073206F0066205000434638008E
:109FF000353734003F546800697320006D6F64008A
:10A0000065207200657175006972650073206100DA
:10A010006E20610064617000746572004C434400FE
:10A020002074790070653A000D0A2000312E20005E
:10A0300048443400343738003020280075736900F4
:10A040006E67200050434600383537003420490001
:10A050004F206500787061006E64650072294C00C5
:10A060004344200028747900702061006464720009
:10A0700029203D002028200020302E004D61630063
:10A08000726F20006D656E00750D0A0020312E0084
:10A090004C43440020526500736574000D0A200093
:10A0A000322E49006E697400204C4300440D0A00B2
:10A0B00020332E00436C6500617220004C43440045
:10A0C0000D0A2000342E4300757273006F72200059
:10A0D000706F7300697469006F6E200065783A00D4
:10A0E0002834290020300D000A2036002E57720037
:10A0F0006974650020746500737420006E756D00CE
:10A100006265720073206500783A280036292000C5
:10A1100038300D000A2037002E5772006974650030
:10A1200020746500737420006368610072616300CD
:10A130007465720073206500783A28003729200082
:10A1400038304400697370006C617900206C6900DC
:10A150006E6573003A0D0A0020312E002031200078
:10A160000D0A2000322E20004D756C0074697000BD
:10A170006C6549004E495400434C45004152430030
:10A18000555253004F522000534554004E6F20004B
:10A1900041434B002C206300686563006B20610025
:10A1A0006461700074657200434C4B00094D4F00B0
:10A1B00053490900435309004D4953004F5069006A
:10A1C0006E73740061746500733A47004E44090071
:10A1D000332E3300560935002E3056000941440015
:10A1E00043095600505509004155580009500900CF
:10A1F000500950000949090049092D00094F57002D
:10A2000044092D00092D2D000954780044092D0022
:10A2100009527800445343004C095300444109005B
:10A220002D092D00504743000950470044092D00D7
:10A23000092D31002E28420052290900322E280013
:10A240005244290009332E00284F520029093400B6
:10A250002E28590057290900352E2800474E29007D
:10A2600009362E0028424C00290937002E285000BC
:10A2700055290900382E28004752290009392E0097
:10A2800028575400290930002E2842006C6B290001
:10A29000474E440009474E00440941004443090029
:10A2A000352E3000560933002E3356000956500023
:10A2B00055094100555809006578650063757400BB
:10A2C00065203A0020205400494D45004F55540068
:10A2D00020302E00204D610063726F00206D6500FC
:10A2E0006E750D000A2031002E204C006976650045
:10A2F00020696E0070757400206D6F006E697400C7
:10A300006F7249006E70750074206D006F6E690089
:10A31000746F72002C2061006E7920006B657900EB
:10A320002065780069747300202A730074617200DC
:10A33000746269007420650072726F0072202A00D6
:10A34000706172006974790020657200726F72002A
:10A35000202A7300746F70006269740020657200B7
:10A36000726F7200204E4F004E452000554E4B003C
:10A370004E4F57004E20450052524F005220610070
:10A3800075746F0072616E00676520002B4D480088
:10A390007A292B006B487A0029496E007075740089
:10A3A0002061200063757300746F6D0020424100CE
:10A3B0005544200072617400653A570041524E00C6
:10A3C000494E47003A2050006F73730069626C0079
:10A3D000652062007566660065726F0076657200C2
:10A3E000666C6F0077416E0079206B006579200004
:10A3F000746F2000657869007453700061636500B4
:10A4000020746F0020636F006E7469006E756500C4
:10A410004E756D0062657200206F660020626900F3
:10A420007473200072656100642F77007269740094
:10A43000653A200043533A000D0A2000312E2000D7
:10A4400043530D000A2032002E202F0043532000DA
:10A450002A646500666175006C7450006F73690052
:10A4600074696F006E2069006E2064006567720079
:10A470006565730053657200766F20006163740038
:10A480006976650023313200202020002009230056
:10A49000313120002020200009233100302020000D
:10A4A000202009002330390020202000092330001B
:10A4B0003820200020092300303720002020090008
:10A4C00023303600202020000923300035202000D2
:10A4D00020092300303420002020090023303300DD
:10A4E00020202000092330003220200020092300F2
:10A4F00030312000202047004E440900352E300026
:10A50000560933002E3356000956500055094100B4
:10A510004443090041555800320941005558310063
:10A52000094155005809430053094D0049534F0054
:10A5300009434C004B094D004F5349002D092D0094
:10A54000092D09004F5744002D0952007844090095
:10A550002D09540078442D00092D090053434C0067
:10A5600009534400412D09002D09500047430900BB
:10A5700050474400612F41002F402000636F6E0060
:10A5800074726F006C7320004155580031207000C8
:10A59000696E61002F412F00402063006F6E7400D0
:10A5A000726F6C00732041005558320020706900B2
:10A5B0006E45450050524F004D5343004C534400EC
:10A5C000415750005245410044265700524954001B
:10A5D0004556750073625300656C65006374200016
:10A5E0005670750020285000756C6C00757029003D
:10A5F00020536F0075726300653A0D000A20310028
:10A600002920450078746500726E61006C20280076
:10A610006F7220004E6F6E0065290D000A20320017
:10A6200029204F006E626F006172640020332E009B
:10A6300033760D000A20330029204F006E626F0030
:10A640006172640020352E00307620006F6E2D0080
:10A65000626F61007264200070756C006C75700030
:10A6600020766F006C74610067652000656E610084
:10A67000626C650064646900736162006C6564000B
:10A680004E6F72006D616C0020746F002065780061
:10A690006974570061697400696E67002061630026
:10A6A00074697600697479002E2E2E002A2A200003
:10A6B000456172006C7920004578690074212A0098
:10A6C0002A204200617564003E3136006D3A200058
:10A6D0005468650020425000206361006E6E6F0078
:10A6E00074206D0065617300757265002061620001
:10A6F0006F76650020313600303030003030300069
:10A700002C2044006F6E65002E0A0D0043616C0022
:10A7100063756C0061746500643A2000090A0D00DD
:10A7200045737400696D6100746564003A2020000F
:10A730000920620070734700656E650072616C00ED
:10A740000909090009095000726F74006F636F00F6
:10A750006C2069006E7465007261630074696F003B
:10A760006E2D2D002D2D2D002D2D2D002D2D2D008C
:10A770002D2D2D002D2D2D002D2D2D002D2D2D00BD
:10A780002D2D2D002D2D2D002D2D2D002D2D2D00AD
:10A790002D2D2D002D2D2D002D2D2D002D2D2D009D
:10A7A0002D2D2D002D2D2D002D2D2D002D2D2D008D
:10A7B0002D2D2D002D2D2D002D2D2D002D2D2D007D
:10A7C0002D2D2D002D3F090054686900732068006D
:10A7D000656C70000909090028302900094C6900DE
:10A7E000737420006375720072656E0074206D00D2
:10A7F000616372006F733D00582F7C00580943005D
:10A800006F6E760065727400732058002F726500B9
:10A8100076657200736520005809090028782900C0
:10A82000094D610063726F0020787E000953650056
:10A830006C66740065737400090909005B095300B4
:10A8400074617200746F090053657400206F7500A5
:10A85000747075007420740079706500090909002E
:10A860005D095300746F700024094A00756D700013
:10A8700020746F0020626F006F746C006F61640061
:10A8800065720900097B090053746100727420002D
:10A89000776974006820720065616400262F2500C6
:10A8A000094465006C6179002031200075732F0028
:10A8B0006D73090009097D00095374006F70610010
:10A8C0002F412F004009410055585000494E2000AB
:10A8D000286C6F00772F4800492F520045414400F3
:10A8E00029090900226162006322090053656E0094
:10A8F00064207300747269006E676200095365001A
:10A900007420620061756400726174006509090059
:10A910000931320033095300656E640020696E000E
:10A92000746567006572200076616C007565630070
:10A930002F432F006B2F4B00094155005820610019
:10A9400073736900676E6D00656E740020284100A6
:10A95000302F4300532F4100312F4100322909008D
:10A96000307831003233090053656E00642068008E
:10A970006578200076616C00756564002F440900DD
:10A980004D656100737572006520410044432000ED
:10A99000286F6E0063652F00434F4E00542E290030
:10A9A0000930620031313000095365006E642000C7
:10A9B00062696E0061727900207661006C756500D5
:10A9C00066094D006561730075726500206672004E
:10A9D00065717500656E630079090900720952009E
:10A9E00065616400672F5300094765006E6572005A
:10A9F00061746500205057004D2F5300657276003A
:10AA00006F0909002F0943004C4B2000686968005A
:10AA100009436F006D6D61006E64680069737400B6
:10AA20006F727900090909005C0943004C4B200052
:10AA30006C6F690009566500727369006F6E69007A
:10AA40006E666F002F7374006174750073696E0019
:10AA5000666F0900095E0900434C4B0020746900D1
:10AA6000636B6C002F4C0900426974006F726400C4
:10AA700065722000286D7300622F4C00534229003C
:10AA800009092D000944410054206800696D09003E
:10AA9000436861006E676500206D6F0064650900A2
:10AAA00009095F000944410054206C006F650900EA
:10AAB00053657400205075006C6C750070204D005B
:10AAC000657468006F640900092E09004441540050
:10AAD00020726500616470002F50090050756C0091
:10AAE0006C7570002072650073697300746F72007A
:10AAF000732028006F6666002F4F4E002909210041
:10AB00000942690074207200656164007309530092
:10AB10006372690070742000656E6700696E65007D
:10AB2000090909003A095200657065006174200046
:10AB3000652E67002E2072003A31300076095300EE
:10AB4000686F770020766F006C7473002F73740049
:10AB500061746500730909003B0942006974730060
:10AB600020746F002072650061642F0077726900A5
:10AB700074652000652E67002E2030007835350082
:10AB80003B3277002F5709005053550020286F00A3
:10AB900066662F004F4E290009093C00783E2F00C1
:10ABA0003C783D00203E2F003C303E0009557300AC
:10ABB00065726D00616372006F2078002F61730011
:10ABC000736967006E2078002F6C69007374200031
:10ABD000616C6C0020438100C186220061417800D5
:10ABE00031C8B300814F510007003A000000E8006F
:10ABF000C18622006141780001CEB300814F51002F
:10AC0000FAFF36002043890000000600800178002A
:10AC10000000EB00C18622006141780004CEB30041
:10AC2000844F51000D0036000002E80061427A00B6
:10AC30004822DD008082E800E1C07A008180FB00CC
:10AC400081004200818F5100050032000281FB002B
:10AC5000D20DB10002004000EEFF37000080EB0093
:10AC600000000600881F7800E1000700000478005B
:10AC700020438100C1862200E1407800D2C2B300A7
:10AC800082CF50001000320002C1E90082CF500094
:10AC90000D0032007141410082CF50000A003200A5
:10ACA00002C1E80082CF5000070032000241E900F3
:10ACB00082CF500004003200204389000800780051
:10ACC0004F047800000006000000E800C2C3B30093
:10ACD00082CF50002700320007003E007141510032
:10ACE00082CF50000F00320002C1E80082CF500036
:10ACF000E0FF3A0007003700D2C3B30082CF500014
:10AD00003E003200E3C3B30083CF5000D9FF3A00C6
:10AD10000800370020438900B500070000045400F4
:10AD2000D3FF370020438900B1000700000444002E
:10AD3000CFFF3700204389000000E800C1862200D1
:10AD400061407800824F500005003A00A8000700DB
:10AD500011002000800F54001C0031001A00370041
:10AD6000A300070011002000800F540021003E00C6
:10AD70001F003700204389000000E800C186220040
:10AD800061407800E1C3B300814F500007003A00F2
:10AD90009700070000046C0008F0A7000804EA0010
:10ADA0000804EA004F44DE0009003700D1C3B300B5
:10ADB000814F50000A003A008D000700110020006A
:10ADC000800F5400010036008000EB000104780081
:10ADD000204381000000E80020438900A4FF3700E1
:10ADE0008300070011002000800F5400010039008B
:10ADF0008000EB00010478009DFF370020438900AC
:10AE00007B00070000046C0008F0A7000804EA00BB
:10AE10000804E9004F44DE0095FF3700881F7800E2
:10AE200021438100C886220068C1780080C2B30037
:10AE3000804F510009003A008100E8002143890059
:10AE400088FF070021438100E8C1780092C2B30067
:10AE500082CF510064003A0009003700F0CBB30004
:10AE600000404100F94F500008003E000281FB0005
:10AE70001204B1000201410040802200600079000C
:10AE80008100E80021438900570037000000EB00F3
:10AE900003C8B300834F51004B0036008100E80027
:10AEA000214389000280FB008000EB003009B100E3
:10AEB0000180B100EA0F5000E08F580049003E00C9
:10AEC000006001000F00370009003700450037001F
:10AED000180037001F0037003000370041003700EE
:10AEE00025003700280037003E0037000E003700ED
:10AEF0000003200081A681000088B9006A0040009C
:10AF0000100037000003200081A681000088B900EE
:10AF100068004000C1C622006104780051FF0700AC
:10AF200008000100300037002A86020000000000FF
:10AF30002D0037000003200081A681000088B900A1
:10AF400074004000C1C622006100780000000100CA
:10AF5000250037000003200081A681000088B90089
:10AF600078004000C1C622006100780000000100A6
:10AF70000080FB001C003700501680004900DE00F6
:10AF80006100600018003700101780004400DE00E8
:10AF9000610060000080EA001300370021E3A80090
:10AFA00010002000D0BA02000000000021E3A90038
:10AFB0000D0037006A02B9000280FB000003B100F7
:10AFC000040040008100E800C286220062C17800CF
:10AFD00003CDB30083414100E9CF5100F5FF3600B6
:10AFE000A8FF37000000EB004F04780000000600C7
:10AFF000889FBE0089FF070000047800214381007C
:10B00000C086220060C07800A2C2B300824F500008
:10B010000D00320065414100824F50000A003200AD
:10B0200069415100824F500007003200C2C7B3008F
:10B03000824F50000400320021438900080078004C
:10B040004F04BE00000006008100E800A2C2B30069
:10B05000824F50000C00320004003E006441510059
:10B06000824F5000E6FF3A0011003700F2C2B300F1
:10B07000824F500008003200C2C7B300824F500018
:10B08000DFFF3A000E0037002143890063FF07000D
:10B0900000C4B900D9FF3700214389005FFF0700D2
:10B0A00080017800110009000304D800D2FF3700A6
:10B0B0002143890059FF070000046400CFFF3700D7
:10B0C0002143890055FF070008047000CBFF3700BB
:10B0D000889FBE008A9FBE008C1F78000000EB0096
:10B0E0002043890030438900404389005043890050
:10B0F000B0A681000080A000B0A6890020802200B8
:10B1000041032000808040000028EB00810F5000A8
:10B11000FDFF3A008004EB0021438100C08622003D
:10B1200060C5780028002000F2CDB300824F5500A2
:10B130005F0236000A85FB000A0EB1000101E8003B
:10B14000E0447900C84CDD008880400060C0780091
:10B150000080FB008904700020438100E300400070
:10B16000C486220064C178000281FB008001EB00EC
:10B170000208B1000380B10015022000850F5100C4
:10B18000E08F59006A023E00026001002100370092
:10B190002C00370066023700650237004500370093
:10B1A000470037005A003700860137006600370035
:10B1B000B1003700E70037005D023700200137009B
:10B1C0003F0137007F0137008901370080013700D8
:10B1D000950137008D0137009A013700540237007E
:10B1E000F9013700EA0137005102370050023700F9
:10B1F000B5013700A90137000E02370018023700E9
:10B200009B013700B9013700C70137001A02370028
:10B2100045023700E60040002143890064004000F9
:10B22000C1862200614478000884FB001804B10044
:10B230008CFE0700080444004180220080307C001E
:10B2400017023700640040002043890085FE070094
:10B2500080007800204381000100E00009003200F6
:10B26000C1862200614178008000E8002143890006
:10B2700021C8B300814F5100A7FF3A0006003700F4
:10B280000000E800C1862200E140780032C8B30027
:10B2900082CF500003003A000080E900204389007B
:10B2A000ADFF370002CEB30082CF5000F4FF36006E
:10B2B0001500370064004000204389000D0037006E
:10B2C000E4004000214389004143810078002000D0
:10B2D000E98F5000F6013C00018140008383220089
:10B2E00002814100630040000A0940008100E8003B
:10B2F000414389005BFE070044FE07006800200010
:10B30000E10F4000EA0132002043890082FF37004C
:10B3100000B62A00C8A402000000000040438100DB
:10B32000880020000000E000E10132000000E90098
:10B33000404389000000400081832200E100780042
:10B340002143890074FF37006400400020438900D6
:10B350003000370022C2B300824F500015003A007F
:10B360008100E8002143890009003700B1A681006F
:10B370000180A100B1A68900224389008CA30200AC
:10B3800000000000B0A681000080A000B0A68900E7
:10B3900022438100C0862200604079000201E8005B
:10B3A00021C2B300814F5000F0FF3A0022438900D0
:10B3B00018003700F2CBB30002414000F94F5100B2
:10B3C0000500360003C8B30083414000F2C5B30056
:10B3D00082CF51000A003E0022FE0700B1A6810084
:10B3E0000180A100B1A689000AA4020000000000AB
:10B3F000B0A681000080A000B0A68900050037003B
:10B40000B2C3B300824F500002003A008100E8004E
:10B410002143890021438100C086220060C078005A
:10B42000F2CDB300824F500003003E0032C8B3009B
:10B43000824F5000C7FF3A008100E900C086220019
:10B44000E0C07800B0C3B30080CF50009401320058
:10B45000B0A681000080A100B0A6890070B62A00C5
:10B46000AEA4020000000000B0A681000080A00091
:10B47000B0A689008A013700B1A681000180A10031
:10B48000B1A68900E400400021438900C286220061
:10B4900062C1780021C2B300814F51000E003A0012
:10B4A00065004000204389000300370021438900E4
:10B4B0008CA302000000000021438100C08622000E
:10B4C00060C078008100E80022C2B300824F5000C3
:10B4D000F6FF3A002143890020438100C186220003
:10B4E0006141780038002000C1C2B300814F510093
:10B4F00003003A000000E800204389000004EB004C
:10B5000020438100C1862200614578000A85FB0046
:10B510001A04B1008001EB00F2FF27006000B800C0
:10B5200026300200000000000A054500418022008C
:10B5300080307D00204381000000E8002043890026
:10B54000A4FD0700B0A681000080A000B0A689007D
:10B55000550137006400400031438100480020005D
:10B56000E38F500003003C008100E8003143890074
:10B570000004EB00C1862200614578000A85FB00CB
:10B580000A04B100324381006611B900E48422004C
:10B590000A3279000000E800204389006141780008
:10B5A000D1C3B300814F510008003A000000E80009
:10B5B00020438900ABFD07000A05E9000A054500A4
:10B5C0004180220080307D000100370038002000DB
:10B5D00020438100C1862200E14078000000E8009D
:10B5E00020438900B0C8B30080CF500006003A0065
:10B5F0003A4381009BFD07006655B9000185220092
:10B6000080307D0001003700380020002043810099
:10B61000C186220061417800F1CDB300814F510015
:10B6200005003600324381006611B900C184220052
:10B630008030790061003700380020005F0037005B
:10B64000E400400064C278000482FB000404B100FE
:10B650006500400032438100E18422005800200050
:10B660008001EB0011003700910F12000D003A002D
:10B670000403E9000603430047802200E7027B0041
:10B6800011049000888F520004003D00068343009F
:10B69000050BE80071B89700010037000201E900CE
:10B6A0000004EB008301E800E6804000828F510037
:10B6B000EDFF340020438900324389003F0037000A
:10B6C00064004000204389000004EB0050438100E7
:10B6D0000000E00015003A00030037008180FB0005
:10B6E000D10DB1000100400063014000C18622007D
:10B6F000E1417900E2C8B30082CF5100030032007B
:10B70000E14078000104E000F4FF3A00C186220025
:10B71000E1407800980020000104E00003003200BE
:10B7200064004000504389000004EB002B4381007B
:10B730005043810020438900CA8622006AC67D00EA
:10B740000C86FB001C04B100B4FD07000C0646008B
:10B750004180220080307E002043810050438900D8
:10B760008B05E8002B4389006A417800C1C2B30011
:10B77000814F510002003A000000E8005043890068
:10B7800050438100C1862200E141780002CEB3001F
:10B7900082CF510009003600630140006141790009
:10B7A000E1C8B300814F5100020032000000EB00FD
:10B7B00001003700640040005043890005FD070088
:10B7C000B9003700010545002A43890052FE3700C1
:10B7D00064004000204389000003200081A681000E
:10B7E0000088B900C2C62200620078008F003700CE
:10B7F00064004000204389000003200081A68100EE
:10B800000088B9000080E80086003700640040002E
:10B81000204389000003200081A681000088B90030
:10B82000640040007F00370064004000204389002E
:10B830000003200081A681000088B9006600400056
:10B840007800370064004000204389000003200096
:10B8500081A681000088B90068004000C1C62200AE
:10B8600061047800FFFC0700080001008C0037002D
:10B870006400400020438900FAFC07000000E0005B
:10B8800003003200C685020000000000840037007B
:10B89000F8850200000000008100370064004000CD
:10B8A00020438900EFFC07000000E00003003200A5
:10B8B000C922A900CB22A80079003700C922A9001B
:10B8C000CB22A900760037006400400020438900A5
:10B8D000E4FC0700414B2300114078000000A00069
:10B8E0000014A100804878006D003700640040001B
:10B8F00020438900DBFC0700E0A389000000E00092
:10B9000002003D000000EB00E0A3890000FA2000E7
:10B91000E1A38100808F500001003400E0A3890082
:10B92000F0A381000E00370064004000204389002E
:10B93000CCFC0700F0A38900E1A381000100E00036
:10B9400002003D008000EB00E1A3890001FA200025
:10B95000E2A38100810F510001003400E1A38900BE
:10B96000E10F500002003C0020002000F0A38900FD
:10B9700030062000F1A38100808F500001003400C8
:10B98000F0A389002280020000000000440037007C
:10B990006400400020438900B2FC070082A68100B9
:10B9A000010320000000E000030032000191B90013
:10B9B000F0004100020037000191B900F20041009F
:10B9C000C0C62200180037006400400020438900F0
:10B9D000A4FC0700E10F500009003200E20F500004
:10B9E0000C0032000000E0002D003A0000032000AF
:10B9F00081A681000088B9006E0040000900370070
:10BA00000003200081A681000088B9006C0040007E
:10BA1000040037000003200081A681000088B900DF
:10BA200076004000C1C622006100780000000100DD
:10BA30001B003700640040002043890089FC070098
:10BA40000000E00003003200E082A800E282A900CA
:10BA500013003700E282A900E082A900100037003D
:10BA600064004000204389007EFC0700F6BB020012
:10BA7000000000000A0037006400400020438900F5
:10BA800078FC07000103200082A681000191B90023
:10BA9000FC004100C2C62200E280780001000100E3
:10BAA0004CFC07009CFD37000800E0009AFD3200C6
:10BAB000B0A681000080A100B0A68900E10F54006B
:10BAC0001F00320061002000C037200044BD02008A
:10BAD00000000000080078000AA402000000000036
:10BAE000810020002038200044BD0200000000003A
:10BAF000090078000AA4020000000000B100200044
:10BB0000A038200044BD0200000000002043810056
:10BB10000AA402000000000070B62A00AEA40200D1
:10BB20000000000006003700180020000100370068
:10BB300038002000010545002A438900DCFF37005A
:10BB40004F0678004F05BE004F04BE0000000600FF
:10BB5000881F78000004780000C2B3008CA30200A4
:10BB60000000000008007800C8A4020000000000E7
:10BB700000C2B3008CA30200000000004F04780054
:10BB800000000600889FBE000000EB002500370083
:10BB90000804E00002003500084078001D0037006E
:10BBA00000CEB300804F54000F00360070B62A005C
:10BBB000AEA4020000000000204381008080E80065
:10BBC0000000E800694178004811DD0069C0780094
:10BBD0000080FB0000004100214389000AA402000C
:10BBE000000000000A00370000C2B3008CA302006E
:10BBF000000000000884FB000808B10008044400AD
:10BC00006040230060007C00C8A402000000000027
:10BC100000C2B3008CA3020000000000204381009A
:10BC20000000E80020438900C986220020438100EB
:10BC3000694478000804E000D5FF3A0070B62A0095
:10BC4000AEA4020000000000204381000000E900D3
:10BC50000AA40200000000007100200050392000FA
:10BC60008ABD0200000000004F04BE000000060074
:10BC7000139881000A0037001198810004202300E6
:10BC800064C27800844F510002003200139889008A
:10BC9000000005008100E800F10FB2001198890052
:10BCA000304178000204E000F3FF3A001000050084
:10BCB000889FBE00494023000004EB005900780033
:10BCC000EBFF07000000E0000300320000C8B300F3
:10BCD00000404400050037000804E800200220006E
:10BCE000800F5400F5FF3A000040EB004F04BE0007
:10BCF00000000600B0862200B1C622000068EB00FA
:10BD0000810F5000FDFF3A0011CEB300C086220023
:10BD1000014878000000E80000C8EB000000E800DF
:10BD200000C8EB0011CAB3000000E8000148780029
:10BD3000000006002400FA00889FBE008A1F7800D9
:10BD400013988100030078000498810009003700EF
:10BD500061417800F5C9B30085424100F9CF520036
:10BD600002003E000254A100827078000000E8004A
:10BD7000F00FB20001202300840F5000F4FF3A00BE
:10BD8000E1C0790000CDB30000C04000E94F500091
:10BD90008E003E005AFD2F000F054500E880570039
:10BDA0000A0078000068EB00810F5000FDFF3A00A8
:10BDB000902E020000000000C880DE00F1D79F0036
:10BDC00080DF9F0091FB0700E10F40001800320068
:10BDD000C2862200E24078008180FB0033F22F000F
:10BDE0008181410081004000E10DB100828040006E
:10BDF00003003700C2862200517178000000E8007D
:10BE00000240200003015100820F5000F9FF35006D
:10BE1000040037000041EB00C186220082707800E8
:10BE20000000E800F13F2000810F5000F9FF3400CE
:10BE300010300200000000008004EB0038002000F9
:10BE4000260037000900E0000D003A001030020023
:10BE50000000000096FF07008080FB000800320011
:10BE60008041780062FD2F000F01410003717C00CA
:10BE700070082000808F500011003A000F0037003A
:10BE80001098810001202300E140780022C2B30015
:10BE900082CF500001003A000900A2000141780061
:10BEA00064FD2F000F02420002727C000000E800D7
:10BEB000F00FB2001098890001003700190020002F
:10BEC0000804E80040022000800F540003003A00FC
:10BED00091002000C03920007200370000988100D6
:10BEE00011988100808F5000D6FF3A00E30F540074
:10BEF0006E003200E40F54006C003200C0CDB3007D
:10BF000000444400E8D79F007FD297004822DD001C
:10BF10000FD897000080FB00000242006000B800CC
:10BF20000F0037008381FB00030EB1008002E800A0
:10BF3000E2C27A00C82ADD000083E80062417B008B
:10BF40000281FB0002814200840F51000200310097
:10BF5000E300400083804000E38141000300400093
:10BF6000C2862200E241780005CEB30085CF5100A1
:10BF7000ECFF3E000000E000FEFF32000884FB0002
:10BF8000D80DB10080014400D28622008281410098
:10BF900002003700E26178000000E900C28622005A
:10BFA000810F5000FBFF3D008100E900810041004E
:10BFB0000000EB0002003700DA6878000000E800BB
:10BFC000880F5000FCFF35003800370080B62A008B
:10BFD00027FF07000000E000050032003CFC0700DE
:10BFE00070B62A00AEA40200000000002F00370047
:10BFF000C0B62A001EFF07000000E0000200320069
:10C00000E0FE07002900370010B72A0018FF0700DC
:10C010000000E00004003200B0A6810000A0A100F2
:10C02000B0A689002100370060B72A0010FF070082
:10C030000084EB000000E0000E003A001100370021
:10C040005A80FB00FAA502000000000000C2B30005
:10C050008CA30200000000008904E800F08F540067
:10C06000F7FF3A0070044400F03F2000800F5400B6
:10C070000E003200CA8622000A0544008004EB004C
:10C08000EFFF3700C0B72A00F9FE07000000E0000C
:10C090000200320017FF070004003700C100200033
:10C0A000503A20008ABD0200000000004F057800D1
:10C0B0004F04BE000080FA0000000600404B230041
:10C0C0001064A00000512300104078006840600018
:10C0D00005003200DA82A900F0C2B3008CA302008E
:10C0E0000000000001003700DA82A800A100200053
:10C0F00000BD20008ABD040000000000404B23006A
:10C100001064A100005123001040780068406000D6
:10C1100005003200DA82A900F0C2B3008CA302004D
:10C120000000000001003700DA82A800A100200012
:10C1300000BD20008ABD0400000000000051230063
:10C14000104078006840600005003200DA82A800E4
:10C15000F0C2B3008CA30200000000000100370011
:10C16000DA82A900B1002000A0BD20008ABD040031
:10C1700000000000881F780001022000C0DA2000C3
:10C1800044BD020000000000204A23001040E800E7
:10C190009AA302000000000000C2B3008CA30200BA
:10C1A00000000000085123009840780061C0600042
:10C1B0009AA302000000000000C2B3008CA302009A
:10C1C000000000001800D100614060009AA3020046
:10C1D0000000000000C2B3008CA3020000000000B9
:10C1E000180078004200DE00614060009AA302005F
:10C1F0000000000000C2B3008CA302000000000099
:10C20000180078004300DE00614060009AA302003D
:10C210000000000000C2B3008CA302000000000078
:10C22000404B23001080FB004400DE0061406000B2
:10C230009AA302000000000000C2B3008CA3020019
:10C24000000000003100200090BF200044BD02002B
:10C25000000000004F04780000000600889FBE0028
:10C260008A9FBE008C1F7800103002000000000082
:10C27000902E020000000000000478001030020040
:10C2800000000000902E0200000000000006780070
:10C290001030020000000000902E0200000000009C
:10C2A000800578001030020000000000902E02008F
:10C2B00000000000000578001030020000000000BF
:10C2C000902E020000000000800478001030020070
:10C2D00000000000902E0200000000008800E9002D
:10C2E000E38F500003003E00214A23008848E90004
:10C2F000010037000004EB008C00E900E18F5000E2
:10C3000007003E00015123000C46E900614666002B
:10C31000114178000204A1008C487100010037002F
:10C320000004EB008B00E900E18F500008003E00A4
:10C33000015123008B45E900E1C565008BC545002F
:10C34000114178000214A1008B48710001003700F0
:10C350000004EB008A00E900E18F500009003E0074
:10C36000015123000A45E9006145650022002000D3
:10C370000255DD00114178000224A1008A487100B5
:10C38000010037000004EB008900E900E18F500054
:10C3900009003E00015123008944E900E1C4640022
:10C3A00032002000824CDD00114178000234A100EF
:10C3B00089487100010037000004EB008000E900AB
:10C3C000E18F500009003E00414B230061406000B6
:10C3D000420020000200DD00114178000244A1006B
:10C3E000804871000800E00062003A0040302300FD
:10C3F0000048EB0071032000C0CC20008ABD020081
:10C40000000000008001EB0042002000110020002D
:10C41000100020002630020000000000214A230006
:10C420008048E9005103200030D020008ABD02007E
:10C43000000000008001EB0022002000110020001D
:10C4400010002000263002000000000008512300E8
:10C450000040E90061406000984078000104A100BC
:10C4600000CC70003104200080D320008ABD02007F
:10C47000000000008001EB002200200011002000DD
:10C480002000200026300200000000000040E900EB
:10C490006140600000404000984078000114A10015
:10C4A00000CC700011032000B0D720008ABD02002C
:10C4B000000000008001EB0022002000110020009D
:10C4C0001000200026300200000000000040E900BB
:10C4D00061406000290020000900DD0098407800DC
:10C4E0000124A10000CC7000D1012000B036210051
:10C4F0008ABD0200000000008001EB000901780005
:10C500001100200009007800263002000000000021
:10C510000040E90061406000310020000100DD00C2
:10C52000984078000134A10000CC7000F104200094
:10C5300050A520008ABD0200000000008001EB0031
:10C5400009017800110020001000200026300200B0
:10C5500000000000414B23006140600042002000C9
:10C560000200DD00114178000244A1008048710002
:10C5700001003700FFFE0700404B23001064A100BC
:10C580004F0678004F05BE004F04BE0000000600B5
:10C5900001012000104221008ABD040000000000BB
:10C5A00041E2A900414B230091407800F0C06000B7
:10C5B00004003200DE22A800DE42A800DE82A800CD
:10C5C00003003700DE22A900DE42A900DE82A900B6
:10C5D00001FC2F0043358000038160006201B3003D
:10C5E00042358800C2368000828060007100B3004E
:10C5F000C1368800F10F2C00B336800083806000C4
:10C6000001B0A000B1368800DA82A800D882A90063
:10C61000D842A900D862A800D822A9000080FB0057
:10C620001012880042A2A80080A881006101600069
:10C630004611DD00111280000160A100810071002F
:10C6400011128800C700DD000110B2001212800034
:10C650000280A10002817000121288004700DD00F4
:10C660000020B200111280000190A1008100700032
:10C67000111288004422EF004022EF0041E2A8009E
:10C6800000000600204A23001080FB0031E12A0050
:10C6900061407800C2FF070080A881000000D00040
:10C6A00070006000F1FE2F00D216800082806000D2
:10C6B00081007000D11688000000060041E2A90048
:10C6C00001FC2F004235800002806000F001B300C1
:10C6D00040358800806D200010886000F00F2C002D
:10C6E000D626B600DE22A900DE42A900DE82A9001D
:10C6F00000000600F1FF37000080FB0040128800B8
:10C700008540AB00FEFF3200401280008540A9004A
:10C7100000000600F8FF070080407800404B23002F
:10C7200003C4B30010C161000000EB00010032003F
:10C730000180FB000000060000C0EB00EEFF0700D8
:10C740000080FB0000000600D882A800D842A800A4
:10C75000D862A800D822A80000FC2F005235800023
:10C76000820060009101B30051358800743580006B
:10C77000840060009101B300713588004535800068
:10C78000850060008101B30041358800F20F2C0064
:10C7900046358000860161000170210083817000B0
:10C7A00043358800AC06B6006001B30060358800F0
:10C7B00060358000000161000281700062358800F0
:10C7C000204A23001080FB0031E12A0061427800FA
:10C7D0000482FB001412880080A8810061016000BF
:10C7E0004611DD00F3FB2F001512800085806100EB
:10C7F00081007100111288004700DD000010B200B6
:10C80000F1EF2F0016128000868260008502700012
:10C81000151288004422EF004022EF001413880014
:10C820001413800084816100830171001313880058
:10C83000151380008580600081007000111388004E
:10C840006422EF006022EF004822EF006822EF0030
:10C850004322A9006322A9004362A80042A2A900C2
:10C860006362A80062A2A90040C2A90060C2A90038
:10C870004402A8006402A8000000060041E2A900EA
:10C880004362A90061E2A9006362A90000FC2F00D5
:10C890005235800082006000F101B30051358800FC
:10C8A0007235800082006000F101B30071358800AC
:10C8B0004235800082006000F101B30041358800FC
:10C8C000F20F2C00413580008101610001F0210050
:10C8D0008381700043358800AC06B600F001B300D8
:10C8E00060358800603580000001610002817000C1
:10C8F0006235880000000600889FBE008A9FBE0047
:10C9000000447800014578006AA60200000000009B
:10C910006AFF07008CFF07000804E00003003A00EC
:10C9200042E2A80062E2A80002003700E14F540092
:10C930000A003E0041E2A80061E2A80007003700BB
:10C940000904E00005003A00DA82AB00040032007E
:10C95000D0C5B30024A602000000000019C0B30037
:10C9600040A2AB0022003A0060A2AB0020003A00D7
:10C970004B128000E1CF540003003A00B0C5B30071
:10C9800024A60200000000000A04E00004003200B7
:10C990000B80FB0026A60200000000000600370006
:10C9A000C0C5B30024A60200000000000B407800C0
:10C9B00024A602000000000040138000804478009C
:10C9C0000A04E0000700320080C2B30024A602007F
:10C9D000000000000980FB0026A602000000000005
:10C9E00090C2B30024A60200000000008044EB00C7
:10C9F00040C2AB0006003A0060C2AB0004003A003F
:10CA000000202000614D2300110060001000320062
:10CA100000202000614D23001100600002003A0058
:10CA200064A60200000000004022EF006022EF0038
:10CA30000A04E0000400320040DF2A00AEA4020035
:10CA400000000000B0FF3700CB02A9000D00370046
:10CA50006CA60200000000004CA6020000000000CE
:10CA6000E14F5000B6FF3A0060A60200000000004F
:10CA70000A04E0000300320050E02A00AEA40200E5
:10CA8000000000007DFF0700204A23001080FB000B
:10CA900031E12A0061407800C1FE07004F05BE0069
:10CAA0004F04BE00000006008000EB00EF0F5000B6
:10CAB000E08F580050003E00006001000F0037007A
:10CAC000120037001C0037004F0037004A003700C3
:10CAD000490037004800370047003700460037005C
:10CAE000450037001F0037002100370023003700C2
:10CAF00025003700270037002900370041032000B8
:10CB0000C0DC20008ABD040000000000710020008D
:10CB1000D05A20008ABD020000000000F100200071
:10CB2000003321008ABD02000000000011C0B300E4
:10CB30000040EB000A00370071002000D05A2000AE
:10CB40008ABD020000000000F10020000033210037
:10CB50008ABD02000000000011C0B300014078004F
:10CB600065FF3700005123001004A1000E003700BC
:10CB7000005123001004A0000B00370000512300D7
:10CB80001014A10008003700005123001014A00069
:10CB900005003700005123001024A10002003700D7
:10CBA000005123001024A00080A8810061016000D2
:10CBB0004611DD00111280000160A10081007100AA
:10CBC00011128800C700DD000110B20012128000AF
:10CBD0000280A10002817000121288004700DD006F
:10CBE0000020B200111280000190A10081007000AD
:10CBF000111288005FFD370041022000E01D200077
:10CC00008ABD0200000000000000060060E02A006B
:10CC1000C8A4040000000000889FBE008A9FBE00D8
:10CC20008C1F780011C0B300204A2300014878000F
:10CC300001512300114078000000A1000010A00065
:10CC40000020A10080487800404B23001044A00041
:10CC500080C1B30052FE0700ECFF070060A602008F
:10CC60000000000031512300804878000081FB0063
:10CC70004411DE0023512300824978000281FB0029
:10CC80008001EB00E80F5100E08F590024013E00C5
:10CC90000260010008003700E10037002001370082
:10CCA0001F013700F2003700F4003700F6003700AC
:10CCB0001B013700FA0037000080FB008000EB000A
:10CCC000EE0F5000E08F580015013E00006001009B
:10CCD0000E003700E0FF3700110037001200370068
:10CCE000200037001F003700680037000C013700B4
:10CCF0000B0137000A01370009013700080137002E
:10CD0000070137000A0037000F0037006BFE0700ED
:10CD10004F0678004F05BE004F04BE00000006001D
:10CD2000DC82A900FC003700DC82A800FA00370092
:10CD300010C0B3008CA30200000000008040EB0094
:10CD400010C0B3000500370010C0B3008CA3020070
:10CD5000000000008040EB0001407800E6FE070084
:10CD6000BEFF370060A60200000000004804DD009E
:10CD700060A60200000000000086FB0008067600A6
:10CD800060A60200000000000044780060A60200D7
:10CD90000000000001002100810F5600E0003E006D
:10CDA0004845DD000080FB000A0570000004EB0030
:10CDB000810F550007003600D9003700A04C230032
:10CDC0009004440060A6020000000000804C78003F
:10CDD0000804E8008C0F5400F8FF3900305123009C
:10CDE00041C0B30090CF100001003A00DA82A900E0
:10CDF0000004EB000400370050A6810060407C0076
:10CE00003DFE07000804E8008C0F5400FAFF3900CB
:10CE100010002000CABB0200000000000004EB006C
:10CE200006003700A04C23001006440000C0EB00B1
:10CE300031FE0700004E78000804E8008A0F540015
:10CE4000F8FF39003051230041C0B30090CF1000EB
:10CE500001003A00DA82A80010C0B3008CA30200DF
:10CE6000000000000004EB000500370050A6810020
:10CE700060407C008CA30200000000000804E80071
:10CE80008A0F5400F9FF390074FF370010C0B30057
:10CE90008CA302000000000060A602000000000059
:10CEA000004478003051230008487800E14F5400D6
:10CEB0000400320098003900E24F540098003A0014
:10CEC00008003700084078008CA302000000000032
:10CED0000040EB008CA30200000000000840780036
:10CEE00090003700480020006055B80060A602009E
:10CEF0000000000031512300804878004859DD00CF
:10CF0000C851DE00830171004851DD000085FB003F
:10CF10008005EB0002057500838575000804E900B3
:10CF2000F2FF3A006044B8000006EB0060A6020081
:10CF30000000000031512300804878004849DD009E
:10CF4000C841DE00830171004841DD000084FB0020
:10CF50008004EB0002047400838474000C06E80073
:10CF6000E40F5600F1FF3A00E10F4500E08F5D004D
:10CF70006B003E00E10F4400E08F5C0068003E0063
:10CF80000800450089804D00E10F4000E08F580007
:10CF900063003E0010C0B3008CA30200000000003C
:10CFA0001B00370000C2B300D3FD07004856DE0067
:10CFB0000C407800D0FD07000A407800CEFD070045
:10CFC0000040EB00CCFD07008CA302000000000035
:10CFD000E10F5400E08F5C0020FF320080C2B300FC
:10CFE000C5FD07000C407800C3FD07000A4078002B
:10CFF000C1FD07000040EB00BFFD07008CA302004D
:10D000000000000062045400E0845C000A05E800AF
:10D01000E00F5400E08F5C00E2FF3A000FFF3700A2
:10D020006F4060008048E80010C0B3008CA302008D
:10D0300000000000105123000048EB0006003700FC
:10D0400060A6020000000000ABFD07008CA30200F8
:10D0500000000000184CE800185123003051230054
:10D060009840780090CF5000F5FF3900FBFE370064
:10D0700072C102000000000027003700B8C10200A2
:10D0800000000000270037006740600080487800FB
:10D09000214A2300804878000080FB001B003700F5
:10D0A00001512300114178000200A1000210A100EB
:10D0B0000220A10082487800434B23001344A100C2
:10D0C0000080FB000028A300020032000204A00040
:10D0D000824878000018A3000200320001512300AA
:10D0E0001114A0000008A300020032000151230027
:10D0F0001124A0000038A30002003A00404B230096
:10D100001044A000204A23001080FB00B1E02A0058
:10D110006140780022FD070010C0B3000100370015
:10D120000040EB008CA3020000000000CBFE3700A3
:10D13000881F78002CC30200000000000004E000FB
:10D14000170032003262AB000400320031002000D0
:10D1500000E0200044BD0200000000003242AB00AD
:10D16000040032003100200030E0200044BD020005
:10D170000000000024C3020000000000000478004A
:10D180003222AB000B003200F100200060E02000F2
:10D1900044BD0200000000003222A9000500370053
:10D1A000F100200050E1200044BD0200000000001A
:10D1B0000004EB00080078004F047800000006002F
:10D1C0001CC302000000000000000500881F78005A
:10D1D00001022000B0EC200044BD0200000000006D
:10D1E000284A2300184078009AA30200000000009B
:10D1F00000C2B3008CA302000000000018407800B9
:10D20000E94F500002003A00C011800004003700CE
:10D210000080FB000000400061D52A00610078001A
:10D220000AA402000000000000C2B3008CA30200A8
:10D230000000000060A78100634060009AA3020024
:10D240000000000000C2B3008CA302000000000038
:10D2500060A781004200DE00614060009AA30200E6
:10D260000000000000C2B3008CA302000000000018
:10D2700060A781004300DE00614060009AA30200C5
:10D280000000000000C2B3008CA3020000000000F8
:10D29000404B23001080FB004400DE006140600032
:10D2A0009AA302000000000000C2B3008CA3020099
:10D2B000000000003100200090BF200044BD0200AB
:10D2C000000000004F047800000006000200FA0091
:10D2D000889FBE008A9FBE00C04E23001054A1004C
:10D2E0001030020000000000902E0200000000003C
:10D2F000000178000004EB00EA0F510007003A003B
:10D30000B2BF9F001030020000000000902E02000B
:10D3100000000000000478003FB99700B2BF9F00F2
:10D320001030020000000000902E020000000000FB
:10D33000800578001030020000000000902E0200EE
:10D34000000000000005780010300200000000001E
:10D35000902E0200000000008004780010300200CF
:10D3600000000000902E0200000000003FB997006E
:10D370008200E900E98F500003003E00214A2300AB
:10D380008248E900010037000001EB008B00E90052
:10D39000E38F500007003E00C14E23008B45E9009B
:10D3A000E3C56500C3CFB30091C161008BC87100B4
:10D3B000010037000001EB008A00E900E18F500016
:10D3C00009003E00C14E23000A45E90061456500A1
:10D3D000230020000355DD00914178000324A100C3
:10D3E0008AC87100010037000001EB008900E900E4
:10D3F000E18F500009003E00C14E23008944E9003E
:10D40000E1C4640033002000834CDD0091417800CA
:10D410000334A10089C87100010037000001EB004E
:10D420008000E900E18F500009003E00414B2300DD
:10D4300061406000430020000300DD00914178005E
:10D440000344A10080C871000200E00074003A00AB
:10D45000403023000048EB00E10B2000C095200085
:10D460008ABD0200000000008001EB00B200200035
:10D4700011002000100020002630020000000000F3
:10D480000040E900214A230080487800EA4F50001C
:10D4900007003A0080C0B30080487800C04E2300E7
:10D4A0001054A00000CE2A00AEA40200000000002C
:10D4B000204A230091C0B30090CF100014003A001E
:10D4C00091012000702F21008ABD020000000000A1
:10D4D0008001EB00F4232400F5002000120020005E
:10D4E00000202C0011002000B832020000000000D3
:10D4F0000001BE0000902000D10320001826020089
:10D500000000000061015000E0815800C211880055
:10D510004105200040E2200044BD02000000000060
:10D520008001EB00420020001100200010002000CC
:10D530002630020000000000C84E23000040E90031
:10D5400063406000C1CFB30098C0600000CC7000A1
:10D550001102200080E7200044BD0200000000000E
:10D560008001EB00220020001100200010002000AC
:10D5700026300200000000000040E9006140600029
:10D58000290020000900DD00984078000124A10056
:10D5900000CC70002103200090E9200044BD02006F
:10D5A000000000008001EB0009017800110020005C
:10D5B0001000200026300200000000000040E900BA
:10D5C00061406000310020000100DD0098407800DB
:10D5D0000134A10000CC7000F104200050A520000F
:10D5E0008ABD0200000000008001EB000901780004
:10D5F0001100200010002000263002000000000072
:10D60000414B230061406000420020000200DD0029
:10D61000114178000244A100804871000D003700DC
:10D62000204A230091C0B30090CF100008003A00B8
:10D630006141B90000902000D103200018260200AB
:10D640000000000061015000E0815800C211880014
:10D65000DEFE07004F05BE004F04BE000080FA004A
:10D660000000060004C30400000000003222A900EC
:10D67000C04E23001044A000404B23001024A00003
:10D68000C1012000D0F820008ABD04000000000085
:10D69000C04E23001044A100404B23001024A100E1
:10D6A0004101200090FA20008ABD04000000000023
:10D6B000881F78000004EB0029003700C04E2300CB
:10D6C000104078007040600022003200A0CF2A0095
:10D6D000AEA402000000000061002000E074200001
:10D6E00044BD0200000000003262AB0004003200C2
:10D6F0003100200000E0200044BD020000000000D6
:10D700003242AB00040032003100200030E0200043
:10D7100044BD02000000000024C30200000000001D
:10D720003EBB0200000000003222AB0005003200C8
:10D73000F100200060E0200044BD02000000000075
:10D740003222A900A0CF2A00AEA4020000000000EF
:10D750000200370024C3020000000000180020006F
:10D760002CC30200000000000004E000D3FF3A00D8
:10D77000080078004F04780000000600B100200087
:10D78000A04321008ABD0400000000001E21EF001C
:10D790001021EF0080002000800888000821EF00A1
:10D7A0000621EF001621EF001421EF00F008880099
:10D7B0000000060011E1A9001FE1A90000FC2F00F4
:10D7C0008606B600F001B300303488001E21EF0059
:10D7D0001021EF000621EF000821EF0000000600F5
:10D7E0000003BE0060D12A00110020005002BE00DC
:10D7F000840F5300858F5B00100031008100E90029
:10D80000C208DD0060D12A00810040001101BE0085
:10D810000200520083805A008100D1000080D300B2
:10D820000000410081804900800F5300818F5B0020
:10D83000070036000400BE00000006008100E8007A
:10D84000EF8F5000E9FF3A000100200000000500C2
:10D850000200BE00000006000400FA00881F7800E5
:10D860008A9FBE0000047800DA62A900D862A8008E
:10D870000800E00006003A0031012000205321009A
:10D880008ABD020000000000010037000000000017
:10D89000DA62AB00020032002202AB00FBFF320072
:10D8A0006011B8000005EB002202AB000800320056
:10D8B00030118000BFFF0700E1002000505421001C
:10D8C0008ABD0200000000006055B800510037001A
:10D8D000B2BF9F00C3BF9F00ACFF0700CFB9970046
:10D8E0003FB99700DA62AB00FEFF32001FE1A800EB
:10D8F00011E1A800DA62AB00FEFF3A0011E1A900D5
:10D900001FE1A90000FC2F008606B600F001B3005D
:10D91000303488001E21EF001021EF004008800005
:10D92000340880000A00E0000C0032008000EB00A8
:10D93000C000DD000000200000004200E080480040
:10D94000E00F5100E08F590003003200800F5100BA
:10D95000818F5900010036000001BE000A05E80071
:10D96000F90F5500DAFF3A00B2BF9F00C3BF9F0016
:10D9700090FF07003FB99700CFB997000040220001
:10D98000410F200018260200000000000005BE0024
:10D990000800E0001F003A00009F24002100200042
:10D9A000800F5500818F5D00030036008103200049
:10D9B0003055210015003700F1002000B05821003B
:10D9C00044BD0200000000000A00BE004AA402009C
:10D9D0000000000041002000905A21008ABD020092
:10D9E00000000000F1002000A059210044BD020009
:10D9F000000000000A00BE0079FF07004AA40200F0
:10DA00000000000041002000905A21008ABD020061
:10DA1000000000000A00BE004F05BE004F04780061
:10DA20000080FA00000006008000EB00E40F5000C8
:10DA3000E08F58004C003E000060010004003700F9
:10DA40000700370029003700050037004000370085
:10DA5000C1072000B0EE200044BD0400000000001B
:10DA6000B100200070F620008ABD02000000000016
:10DA7000E1002000405221008ABD020000000000A9
:10DA80001CBE0200000000000004E0003A0032006A
:10DA90003222A900D3C2AB00370032003202AB0001
:10DAA00003003200B01180008CA3020000000000CF
:10DAB0004CA6020000000000E14F500006003A00B2
:10DAC0003322AB0004003A0060A602000000000010
:10DAD0000080FB00A01188003222AB00EDFF320075
:10DAE0003222A900CB02A900EAFF3700E1002000A2
:10DAF000F0F720008ABD020000000000F1002000C5
:10DB0000003321008ABD0200000000003222A9007B
:10DB1000D3C2AB00180032002CC30200000000008A
:10DB20000004E0000400320024C3020000000000F2
:10DB30008CA30200000000004CA6020000000000C0
:10DB4000E14F5000F2FF3A0060A604000000000020
:10DB500004C30200000000000000EB003EFF0700CD
:10DB6000FAC204000000000041022000E01D200075
:10DB70008ABD020000000000000006000400FA0058
:10DB8000204A23001040780063A78100E94F50002D
:10DB90000B003A00C0118000421ADE004319DE007B
:10DBA00061416100414B23009180FB00C408DE000D
:10DBB000E1C0600061426200E3C161000D00370016
:10DBC000421ADE004319DE0061416100414B23002F
:10DBD0009180FB00C408DE00E1C060000080FB0013
:10DBE0000000400061426200E3C1610065D52A0087
:10DBF00065007800A2C2020000000000C04E2300B1
:10DC00001040780063406000E34F500003003A008A
:10DC100091C0B300304A230001487800FAC20200E4
:10DC200000000000C04E230001C2B30010C060001D
:10DC30003800320004C3020000000000B0CF2A0008
:10DC4000AEA40200000000000000EB0002FF07008D
:10DC5000E3FE07000001BE00B0CF2A00E2BF9F0034
:10DC6000F3BF9F00AEA40200000000006FB9970050
:10DC7000FFB99700E00F5100E08F59000C003A0007
:10DC800063A78100421ADE004319DE006141610092
:10DC9000404B23009080FB00C408DE00E1C0600020
:10DCA00061426200E3C161002002200015003700DC
:10DCB00091C0B300204A2300014878000090200062
:10DCC000D103200018260200000000000003BE005F
:10DCD00063A78100421ADE004319DE006141610042
:10DCE000404B23009080FB00C408DE00E1C06000D0
:10DCF00061035300E0835B0061426200E3C16100A5
:10DD000006007800A2C2020000000000FAC2020071
:10DD1000000000000080FA0000000600D0CF2A00BA
:10DD2000C8A4040000000000881F7800C24E230031
:10DD3000924078000100A100404B23001044A00055
:10DD40004041230070A7890003CEB30003C96000DF
:10DD50000042EB00844178000441780011C0B30018
:10DD6000A2C2020000000000FAC20200000000008F
:10DD7000EAFF07002CC30200000000000004E000DE
:10DD80000B003200C04E230010407800704060004D
:10DD90000500320024C30200000000008CA3020032
:10DDA000000000000200370024C302000000000051
:10DDB0003222AB00010032003222A9004CA6020040
:10DDC00000000000E14F5000EAFF3A0060A60200A8
:10DDD00000000000214F2300804878000081FB00F4
:10DDE0004411DE00134F2300824978000281FB00BA
:10DDF0008001EB00E90F5100E08F5900C3003E00A5
:10DE000002600100090037005F003700BF003700E3
:10DE1000BE00370073003700750037007700370009
:10DE2000BA00370083003700820037000080FB0013
:10DE30008000EB00EF0F5000E08F5800B3003E0071
:10DE4000006001000F003700C9FF370011003700E4
:10DE500019003700AD003700AC003700AB003700C9
:10DE600018003700A9003700A8003700A7003700C6
:10DE7000A6003700A5003700A4003700A300370034
:10DE80002D00370004C30200000000004F0478009A
:10DE90000000060010C0B3008CA3020000000000C8
:10DEA0003222AB00010032003222A900C04E230012
:10DEB0001044A000AFFF3700C04E23001044A10063
:10DEC0009000370010C0B3008CA3020000000000D7
:10DED00004C302000000000060A602000000000071
:10DEE0004800DD0070A7890010C0B3008CA30200B9
:10DEF0000000000078A7810060A60200000000007A
:10DF00000080FB000000740070A7890063A78100F7
:10DF1000421ADE004319DE0061416100414B2300DB
:10DF20009180FB00C408DE00E1C060006142620035
:10DF3000E3C161006F00370010C0B3008CA3020082
:10DF4000000000003222A9003202AB0003003200C0
:10DF5000B01180008CA30200000000004CA602005B
:10DF600000000000E14F5000F7FF3A003322AB0001
:10DF7000F5FF3A0060A60200000000000080FB00F0
:10DF8000A0118800F0FF37006F4060008048E80073
:10DF900010C0B3008CA3020000000000004F23005B
:10DFA0000048EB000900370060A6020000000000F6
:10DFB0000080FB001CC302000000000010C0B30082
:10DFC0008CA3020000000000184CE800084F23005A
:10DFD000204F23009840780090CF5000F2FF390086
:10DFE00064FF370072C102000000000045003700E6
:10DFF000B8C1020000000000450037006F4060001B
:10E0000080487800EA4F500003003600A1C0B300FA
:10E01000204F230001487800204F23001080FB0090
:10E020000000400021D02A00E100780071A789009B
:10E0300023003700C24E2300924078000100A10067
:10E040000110A1000120A1000130A10001497800C8
:10E05000434B23001344A1000080FB000038A300C1
:10E06000020032000114A000014978000028A3003A
:10E0700007003200C24E230061A78100E3C06000A8
:10E080000104A000C3CFB30092C1610001C97100B7
:10E090000018A30002003200C14E23001124A0008A
:10E0A0000008A30002003200C14E23001134A0007A
:10E0B0000048A30002003A00404B23001044A00097
:10E0C00004C302000000000063A78100421ADE00C2
:10E0D0004319DE0061416100404B23009080FB004A
:10E0E000C408DE00E1C0600061426200E3C161007B
:10E0F00070A78100A2C2020000000000FAC2020064
:10E100000000000010C0B300010037000040EB0029
:10E110008CA302000000000016FF3700800078008A
:10E1200040002000B00098000000060011C0B300BD
:10E1300001487800000005000200FA00881F7800FE
:10E140000004780064805700ECC00200000000006A
:10E150004FF897000004E000FAFF3A000000EB00DF
:10E16000300498004F0478000080FA000000060098
:10E170000200FA00881F78000004780064805700CD
:10E18000ECC00200000000004FF89700E14F500083
:10E1900012003E0098409000F3CF500007003A0074
:10E1A0000004E00002003A0010C0B3000100370094
:10E1B000D0C0B300104C9800060037000004E00007
:10E1C00002003A0010C0B3000100370060C0B30085
:10E1D000204C98000000EB000200370050002000A7
:10E1E000300498004F0478000080FA000000060018
:10E1F0006B004000ECC002000000000000000500C1
:10E20000881F780000047800E00E2000080040001D
:10E21000A808900092C002000000000040122000F8
:10E2200008004000A808900092C002000000000012
:10E230000000EB004F04780000000600800078002A
:10E24000800B200001004000A108900092C0020055
:10E250000000000000000500889FBE000004780058
:10E26000F6044400410020000900780092C002003A
:10E270000000000009007800E6BF02000000000076
:10E2800060049800710498000000EB004F04BE0089
:10E29000000006000042EB0004487800144098009B
:10E2A0006011B80012009800230098008000EB0075
:10E2B00031009800314898000448980014C0B30019
:10E2C0001448980024489800020898001308980001
:10E2D00021089800620098007300980001007800FF
:10E2E000000006000000060067014000E0814800D1
:10E2F00002003B006E014000E08148004D1ADD0045
:10E300004310DE0000007200C398DE00000006002B
:10E31000889FBE0000047800F604440041002000FD
:10E320000900780092C00200000000000900780097
:10E33000E6BF020000000000000C9800110C9800DD
:10E34000E9FF070080007800210C98000000EB0036
:10E3500022032000828F5000020034006000200061
:10E36000300498004F04BE000000060080007800D2
:10E3700010002000BAC00200000000006000B800D9
:10E38000BAC0020000000000110020000000EB00F5
:10E39000BAC0040000000000889FBE008A1F7800F9
:10E3A00000047800814478000904E00010003A007D
:10E3B00010002000EDFF07008004EB006000B800B3
:10E3C000BAC0020000000000110020000000EB00B5
:10E3D000BAC00200000000008904E800E58F540084
:10E3E000F6FF3A00004CEB000005EB007B00370025
:10E3F0001840780080CF54000C003200E7CF540062
:10E4000004003A005A002000E64F500073003A0022
:10E4100012003700EECF540010003A005A002000DE
:10E42000ED4F50006D003A000C003700E6CF54006D
:10E4300004003A0010002000CCFF070070C0B300B9
:10E4400005003700EDCF540004003A001000200012
:10E45000C6FF0700E0C0B300004C78000005EB00E9
:10E460005B0037000080FB008000EB00EF0F5000E6
:10E47000E08F580054003E00006001000F0037009C
:10E4800012003700160037001F0037002000370049
:10E4900023003700250037002800370044003700EC
:10E4A0002C0037002F0037003000370033003700D2
:10E4B00035003700380037003D0037000000EB0022
:10E4C000AAFF070010C0B3000300370010002000AF
:10E4D000A6FF070020C0B300004C78003C003700C6
:10E4E000E8CF540004003600100020009FFF070012
:10E4F00090C0B300F8FF37000000EB009BFF07005F
:10E5000030C0B300F4FF3700E4CF54002A003200DB
:10E510001000200095FF070050C0B300EEFF370049
:10E52000E6CF540007003A00230037001000200017
:10E530008EFF070070C0B300E7FF3700E4CF540040
:10E540001D0032001000200088FF070080C0B300CB
:10E55000E1FF37000000EB0084FF0700A0C0B3001C
:10E56000DDFF3700EBCF5400130032001000200015
:10E570007EFF0700C0C0B300D7FF3700EDCF5400C7
:10E5800007003A000C0037001000200077FF07005A
:10E59000E0C0B300D0FF3700EBCF540006003200DC
:10E5A0001000200071FF0700F0C0B300CAFF370061
:10E5B000E1CF5400C5FF3A000000EB006BFF0700FD
:10E5C000094C780002003700094C78005A002000FE
:10E5D0001840780080CF5400A2FF3A000A0078006B
:10E5E0004F0578004F04BE0000000600889FBE0063
:10E5F0008A9FBE008C9FBE0000047800F604440091
:10E60000110020000900780092C002000000000004
:10E61000885D9000110020000900780092C002007F
:10E6200000000000085D9000410020000900780013
:10E6300092C002000000000009007800E6BF02005E
:10E64000000000000006BE00084890008B4F5000FC
:10E6500003003200680044008B4078004EFF070042
:10E660000C00BE0046C102000000000008489000F7
:10E670008A4F500003003200680044008A4078004E
:10E6800045FF07000000EB004F06BE004F05BE002F
:10E690004F04BE00000006000200FA00881F780048
:10E6A0000004780064805700ECC002000000000005
:10E6B00068004400CFF8970037FF07000000E00033
:10E6C00001003200300498004F0478000080FA0006
:10E6D00000000600E4874700889FBE008A9FBE00B6
:10E6E0008C9FBE008E1F78000004BE0084BF9F0078
:10E6F0000005EB000300E0000300320092097800FF
:10E700001285E8000A8541001287E8000E074100E3
:10E710002D003700CE4678008005EB000046EB0068
:10E7200061045400E0845C000FB897000000E00032
:10E7300007003200E00F5400E08F5C0004003A0054
:10E740001100200010002000BAC0020000000000EC
:10E75000E180660020002000BAC002000000000036
:10E760006000B800BAC00200000000000A00E0002B
:10E77000050032003EC10200000000000080FB00E6
:10E780000B00DD0000467600110020000000EB00C9
:10E79000BAC0020000000000E00F5400E08F5C00EF
:10E7A000060032008B05E800E88F550003003200B8
:10E7B0008D86FB008D06D100D9FF37000A00E000EE
:10E7C000010032000C657800E00F5400E08F5C001F
:10E7D000D0FF3A004F0778004F06BE004F05BE003D
:10E7E0004F04BE004F00B10000000600EE87470056
:10E7F000889FBE008A9FBE008C9FBE008E1F78003F
:10E8000000057800E1EF9F000204BE00C4B79F003E
:10E81000E5B79F00D6B79F00B7B79F005FAE9700E0
:10E82000EFAE97006FD9970002C068000080FB0030
:10E830000000EA004F00DE0080BF9F008045EB0033
:10E840000007EB00E00F5400E08F5C000C003A0082
:10E850000000EB00E00F5600E08F5E004E0032003B
:10E8600011C0B3000A007800CBFE07000C00BE0008
:10E8700046C1020000000000460037001E002000D4
:10E88000EFE897000A007800C3FE07000FBA970070
:10E89000EFB197004FB197000800BE008DFF070051
:10E8A0005FB097000000E000080032003FB1970021
:10E8B000EFB0970014C002000000000000F0A700B5
:10E8C0000000EA000007E9004F77DE008FB89700EC
:10E8D0000100E000220032001A4DE8000E00E000C6
:10E8E00013003200E00F5600E08F5E00100032008F
:10E8F0000FD9970082CF55000D00310061C0B300E1
:10E900000A007800A4FE070041C0B3000A007800A6
:10E91000A1FE07004E69DD004260DE0000007100CC
:10E92000C2E8DE000C0640008D8648000300370078
:10E93000EFD897000A00780097FE0700E00F560016
:10E94000E08F5E000600320011C0B3000A007800BC
:10E9500091FE07000C00BE0046C10200000000004E
:10E960000E00E0000B0032008B45E8000B40E90090
:10E970008FD89700814F5000C0FF39000C0037003E
:10E98000300020000FD9970082CF55000B003600D1
:10E99000010037000000EB004F0778004F06BE0073
:10E9A0004F05BE004F04BE00EF00B100000006009E
:10E9B0000FD897000004E000F1FF3A00200020008B
:10E9C000F5FF3700889FBE0000047800F60444007D
:10E9D000A80890000900780092C002000000000022
:10E9E000870B20008883430068004400B8489000EB
:10E9F000811F780068019000F8019000829FBE009E
:10EA0000A8499000831F7800C60420000803430033
:10EA10002508200088824200090278000809900039
:10EA20009809900041C0B30070FF0700E8875700C5
:10EA30000000E00001003200300498004F04BE00E6
:10EA4000000006000400FA00889FBE008A1F7800BC
:10EA50008004780076854400210020000A007800B8
:10EA600092C00200000000000A007800E6BF020029
:10EA7000000000000001BE00B2BF9F00C3BF9F00A6
:10EA800019FE0700800078006000200024032000A9
:10EA9000848F500015003C000A00780092C00200EC
:10EAA0000000000068844400801FEB0069009000B3
:10EAB000F9009000809FBE0099489000811F780067
:10EAC0006033B8008002EB000A0278007FB1970043
:10EAD0008FB99700B1C0B3000800780043FF07006A
:10EAE000E88757000000E00001003200B004980001
:10EAF0004F0578004F04BE000080FA0000000600B9
:10EB00000200FA00889FBE0000047800668057006B
:10EB1000ECC00200000000002FF997000280FB000B
:10EB20008000EB00F0FD070080007800600020000E
:10EB300022032000828F500016003C00F60444009F
:10EB40000900780092C00200000000002FFA970030
:10EB50000481FB008001EB0068004400801FEB0093
:10EB600068029000F8029000849FBE00984A9000CE
:10EB7000851F78006033B8008002EB00090278003E
:10EB8000B1C0B30019FF0700E88757000000E0009C
:10EB900001003200300498004F04BE000080FA00EB
:10EBA000000006000400FA00889FBE008A9FBE0095
:10EBB0008C9FBE0080047800010478000405BE002C
:10EBC0000606BE00880078000A00780082BF9F0019
:10EBD00093BF9F0092C00200000000000FB9970091
:10EBE0009FB997000C00E000060032008800780012
:10EBF0000C00780092C00200000000009FB997004E
:10EC00000FB997002FE09700801F78001FB0970082
:10EC1000AFB09700809FBE00AFE09700811F7800E3
:10EC20000C03BE000A02BE0041C0B3000900780018
:10EC3000EEFE0700E88757004F06BE004F05BE00F6
:10EC40004F04BE000080FA0000000600881F780014
:10EC5000000478001840900041C0B300F14F50000C
:10EC600001003A00A848900068004400801FEB00B3
:10EC7000801FEB00801FEB00811F78008003EB00FA
:10EC8000C6042000080343002508200088824200B3
:10EC900076024400A80890000809900098099000A6
:10ECA000C0FF0700E88757000000E00001003200C5
:10ECB000300498004F04780000000600881F780098
:10ECC000000478001840900041C0B300EE4F50009F
:10ECD00001003A00A848900068004400801FEB0043
:10ECE000801FEB00801FEB00811F78006033B800AD
:10ECF0008002EB0076024400A8089000080990000A
:10ED000098099000A7FF0700E88757000000E0007F
:10ED100001003200300498004F0478000000060023
:10ED2000881F780000047800870B20008883430048
:10ED300068004400B8489000811F78006801900086
:10ED4000F8019000829FBE00A8499000831F7800C0
:10ED5000C6042000080343002508200088824200E2
:10ED600076024400A80890000809900098099000D5
:10ED70008CFF0700E88757000000E0000100320028
:10ED8000300498004F04780000000600889FBE0001
:10ED90008A9FBE000004BE0003057800880078004A
:10EDA0000800780062C002000000000099027800AC
:10EDB0009A00E9000040EB00004378001E00370095
:10EDC00001014500224290000404E00019003200D5
:10EDD000810344002741900013C0B3000408A3003E
:10EDE0000D0032000004E00004003A008502E90052
:10EDF0000580E8006943780010C0B30086456000D4
:10EE000002003200034171000200370083C5EA00AE
:10EE100002C16500004040000482FB000402D100F2
:10EE20000404E0000200320083C14100EBFF370020
:10EE3000A24398008100E9000100E000E0FF3D00EE
:10EE40004F05BE004F04BE0000000600EA874700E1
:10EE5000889FBE008A9FBE008C9FBE008E1F7800D8
:10EE600000047800F6044400A80890000900780027
:10EE700092C0020000000000800B2000000044004F
:10EE800080BF9F00C104200081004400F1B79F00B3
:10EE90002008200000004400E0B79F00E80644007E
:10EEA000B8489000811F780068009000F80090003A
:10EEB000809FBE00A8489000811F7800CFB39700C4
:10EEC0003FB39700AFB2970009027800080990009D
:10EED0009809900041C0B3000D00780043FE070080
:10EEE00000057800E88757000A00E0003E003A007D
:10EEF000281191000040EB008005EB000A0037006C
:10EF00006112B000E8C07800040037008180FB0087
:10EF1000E1816000838545008100D1000104E000AB
:10EF2000FAFF3A000040E8008080FB00828F50002A
:10EF3000F3FF350076805700ECC0020000000000AF
:10EF40000046EB00230037006158B900E6FC0700DB
:10EF5000AE15200008074700800078000E007800FA
:10EF600092C0020000000000E20E200008014100F3
:10EF700043122000888141008E007800090078004B
:10EF800082FF070038489000801F780068009000DA
:10EF9000F8009000809FBE00A8489000811F780074
:10EFA000CFB397003FB39700AFB297000902780044
:10EFB000080990009809900041C0B3000D00780046
:10EFC0000AFE0700E88757000000E00005003A004D
:10EFD0000C46E8002FE89700804F5600DAFF390012
:10EFE00002003700000578003A0498000A00780013
:10EFF0004F0778004F06BE004F05BE004F04BE000D
:10F00000AF00B10000000600881F780000047800FF
:10F01000080078009FFC0700300498000000E00022
:10F0200004003A00680044008040EB00DAFC07006E
:10F0300030049800380090004F047800000006006B
:10F04000881F780000047800380090000000E0007D
:10F0500017003A001804E00015003A000800E80024
:10F06000ECC002000000000018009000A800900012
:10F0700061004000E08048001004980021049800DE
:10F0800018409000F74F500007003E000080FB0042
:10F0900000004000C1442300E1007800080078002F
:10F0A0000100010002003700080078001BFC070087
:10F0B000380090004F0478000000060000000600B1
:10F0C0009001FA0000E72F000F004000CEFF07007C
:10F0D0000300370000E72F000F004000D8FF0700B3
:10F0E0003F3896000000E00003003A008FF09400E3
:10F0F0000104E000F7FF32000080FA000000060083
:10F1000001012000404F200044BD0200000000002B
:10F11000C050230010407800614060009AA30200B4
:10F120000000000000C2B3008CA302000000000039
:10F13000204A2300104078009AA30200000000003B
:10F1400000C2B3008CA3020000000000A0D62A0079
:10F15000AEA4040000000000881F780010300200F8
:10F1600000000000902E0200000000000004780063
:10F170001030020000000000902E0200000000008D
:10F180008800E900E18F500007003E00C1502300D5
:10F190000844E90061446400114178000204A100C0
:10F1A00088487100010037000000EB008000E90092
:10F1B000E38F50001D003E00214A23008048E900F3
:10F1C000CFFF0700C05023001014A1001300370028
:10F1D000B1032000804520008ABD0200000000002D
:10F1E0008001EB004200200006003700C102200031
:10F1F000804C200044BD0200000000008001EB00B4
:10F2000032002000110020001000200026300200F3
:10F2100000000000214A23008048E900404B230001
:10F220001044A0004F047800000006004030230086
:10F230000048EB0051022000304320008ABD02004C
:10F24000000000008001EB002200200011002000DF
:10F25000100020002630020000000000C1502300F2
:10F260000040E90061406000114178000204A10003
:10F2700000407100804878000008A300D4FF3200ED
:10F28000DAFF3700C1502300114078000010A100C0
:10F29000804878000008A3000200320007E2A900BD
:10F2A00077E2A90000000600B100200050442100D0
:10F2B0008ABD040000000000C05023001040780008
:10F2C0006440600004003A007602A8007602AB00B9
:10F2D000FEFF3A00000006000602A8000602AB008E
:10F2E000FEFF3A0000000600C050230010407800E6
:10F2F0006440600004003A007642A8007642AB0009
:10F30000FEFF3A00000006000642A8000642AB00DD
:10F31000FEFF3A0000000600C050230010407800B5
:10F320006440600003003A00C01380004F00DE001C
:10F3300000000600401080004F00DE0000000600C4
:10F34000C150230091407800E4C06000614060003B
:10F350000104E0000A003A00E1006000C508DD0099
:10F36000B01380000050A10000807000B01388002E
:10F370007682A8007682AB00FEFF3A00000006000D
:10F38000E1006000C508DD00301080000050A100E1
:10F3900000807000301088000682A8000682AB0052
:10F3A000FEFF3A0000000600881F7800C8502300C6
:10F3B0009840780062C060001200320041002000D6
:10F3C0006041200044BD020000000000C0D62A00B9
:10F3D000AEA4020000000000184478006140640000
:10F3E00004003A0010C0B3001AB50200000000008B
:10F3F0000200370010C0B300D1FF0700C050230047
:10F400001014A100C050230010407800614060003B
:10F4100003003A0088B40200000000000100370039
:10F42000B1FF0700C1002000704220008ABD020029
:10F43000000000004F04780000000600881F7800DC
:10F44000C85023009840780062C06000120032006B
:10F45000410020006041200044BD02000000000087
:10F46000C0D62A00AEA402000000000018447800B4
:10F470006140640004003A0010C0B3001AB50200F5
:10F48000000000000200370010C0B300ACFF07000E
:10F49000C05023001014A100C05023001040780079
:10F4A0006140600010003A00A4B4020000000000B7
:10F4B0000000E0000D00320091002000C02020007C
:10F4C00044BD020000000000510120005021200036
:10F4D00044BD020000000000C0D62A00AEA4020015
:10F4E000000000000100370073FF0700D10020007A
:10F4F000A04120008ABD0200000000004F047800F7
:10F5000000000600C150230091407800E4C0600074
:10F510000080FB000104E00004003A009013880022
:10F5200079C2AB00FEFF3A00000006001010880010
:10F5300009C2AB00FEFF3A0000000600889FBE0033
:10F5400000047800C95023009940780062C0600030
:10F550001400320000C2B3008CA3020000000000BF
:10F56000310020003041200044BD020000000000B6
:10F5700000C2B3008CA30200000000009944780090
:10F5800061C0640003003A001AB5020000000000E8
:10F59000020037000040EB0069FF0700C050230065
:10F5A0001014A100C050230010407800614060009A
:10F5B00006003A000800780038B50200000000009C
:10F5C0008EB50200000000000300370008407800FC
:10F5D000CCFF070050FF07000084FB0000C2B3000F
:10F5E0008CA30200000000000800E00006003A00C2
:10F5F000310020003041200044BD02000000000026
:10F60000003020000500370041002000604120004C
:10F6100044BD020000000000001020004F04BE00A6
:10F6200000000600C05023001040780064406000D5
:10F6300005003A007662A8007662AB00FEFF3A0051
:10F6400080138000000006000662A8000662AB007E
:10F65000FEFF3A000010800000000600C0502300AA
:10F66000104078000018A300140032000008A30026
:10F6700004003A000040EB001AB502000000000050
:10F68000020037000040EB002DFF070000C2B3006E
:10F690008CA3020000000000310020003041200057
:10F6A00044BD02000000000000C2B3008CA30200B1
:10F6B00000000000C05023001014A100C05023001F
:10F6C000104078006140600003003A00B0B50200CD
:10F6D0000000000001003700D2FF0700C1502300E6
:10F6E0001114A0000080FB00000006007742A90072
:10F6F0007782A9007A22EF007C22EF007702A9002E
:10F70000204A23001080FB0071DC2A006140780051
:10F710000080FB00A013880077E2A800000006002C
:10F72000C0502300104078006140600009003A009A
:10F73000D822A800D842A800DA42A900DA22A900FB
:10F74000204A23009040780020C0B300E4B30400B6
:10F7500000000000E5FF3700889FBE008A9FBE00C2
:10F760008C9FBE008E1F7800004778006AA60200BA
:10F7700000000000D822A800D842A800DA42A90060
:10F78000DA22A9006640A8006660A8008660A90089
:10F79000DA02D500D81680004244DE0061446400DD
:10F7A000E14460000046EB008C4578008C46780010
:10F7B00008003700004478008A44780005003700CC
:10F7C0008A4478000044EB000200370019C0B300FF
:10F7D000094478008660AB000D003A006CA6020078
:10F7E000000000004CA60200000000000004E00041
:10F7F000F8FF320060A60200000000006640A90089
:10F800006660A9000E04E0004E0032004A00370096
:10F810008660A900DA02D50061456000D01680003C
:10F820004200DE00614060000D04E000280032006C
:10F830000804E00028003A000004E000DEFF320087
:10F84000E7CF550008003E000C4646000A04E000E1
:10F85000010032000C04A0008B45E8008A447800C7
:10F8600018C0B300DBFF37000E04E00004003200D4
:10F870000C80FB0026A602000000000006003700F6
:10F88000C0C5B30024A60200000000000C407800B0
:10F8900024A60200000000000A04E0000600320076
:10F8A000D0C2B30024A60200000000008045EB0097
:10F8B00018C0B3001E003700B0C2B30024A6020077
:10F8C000000000008045EB0018C0B3000E003700B8
:10F8D0000804E000B7FF32000004E000B8FF320087
:10F8E0000904E0000A0032000A04E000B7FF3A0011
:10F8F000B0C5B30024A60200000000008045EB0064
:10F900001DC0B3000D4478008B447800B1FF370070
:10F9100018C0B3000A04E000AEFF3200D0C5B30047
:10F9200024A60200000000008045EB008B46780012
:10F9300088447800A7FF3700C0D62A00AEA4020092
:10F94000000000004F0778004F06BE004F05BE00C4
:10F950004F04BE0000000600881F78008000EB0006
:10F96000E40F5000E08F5800A0003E00006001004E
:10F9700004003700080037006B0037007F003700B5
:10F9800091003700B10720004050200044BD020024
:10F9900000000000990037008040EB00600020006C
:10F9A00040B4020000000000E1022000F0572000F7
:10F9B0008ABD020000000000C05023001040780003
:10F9C0006440600006003A00DA42AB0009003200F1
:10F9D0000004EB00DA22AB000F003A00050037000C
:10F9E0000004EB00DB22AB000B003A00DB42AB0073
:10F9F00009003A0091002000C020200044BD020010
:10FA000000000000510120005021200044BD0200F0
:10FA10000000000040003700C05023001040780074
:10FA20006140600008003A00A4B402000000000039
:10FA30000800780038B50200000000008EB5020012
:10FA400000000000040037001BFE0700084078009B
:10FA5000ACFE070030FE07000080FB0022003A00E9
:10FA6000080078003EBB02000000000080C2B30026
:10FA70008CA30200000000000880D1003EBB020001
:10FA800000000000D0D62A000808A3000E003200B3
:10FA9000C0502300104078006140600006003A002A
:10FAA000B0B502000000000010C0B3001AB502009B
:10FAB0000000000003003700DAFE070010C0B300AA
:10FAC0001FFE070000D72A00C8A4020000000000A3
:10FAD000A0D62A00C8A402000000000000C2B300A3
:10FAE0008CA3020000000000C050230010407800EA
:10FAF0006140600003003A0088B40200000000008A
:10FB000001003700F8FD07000804E800001020009D
:10FB1000800F5400C0FF3A00C0D62A00AEA40200F5
:10FB20000000000035003700C0502300104078006E
:10FB3000614060000100320007E2A900710020006E
:10FB4000D05A20008ABD020000000000F100200011
:10FB5000003321008ABD02000000000010C0B30085
:10FB6000FDFE0700C0502300104078006140600097
:10FB700022003200DDFE07002000370030D72A00C7
:10FB8000AEA4020000000000C05023001024A0001A
:10FB90000742A9000782A9000A22EF000C22EF0009
:10FBA0000702A900204A23001080FB0071DC2A0014
:10FBB000614078000080FB002010880007E2A80068
:10FBC00077E2A9000D003700C050230010407800F4
:10FBD0006440600009003200B0D92A00AEA40200DF
:10FBE00000000000DB62A900040037004102200091
:10FBF000E01D20008ABD0200000000004F047800D4
:10FC00000000060020DC2A00C8A404000000000058
:10FC1000889FBE008A9FBE00D822A800D842A800B4
:10FC2000DA42A900DA22A900D882A900414B2300B8
:10FC3000114078000040A0000034A1008048780006
:10FC400080C0EB0020C0B300E4B30200000000005D
:10FC5000ECFF070060A6020000000000F450230043
:10FC6000004A78000081FB004411DE00E1502300CF
:10FC7000824878000281FB008001EB00E60F510012
:10FC8000E08F5900D3003E000260010006003700FB
:10FC9000AB003700CF003700CE003700C60037007A
:10FCA000C9003700BE0037000080FB008000EB0079
:10FCB000EF0F5000E08F5800C6003E0000600100CA
:10FCC000C8003700E2FF37000D0037000F00370093
:10FCD00011003700BF003700120037001300370053
:10FCE0001600370063003700BA003700B90037004C
:10FCF000B8003700B7003700B60037008D00370076
:10FD0000A4B4020000000000AD00370088B4020077
:10FD100000000000AA003700B0B50200000000009B
:10FD2000AD0037000040EB000100370010C0B30009
:10FD30001AB5020000000000A100370060A6020012
:10FD4000000000004804DD0060A602000000000082
:10FD50000085FB000805750060A602000000000099
:10FD60000044780060A602000000000001002100AD
:10FD7000810F550097003E00C844DD000080FB0065
:10FD8000890470000004EB00818F540007003600E6
:10FD900090003700A04C23009005440060A60200AC
:10FDA00000000000804D78000804E8008A0F54002D
:10FDB000F8FF3900A4B40200000000000004EB00CA
:10FDC0000A00370050A6810060407C000080FB00E4
:10FDD00038B50200000000008EB5020000000000EF
:10FDE000E14F50007B0032000804E8008A0F540005
:10FDF000F4FF39000905E9000004EB000C003700AE
:10FE0000A04C230090054400B0B5020000000000A3
:10FE1000804D78000040EB008A0F5400010039004B
:10FE200010C0B3001AB50200000000000804E8008A
:10FE3000890F5400F2FF390088B40200000000006E
:10FE400010C0B3008CA30200000000000004EB000F
:10FE50000500370050A6810060407C008CA30200A2
:10FE6000000000000804E800890F5400F9FF390081
:10FE700078FF370010C0B3008CA302000000000020
:10FE80002202AB00FEFF32003111800001407800F9
:10FE9000F250230001497800E2CF500014003200F4
:10FEA00005003E000104E0000B003200E1CF5000ED
:10FEB0001E003A000B003700F0CF50001200320055
:10FEC00001C2B300814F500013003200E34F5000D5
:10FED00016003A0009003700F88502000000000013
:10FEE00012003700C6850200000000000F00370036
:10FEF0009C850200000000000C0037002A860200EA
:10FF00000000000034003700404B2300C1CFB30095
:10FF100010C8600005003700414B230011407800F5
:10FF20000000A0000014A10080487800100020000C
:10FF3000290037000040EB0007FE070020003700D3
:10FF40006F406000004AE80010C0B3008CA30200BC
:10FF500000000000D05023000048EB000A003700EA
:10FF600060A60200000000000080FB0038B502001F
:10FF7000000000008EB50200000000008CA302000B
:10FF800000000000184CE800D8502300F050230077
:10FF90009840780090CF5000F1FF39002DFF3700D6
:10FFA000E3406000014A780020C0B300E4B30200DF
:10FFB000000000000200370072C1020000000000D3
:10FFC00010C0B30004003700B8C1020000000000F8
:10FFD000010037000040EB008CA30200000000008D
:10FFE0001CFF37004F05BE004F04BE000000060096
:10FFF000E30F500003003E0010A1A8001081A800EC
:020000040001F9
:10000000E0030500FE0F500003003E0010A1A80011
:100010001081A900A00F0500410F2000810F5000A2
:1000200004003E0010A1A9001081A800007D20005E
:100030000000060010A1A9001081A90000E823001B
:10004000000006001021EF001E21EF00B821EF0094
:10005000E0A381000000E00004003A0001FC2F0052
:10006000426D20001289600016003700E0FF070093
:10007000E2A38100110009000280D8000000E9001D
:1000800060088800F1A381000180B90042062000C9
:10009000110009000280D8008000FD0000FC2F0044
:1000A000D406B6006001B300A0368800F10D8800C8
:1000B000E10D880060002000C00D880011E1A8005B
:1000C0002000200000A4890000000600889FBE00D8
:1000D0008A9FBE008C9FBE001021EF001E21EF0002
:1000E000B821EF0000A48100E20F50000F003A0099
:1000F00000FC2F00D426B600C1002000E02B200019
:100100008ABD0200000000000000EB0000A489008E
:10011000109881000000E800F00FB20001202300D9
:10012000614078000004E000700032001098810007
:100130000000E800F00FB2001098890010300200B3
:1001400000000000902E02000000000080047800F3
:100150001030020000000000902E0200000000009D
:10016000CF80DE00A2240200000000000005BE00D7
:100170008900E90018002000E0F92000808F50007D
:10018000010036000004EB006011B8000A00BE0058
:1001900026240200000000000000E0000A003400F5
:1001A00002002000832C24000A00BE00222402004A
:1001B000000000000000E00003003D00E10F5400DB
:1001C0001300320018002000403023000048EB00EC
:1001D00011012000A02C20008ABD020000000000B8
:1001E00011012000B02D200044BD020000000000DD
:1001F0008001EB0002FA2000110020002003200003
:100200002630020000000000800478000100370062
:10021000280020000900780075FF07001100090080
:100220000980D8008004E900E20F54000E0032007B
:1002300001012000902F200044BD020000000000BA
:100240008001EB00320620008000EB00200320003C
:100250002630020000000000CF80DE00A224020051
:10026000000000000005BE006148B800062502003D
:10027000000000000006BE0002002000832C2400C5
:100280000A00BE0080230200000000000001BE0042
:100290000C00BE00B0250200000000006C2402002B
:1002A000000000000001BE0001FC2F00A03680000D
:1002B000808060006101B300A1368800F20D8800E3
:1002C000E20D880060002000C00D880069088800E9
:1002D00011E1A800A1002000903020008ABD02009A
:1002E000000000002000200000A489004F06BE008E
:1002F0004F05BE004F04BE00000006000EA1EF0037
:100300000CA1EF000821EF000621EF001621EF00FD
:100310001421EF0080002000F0088800400F20002A
:10032000E008880000402200D00888008780A900EB
:100330001FE1A80011E1A8008780AB00FEFF32009A
:1003400011E1A9001FE1A9003108800001A5890081
:10035000420880008001EB00C011DD000200200097
:1003600002804000E0804900E0A48900F1A48900F7
:10037000000006001E21EF001021EF00D8A2A80007
:1003800000FC2F008606B6004001B3003034880020
:10039000A003200080088800D8FF0700F20F20008B
:1003A000820F5000E08F5800050036004809DD003C
:1003B000C801DE00830171004801DD000400370040
:1003C000A000200080088800CCFF07000001BE00CC
:1003D00001FC2F003034800080806000F101B30008
:1003E000313488001E21EF001021EF000200BE0012
:1003F00000000600889FBE008A9FBE008C9FBE0042
:100400008001780084A0A9008420A900F10F2C00AD
:100410007034800080806000004021000100700086
:100420007034880002FC2F007034800000016100ED
:100430004201B300723488001621EF001421EF004E
:1004400080002000F00888001FE1A80030C02000D4
:10045000400A880030802000000A88004001200007
:10046000500A8800100A8800B0A48100C1A481004D
:1004700002003700200A80008000EB004061AB00E2
:10048000FCFF3A00B0A48900C1A489000100370034
:10049000600A80004861AB00FDFF3A004061AB009C
:1004A000FEFF32002C0A80008006EB009CA489002D
:1004B000ADA489006A0A80008005EB005AA4890077
:1004C0006BA489006000B80010A4890021A48900F1
:1004D000B6A48100C7A4810074A4810085A4810012
:1004E00038A4810049A481000001EB00130037000B
:1004F0004061AB00FEFF3200260A80008003EB0063
:10050000640A80008002EB000C0653008D865B00BD
:100510000A0552008B855A00C055DD000A002000F4
:100520000C0445008D844D000000440081804C0087
:100530000201E8000405BE000606BE00830F51005C
:10054000EBFF3900B6A48900C7A489009CA48900E8
:10055000ADA4890074A4890085A489005AA48900E7
:100560006BA4890038A4890049A4890010A48900DB
:1005700021A48900D2A489004021EF004221EF008C
:100580001FE1A9006119B800182602000000000050
:100590004F06BE004F05BE004F04BE00000006001F
:1005A000889FBE008A9FBE0000A48100E20F500019
:1005B00005003A00F1012000303120008ABD020020
:1005C0000000000059013700F10020002033200016
:1005D00044BD0200000000001E21EF001021EF00CA
:1005E000D8A2A80000FC2F008606B6004001B30088
:1005F00030348800A0032000800888003FFF0700F7
:100600000004BE006055B800F2FF2300820F5000C6
:10061000E08F580005003600C84CDD004840DE0081
:10062000890470004844DD000D003700B10020004F
:10063000202E210044BD020000000000A000200088
:10064000800888002DFF07000004BE006055B80038
:10065000F2F92000820F5000E08F580004003600AD
:100660000800BE00DAA402000000000026013700E6
:10067000E0DC2A00E00F5400E08F5C00E00F5D003A
:10068000E08F5D0021013200B1002000202E21000A
:1006900044BD0200000000000800780055FF07007C
:1006A0006011B80004A82100650020006033B80084
:1006B0000400E1000588E1000690E1000798E100F0
:1006C0004E003600A8240200000000000001BE0019
:1006D000703B2400A13B25008023020000000000A5
:1006E0002A240200000000000205BE000004BE0033
:1006F000046A2800150020006033B8007C2702003F
:1007000000000000DAA4020000000000E0C2B30014
:100710008CA3020000000000046A280015002000DD
:100720006033B8000800BE000A01BE008A2702003C
:10073000000000000205BE000004BE00F0702200B0
:10074000010020006011B8000040E10001C8E10094
:1007500002D0E10003D8E10024003E0000C3B30052
:100760008CA3020000000000703E20000100200069
:100770006011B8000040E10001C8E10002D0E100D2
:1007800003D8E10019003E0000C3B3008CA30200AF
:100790000000000030062000010020006011B800B9
:1007A0000040E10001C8E10002D0E10003D8E1000F
:1007B0000E003E0000C3B3008CA302000000000046
:1007C00090002000010020006011B8000040E1000E
:1007D00001C8E10002D0E10003D8E10003003E00BF
:1007E00000C3B3008CA30200000000000800BE009C
:1007F0004AA4020000000000C3003700B4E12E004C
:10080000150020006033B8000400E1000588E10015
:100810000690E1000798E1002A003600A8240200B3
:10082000000000000001BE00902F20005121250093
:1008300080230200000000002A24020000000000C3
:100840000205BE000004BE00047122000500200065
:100850006033B8007C27020000000000DAA4020028
:1008600000000000E0C2B3008CA302000000000002
:1008700004712200050020006033B8000800BE00AB
:100880000A01BE008A270200000000000205BE0027
:100890000004BE00703E2000010020006011B8007E
:1008A0000040E10001C8E10002D0E10003D8E1000E
:1008B00040003E0000C3B3008CA302000000000013
:1008C0002600370004C42900050020006033B8006A
:1008D0000400E1000588E1000690E1000798E100CE
:1008E00038003600A8240200000000000001BE000D
:1008F00080B22600E10625008023020000000000EF
:100900002A240200000000000205BE000004BE0010
:10091000843E2000050020006033B8007C270200E0
:1009200000000000DAA4020000000000E0C2B300F2
:100930008CA3020000000000843E2000050020007F
:100940006033B8000800BE000A01BE008A2702001A
:10095000000000000205BE000004BE0030062000BA
:10096000010020006011B8000040E10001C8E10072
:1009700002D0E10003D8E1000E003E0000C3B30046
:100980008CA3020000000000900020000100200065
:100990006011B8000040E10001C8E10002D0E100B0
:1009A00003D8E10003003E0000C3B3008CA30200A3
:1009B00000000000080078000AA402000000000007
:1009C0005100370094162300050020006033B80062
:1009D0000400E1000588E1000690E1000798E100CD
:1009E0002B003600A8240200000000000001BE0019
:1009F00000C22B00E1EB2400802302000000000075
:100A00002A240200000000000205BE000004BE000F
:100A100044062000050020006033B8007C27020057
:100A200000000000DAA4020000000000E0C2B300F1
:100A30008CA30200000000004406200005002000F6
:100A40006033B8000800BE000A01BE008A27020019
:100A5000000000000205BE000004BE00900020005F
:100A6000010020006011B8000040E10001C8E10071
:100A700002D0E10003D8E10003003E0000C3B30050
:100A80008CA3020000000000084078001C00370022
:100A9000A8240200000000000001BE000068290038
:100AA00081D1240080230200000000002A240200DB
:100AB000000000000205BE000004BE00A4002000EB
:100AC000050020006033B8007C2702000000000011
:100AD000DAA4020000000000E0C2B3008CA3020010
:100AE00000000000A4002000050020006033B800D2
:100AF0000800BE000A01BE008A27020000000000B4
:100B00009AA3020000000000A0DC2A00AEA40200AC
:100B10000000000000FC2F008606B600F001B300C4
:100B2000303488001E21EF001021EF004F05BE0079
:100B30004F04BE0000000600404B23001040780028
:100B4000634060000080FB00E20F500008003200AC
:100B5000E30F500008003200E10F500002003200A5
:100B6000D8A2A80005003700D882A80003003700EB
:100B7000D902A80001003700D802A800E100200037
:100B80001034200044BD040000000000404B23004E
:100B900010407800634060000080FB00E20F5000CE
:100BA0000A003200E30F50000B003200E10F50004A
:100BB00003003200D8A2A900DAA2A800080037007A
:100BC000D882A900DA82A80005003700D902A9005E
:100BD000DB02A80002003700D802A900DA02A80050
:100BE00081002000F03420008ABD040000000000D5
:100BF000404B230010407800634060000080FB0001
:100C0000E20F50000A003200E30F50000B003200E8
:100C1000E10F500003003200D8A2A900DAA2A90017
:100C200008003700D882A900DA82A9000500370041
:100C3000D902A900DB02A90002003700D802A900EE
:100C4000DA02A90071002000703520008ABD04007E
:100C500000000000404B230010407800634060001B
:100C60000080FB00E20F500010003200E30F500044
:100C700014003200E10F500006003200D8A2A80094
:100C80000000000000000000D01680004500DE00DB
:100C900010003700D882A80000000000000000000B
:100CA000D01680004400DE000A003700D902A800F8
:100CB0000000000000000000D01680004800DE00A8
:100CC00004003700D802A800000000000000000067
:100CD000D0168000614060000080FB00000006002C
:100CE000889FBE008A1F78001021EF001E21EF00B0
:100CF000B821EF0000A48100E20F500010003A007C
:100D0000109881000000E800F00FB20001202300DD
:100D1000614078000004E00009003A0000FC2F0068
:100D2000D426B600C1002000E02B20008ABD0200BE
:100D3000000000000000EB0000A489005F00370005
:100D4000109881000000E800F00FB20010988900B0
:100D50001030020000000000902E02000000000091
:100D6000413023001104E0000B003A00CF80DE0088
:100D7000A2240200000000000004BE0002002000C7
:100D80004333240026240200000000000045EB004D
:100D90000000E00011003400403023000048EB0068
:100DA00031012000803821008ABD020000000000CF
:100DB0008001EB00420B20008000EB00A00520002A
:100DC0002630020000000000CF80DE00A2240200D6
:100DD000000000000004BE001AC0B30010A1A8006B
:100DE0001081A80002002C00A35524000800BE00BA
:100DF000802302000000000002002400C3492400F8
:100E0000B02502000000000002002000832724001B
:100E1000C6220200000000006C2402000000000056
:100E20000001BE0001FC2F00A03680008080600021
:100E30006101B300A1368800F20D8800E20D880040
:100E400060002000C00D8800204E2000600888004F
:100E500011E1A800C1002000B03921008ABD0200C4
:100E6000000000002000200000A48900E14F550090
:100E700012003A0013002000420B20008000EB001B
:100E80000080EB002630020000000000CF80DE0072
:100E9000A2240200000000000004BE006011B8009F
:100EA00022240200000000000000E000CBFF3D0013
:100EB00030DF2A00AEA40200000000004F057800D9
:100EC0004F04BE0000000600A0E72A00C8A40400EA
:100ED00000000000889FBE008044780068C0B30016
:100EE00061C064001AB50200000000008984FB00A4
:100EF0008904D1000844E900F9FF3A00B0B50200C6
:100F0000000000008CA3020000000000B0B5020049
:100F1000000000008CA30200000000004F04BE008F
:100F200000000600889FBE008A9FBE008C1F7800CC
:100F30000044780081447800824578000CC8B300F2
:100F40000C4664006AC0B300614064001AB5020038
:100F5000000000000884FB000804D1000A45E900F5
:100F6000F9FF3A000C04E00006003A000980FB009B
:100F700038B50200000000000B80FB0038B502000D
:100F8000000000004F0678004F05BE004F04BE0071
:100F900000000600889FBE008044780048C0B3006F
:100FA00010C0B3000908A30001003A000040EB00A4
:100FB0001AB50200000000000844E90003003200F6
:100FC0008984FB008904D100F5FF3700B0B5020029
:100FD00000000000B0B50200000000008CA3020079
:100FE000000000004F04BE0000000600889FBE0005
:100FF0008A9FBE008C1F78000044780081447800EE
:10100000024678008885FB00C65DDE000045EB00E7
:10101000E34F55000C003A000B04E0000A003200D8
:1010200010C0B30006B50200000000000B80FB00FA
:10103000F6BB0200000000000040EB0006B5020015
:1010400000000000080037000884FB0010C0B30057
:101050000808A30001003A000040EB001AB50200A6
:10106000000000000804D1000A45E800E44F5500E4
:10107000E7FF3A000980FB0038B5020000000000DD
:101080000C80FB0038B50200000000004F0678001D
:101090004F05BE004F04BE00000006000040EB00FC
:1010A0001AB50200000000000040EB001AB5020073
:1010B000000000000040EB001AB502000000000034
:1010C0000040EB001AB50200000000000000EB0039
:1010D00038B50200000000000000EB0038B5020047
:1010E000000000000000EB0038B504000000000024
:1010F000889FBE0000047800814478000040EB0027
:101100001AB50200000000000040EB001AB5020012
:10111000000000000040EB001AB5020000000000D3
:101120000040EB001AB50200000000001880FB0030
:1011300038B5020000000000184090000080FB005D
:1011400038B5020000000000284090000080FB003D
:1011500038B5020000000000EFC464000200370050
:10116000CEFF07008944E9000904E000FCFF3A00D3
:101170004F04BE0000000600889FBE008A1F780052
:101180000004BE00024578000040EB001AB50200E2
:10119000000000000040EB001AB502000000000053
:1011A0000040EB001AB50200000000000040EB0018
:1011B0001AB50200000000000800780018BC020008
:1011C0000000000038B50200000000004849DD00C2
:1011D0004840DE0000007100C848DE0018BC020074
:1011E0000000000038B50200000000004048DE00AA
:1011F0000100200018BC02000000000038B5020009
:10120000000000006F4565000044EB00020037005D
:10121000A2FF07000844E8008A4F5400FCFF390091
:101220004F0578004F04BE0000000600881F7800BC
:1012300010C0B3001AB50200000000000040EB002F
:101240001AB50200000000000040EB001AB50200D1
:10125000000000000040EB001AB502000000000092
:101260000000EB0038B5020000000000B0B502003D
:101270000000000000047800B0B50200000000008B
:101280008CA3020000000000084078008CA302003C
:101290000000000081FF070080FF07004F04780076
:1012A00000000600881F7800414B230011407800A1
:1012B0000040A0000034A1008048780018C0B300AE
:1012C000728050000848780081C0B3000000E80038
:1012D0000148780020C0B300414C230080487800CA
:1012E00080C0EB00E4B3020000000000D822A90097
:1012F000D842A900D862A80008407800FCB40200D7
:1013000000000000F0FE070060A6020000000000E0
:10131000824C2300004978000082FB004422DE005A
:10132000714C2300844878000482FB008002EB00AB
:10133000046001000F003700560037008C003700B2
:10134000920037000302370005023700070237001A
:10135000420237000A02370040023700A800370077
:101360003E0237003D0237003C0237003B023700A7
:10137000250237000080FB008000EB00ED0F5000DD
:10138000E08F580035023E00006001003702370050
:10139000DCFF37000B0037000D0037000F0037006F
:1013A000150237000F0037002600370028003700ED
:1013B0002A0037002B0037002C0037002F003700A1
:1013C00030003700A4B40200000000002102370002
:1013D00088B40200000000001E0237000040EB004D
:1013E00006023700404C230021C0B30090CF10000C
:1013F00003003A00B0B5020000000000030037000F
:10140000F00F2000EAB5020000000000614C23004C
:1014100080487800404B230010407800684060000E
:1014200005003200684C23001880FB0018BC020045
:1014300000000000004C7800604C23001040780051
:10144000070237008EB502000000000004023700DA
:101450008AB50200000000000102370010C0B3008E
:10146000470037000040EB000100370010C0B30018
:1014700006B5020000000000F60137000040EB0056
:101480000100370010C0B30010B5020000000000DA
:10149000F00137006F4060000049E80010C0B30061
:1014A0008CA3020000000000604C23000048EB0009
:1014B0002900370060A6020000000000584C2300FD
:1014C000004C7800414B230091407800E8C0600058
:1014D000040032000080FB0018BC02000000000085
:1014E000004C7800584C2300404C230021C0B3002E
:1014F00090CF100005003A001880FB0038B50200BC
:101500000000000010C0B3000F0037001880FB007F
:10151000EAB502000000000080407800004C78002E
:10152000404B230010407800684060000400320007
:101530000180FB0018BC020000000000004C780095
:10154000504C2300104078008CA3020000000000E3
:10155000604C23001048E800804C2300614C2300BD
:101560009140780090CF5000D2FF390066FF3700DD
:101570006F4060000040E800814C23008048780004
:1015800064B4020000000000B20137006F40600048
:101590000049E80010C0B3008CA302000000000066
:1015A00060A6020000000000714C23008048780013
:1015B000604C23000048EB000B003700784C230000
:1015C00010C0B3001804E000010035000040EB003B
:1015D0001AB502000000000018407800004C4000DE
:1015E000604C23001048E800804C2300614C23002D
:1015F0009140780090CF5000F0FF390095013700FE
:1016000041CAB300814F50001100320004003E0077
:10161000E4C05000814F500090013A0007003700AD
:1016200051CAB300814F50008100320081C0E800F0
:10163000814F500089013A00D500370060A60200B2
:1016400000000000415123008048780081013700EC
:101650004051230010407800E14F50000300320059
:10166000E24F50007D013A002300370060A60200DF
:10167000000000000080FB006300B90010A6890094
:101680000000EB0007003700A04C230010044400CA
:1016900060A6020000000000004C7800E0A5810078
:1016A0000000E800E0A58900E8A5810010A68100FF
:1016B000800F5400F4FF39000000EB0008003700F1
:1016C00053A681008080410021419000914090000C
:1016D0006340780045FE0700E0A5810063004000FC
:1016E000E0A58900E0A5810011A68100810F5000CE
:1016F000F3FF39005701370060A602000000000028
:101700000080FB004200DD0010A689000000EB0015
:1017100007003700A04C23001004440060A602001C
:1017200000000000004C7800E0A581000000E80007
:10173000E0A58900E8A5810010A68100800F540073
:10174000F4FF39000000EB00330037000040EB00ED
:101750001AB50200000000000040EB001AB50200BC
:10176000000000000040EB001AB50200000000007D
:101770000040EB001AB5020000000000E0A5810067
:1017800051A68100614078000080FB0038B502005E
:1017900000000000E0A5810051A68100008040000B
:1017A000104090000080FB0038B5020000000000EF
:1017B000E0A5810051A681000080400020409000FB
:1017C0000080FB0038B5020000000000E0A58100A9
:1017D00063004000A14C23001100400090407800BD
:1017E0006FC86000604C23000048EB000200370027
:1017F0002AFE0700184CE800E0A58100684C230091
:1018000051A6810080804000B140900098CF100028
:10181000F7FF390064004000E0A5890010A68100B0
:10182000E1A58100808F5000C8FF39000901370011
:101830004051230010407800E14F50000300320077
:10184000E24F5000B0FE3A003000370060A60200C0
:10185000000000000080FB0010A6890060A60200C6
:1018600000000000714C2300804878000000EB006D
:1018700020003700714C2300504C230011487800A1
:10188000604C23000048EB000E003700584C23004A
:101890001880FB000008A3000200320010C0B30053
:1018A000010037000040EB001AB502000000000004
:1018B0001880FB000000D100004C7800604C230031
:1018C0001048E800604C230031C0B30090CF1000F6
:1018D000EEFF3600B0B5020000000000B0B5020017
:1018E000000000008CA3020000000000E0A58100C1
:1018F0000000E800E0A5890010A68100E1A58100B4
:10190000808F5000DBFF39007FFE370060A60200A9
:10191000000000000080FB0010A689000000EB0022
:101920001500370022C0B30060B92000A10B2000D1
:1019300011FE07003DFE070022C0B30060BB2D0072
:10194000A10B20000CFE070022C0B300603D2D005B
:10195000A10B200008FE070034FE070022C0B300E0
:1019600060BB2000A10B200003FE07002FFE070034
:10197000E0A581000000E800E0A5890010A6810034
:10198000E1A58100808F5000E6FF39005EFE370040
:1019900060A60200000000000080FB0000A6890095
:1019A00060A60200000000000080FB00F0A5890096
:1019B0004151230091407800E2CF500004003A00EA
:1019C00002A681006511B90002004000080037003E
:1019D000E1CF500002003200E3CF50009F003A00F8
:1019E00001A681008180400001004000000040000D
:1019F00010A689000000EB0007003700A04C230070
:101A00001004440060A6020000000000004C7800B2
:101A1000E0A581000000E800E0A58900E8A58100BC
:101A200010A68100800F5400F4FF3900F0A581005A
:101A30000000E0000300320010C0B3008CA30200DD
:101A4000000000000000EB003900370050A68100C4
:101A500060C17800E14F51001E003A00425123005E
:101A600012417800E34F510006003A0001004000A7
:101A700030419000A04090001040900029FD0700E8
:101A800007003700E14F510008003A000100400014
:101A900030419000A04090001040900053FD07009E
:101AA000E0A581006400400021003700E24F5100B2
:101AB00020003A00010140008100E80001004000E0
:101AC000C24090008AFD0700E0A58100650040004B
:101AD00017003700E24F510016003A004251230030
:101AE00012417800E34F510004003A000100400029
:101AF00010409000F7FC070005003700E14F51004F
:101B000006003A00010040001040900021FD07004F
:101B1000E0A581000080E80005003700E24F510099
:101B200004003A00C1FD0700E0A581000000E800C4
:101B3000E0A58900E1A5810010A68100808F5000FA
:101B4000C2FF3900F0A581000000E000EEFD3A0080
:101B50004000370072C10200000000003D00370065
:101B6000B8C10200000000003D003700E340600003
:101B700001497800204A2300014878001A00370004
:101B8000424B2300924078000140A10001497800B7
:101B90000080FB000038A30002003A000144A000CE
:101BA00001497800414C230022C0B30082487800EC
:101BB0000028A3000200320032C0B300824878003F
:101BC000424B2300924078000130A1000149780087
:101BD0000018A300020032000134A000014978007F
:101BE000204A230090407800404C230010407800A9
:101BF000E4B302000000000010C0B300FCB4020017
:101C00000000000013003700F04F400003003200D6
:101C1000EF4F400007003A00030037006CC202009B
:101C200000000000B8FD370058C2020000000000AC
:101C3000080037006F0460004844DD0060A6020021
:101C4000000000000080FB00000074000CC20200D5
:101C50000000000010C0B300010037000040EB009E
:101C60008CA3020000000000A7FD37004F0478009D
:101C700000000600813A2300114068000080FB004C
:101C800002A62A0062407800804878000000060022
:101C900041002000C0A52A00B2A5040000000000F9
:101CA000889FBE00D822A800DA22A900D822A90065
:101CB00028022000A0002000CABB02000000000093
:101CC0000804E900FBFF3A00D822A8001004200015
:101CD000CABB02000000000028002000DA22AB008E
:101CE00001003A000004EB0039022000A0002000AF
:101CF000CABB0200000000008904E900FBFF3A00B3
:101D0000DA22AB0001003A00180020000800780039
:101D10004F04BE0000000600881F780000447800D1
:101D2000D822A800DA22A900D822A9004000200069
:101D3000CABB0200000000000804E00001003200FD
:101D4000D822A80080002000CABB020000000000CA
:101D50000804E00004003200DA02D50061446000AB
:101D6000000220000500370090012000CABB0200DD
:101D700000000000D822A80070002000CABB0200AA
:101D80000000000050002000CABB0200000000005C
:101D9000084078004F04780000000600889FBE00CD
:101DA0000044780089C0B3000884FB00610064002F
:101DB000D9FF07000804D1000004E0000100320050
:101DC0000874A0008944E900F7FF3A008000200071
:101DD000CABB020000000000084078004F04BE00AB
:101DE00000000600889FBE008A9FBE008C1F7800FE
:101DF000803A23000048EB00D005B0001040780086
:101E00006240600058003A00A5FF07000000E000B3
:101E100055003A004040230010407800DFFF0700E3
:101E200018C0B3000045EB008A457800884478006C
:101E300010C0B300B8FF07000046780010C0B30020
:101E4000B5FF07000C04E000030032000004E000CE
:101E50001A003200360037000004E0001F003A008C
:101E6000903A23001040780080CF540008003100E1
:101E70008A80FB00A03A23000080400010409000C0
:101E8000004064000080FB000000EA00030037000F
:101E900000C06C000080FB000000E9004F00DE0085
:101EA0000004E00005003A00E8CF54003A003E008C
:101EB000A03A230009487800370037000A80FB0069
:101EC000A13A23008080400011409000084070003B
:101ED0009040980010C0B300080037000A80FB0053
:101EE000A13A23008080400008C1EA001140900020
:101EF00002406000904098000040EB0086FF070021
:101F00008944E8000844440007003A008A80FB0046
:101F1000A03A2300008040001040900055FF0700C9
:101F20000A45E80018C0B300E74F5500C0FF36006F
:101F300000C4B30080CF54000B003600803A230069
:101F40001004E00008003A000000E8000B487800A8
:101F50000B04E00012003A0020A081000090A000D5
:101F600020A089000E003700903A23000048EB00C3
:101F70000000E8000048EB0020A081000090A100D4
:101F800020A089000040EB004F0678004F05BE00FE
:101F90004F04BE000000060089457800CFFF3700DF
:101FA000B03A23001004E000EFFF320010C0B3008D
:101FB000F5FF37000040EB00913A2300804878009D
:101FC0008100E80080487800A00520000100400062
:101FD0001090A10083FF370082FF370000C0EB00A4
:101FE0006EFF07000080FB00000006006BFF07008B
:101FF0000010050010C0B30047FF370020A081008B
:102000004800DE006140600043FF370020A08100EF
:102010004800DE0061006000000006004040230030
:102020001080A10041022000B00020008ABD040001
:1020300000000000404023001080A000410220006A
:10204000B00020008ABD040000000000404B2300C7
:102050001044A000303B23000048EB00D822A80029
:10206000DA22A900000006009100200010432100A0
:102070008ABD040000000000881F780008FF0700E8
:1020800000047800A10020002020200044BD0200B0
:10209000000000000800E00005003A0031002000C8
:1020A00040CC20008ABD0200000000000F00370075
:1020B00091002000C020200044BD0200000000006C
:1020C0005101200050212000E10F54000200320095
:1020D00041012000A022200044BD020000000000B9
:1020E00060A52A00AEA40200000000004F047800A2
:1020F0000000060021C2B300814F500013003200DF
:1021000005003E00E44F500013003200F04F500035
:1021100018003A000700370081C2B300814F500019
:1021200007003200E5C04000814F500011003A0026
:102130000C003700B1012000E02320000B00370025
:10214000A101200090252000080037005101200047
:102150003027200005003700810120008028200062
:102160000200370001012000002A20008ABD04007F
:1021700000000000E1002000002B200044BD04000E
:1021800000000000889FBE008A1F7800800478004D
:102190000104780000C2B3008CA30200000000001C
:1021A000094078009AA302000000000070A52A00F0
:1021B000C8A4020000000000080578008004EB00BD
:1021C0003A80FB003EBB02000000000000C2B300EA
:1021D0008CA30200000000008904E800E88F54008E
:1021E000F7FF3A0061002000A008200044BD020073
:1021F0000000000018407800BEFF07004F0578007F
:102200004F04BE00000006000800FA00889FBE00D0
:10221000000478008804E90000032000808F540047
:1022200024003E00303B23001080FB00808F5400D0
:102230000300390091022000F0022000A6003700C0
:10224000E10020008005200044BD020000000000E5
:102250000940E8009AA302000000000090A52A00AF
:10226000C8A40200000000006A49B900303B230006
:10227000800441000004EB005980FB003EBB0200DB
:102280000000000000C2B3008CA3020000000000A8
:1022900019407800C1FE07000804E800E80F540068
:1022A000F5FF3A0060A52A00AEA40200000000007D
:1022B0008B00370050052000800F5400750032005D
:1022C00006003E000800E0000E003200300320004F
:1022D000800F54007E003A0054003700C00E2000EA
:1022E000800F54002500320064004000800F54002D
:1022F00022003200C00C2000800F540074003A000D
:102300006B003700D1002000600620008ABD02006B
:102310000000000071012000300720008ABD02008B
:1023200000000000303B23001004E00003003200F6
:102330008004E8000004EB0009003700910220004F
:10234000F00220008ABD02000000000008003700F3
:102350000804E8000800BE008AFF0700EA84440081
:10236000303B23001080FB00800F5400F8FF390041
:10237000310D2000000920005700370040402300A5
:1023800008487800C00E2000800F540003003A0077
:10239000310120003016200002003700D10020005B
:1023A000601720008ABD02000000000071012000BB
:1023B000300720008ABD020000000000FDFE07007B
:1023C000313B23008048EB000004EB001200370093
:1023D0000804E800B13A23000800780069FF07000C
:1023E0000800E900E90F50000A003E00303B2300DE
:1023F0001081FB006A11B900EC0041006B01500034
:1024000081014100B43A230007000900B459780063
:102410001048E800F0FE07000004E000ECFF3A007E
:10242000B1022000301820002B00370012FF0700F7
:1024300011012000E01A200044BD0200000000004D
:102440000840780055FE07006D845700E58457006A
:1024500000C0EB0051FE0700006C78000080FB001C
:102460003EBB02000000000000C2B3008CA30200CB
:1024700000000000890F5400F5FF3A0060A52A0013
:10248000AEA40200000000004FF0970019FF070003
:1024900013003700F8FE070001012000F01B2000A8
:1024A0008ABD0200000000000840780006003700E6
:1024B000F1FE0700F1002000F01C20008ABD0200A0
:1024C00000000000C0CCB30034FE07000400370059
:1024D00041022000E01D20008ABD02000000000033
:1024E0004F04BE000080FA0000000600889FBE0076
:1024F000D822A800DA22A900D882A900414B2300E3
:10250000114078000040A0000034A100804878000D
:10251000DFFD070060A60200000000000044780014
:102520000880FB004400DE00E14F50003400320020
:1025300005003900E44F500042003200E54F5000E2
:1025400049003A00440037000880FB008000EB009F
:10255000E90F5000E08F580043003E00006001008A
:1025600045003700EAFF3700070037003E0037001C
:10257000070037003C0037003B0037003A003700C7
:102580000600370005003700C5FD070030003700A2
:1025900000C0EB0001FE07003400370010C0B3009C
:1025A0008CA302000000000000CFB300E94F5400EC
:1025B00001003A00C0CEB3004140230080487800BB
:1025C0007CFE07000500370081002000B03A2300A0
:1025D000B2A50200000000007FFE07000004E0003A
:1025E000F9FF3A008800200000C0EB008CA3020035
:1025F000000000000804E900FBFF3A00C5FF3700B7
:102600006F4464000844E8008CA30200000000004E
:102610008004EB000700370060A602000000000005
:10262000DEFD070010C0B3008CA302000000000014
:102630008904E8000880FB00808F5400F6FF390011
:10264000B4FF37000840780072C1020000000000AB
:1026500010C0B3000500370008407800B8C1020080
:1026600000000000010037000040EB008CA30200D6
:1026700000000000A7FF37004F04BE000000060066
:10268000881F78001030020000000000902E020029
:10269000000000000004780010300200000000007C
:1026A000902E0200000000008000E900E18F500041
:1026B00005003E0050A889000801E9008000EB00F9
:1026C000E10F510018003600403023000048EB00B5
:1026D00021022000405B20008ABD020000000000B3
:1026E0008001EB00220020001100200010002000DB
:1026F0002630020000000000000478006100200085
:10270000605D20008ABD0200000000008001EB0037
:1027100022002000110020001000200026300200BE
:102720000000000011002000E10F540003003200FF
:10273000E20F540005003A0002003700620020005A
:10274000010037004200200042A8890050A88900FB
:102750000100E00010003A00E1002000C05D200010
:1027600044BD02000000000040A881009AA30200BE
:102770000000000000C2B3008CA3020000000000B3
:1027800050A881009AA302000000000000E52A0082
:10279000AEA4020000000000404B230001C3B300C0
:1027A00010C8700041C6B3006000200058B4020099
:1027B000000000004F04780000000600404B23009A
:1027C0001054A00000000600404B23001054A1004C
:1027D0000000060040A881000000A00040A8890079
:1027E00031002000A05E200044BD02000000000077
:1027F00040A881000004A1000043B0008CA30200A7
:1028000000000000404B23001054A10020E52A00E6
:10281000AEA404000000000040A88100E00FB20058
:1028200040A88900404B23001054A0003100200034
:10283000D05E20008ABD040000000000889FBE001A
:1028400040A881000008A3000300320071002000AE
:10285000005F20004D003700E00FB200E40F500091
:1028600021003200E60F500043003A002000200013
:1028700076B502000000000021C3B3004000200034
:1028800040B402000000000021C3B300400020005B
:1028900058B4020000000000E90020000004EB0032
:1028A0000804D10021C3B3004000200040B402005E
:1028B000000000002000200076B5020000000000AB
:1028C0000004E0000100320008D0A00021C3B300E2
:1028D0004000200058B40200000000008904E90014
:1028E000EFFF3A00170037002000200076B5020005
:1028F00000000000090120000004EB000804D100E2
:1029000021C3B3004000200040B4020000000000DA
:102910002000200076B50200000000000004E00066
:1029200002003200000028000804700021C3B30038
:102930004000200058B40200000000008904E900B3
:10294000EEFF3A0021C3B3004000200040B4020073
:102950000000000021C3B3004000200058B4020072
:102960000000000041C1B3002000200058B4020064
:10297000000000000800370030E52A00AEA4020085
:1029800000000000C1002000705F20008ABD02002E
:10299000000000000004EB00080078004F04BE00B7
:1029A00000000600889FBE008A1F7800800478001F
:1029B00040A8810000057800EA0FB2000008A300DB
:1029C00042003200E40F55000400320018002000DD
:1029D000E60F55009E003A00020037001800200064
:1029E0001B00370091C1B3004000200040B402003A
:1029F00000000000090064000500320091C1B3002E
:102A00002000200040B40200000000000400370055
:102A100091C1B3002000200058B402000000000063
:102A200091C1B3004000200058B402000000000033
:102A300091C1B3002000200058B402000000000043
:102A40000A05E9001D00320008044400E5FF3700D4
:102A500091C1B3004000200040B40200000000001B
:102A6000090064000500320091C1B300200020007D
:102A700040B40200000000000400370091C1B30020
:102A80002000200058B402000000000091C1B300F3
:102A90004000200058B402000000000091C1B300C3
:102AA0002000200058B40200000000000A05E900E0
:102AB0000200320008044400E5FF370050A88100FE
:102AC000F6BB02000000000067003700E40F55006D
:102AD00003003200E60F55005D003A0003003700A6
:102AE0000A012000180020003E00370091C1B30009
:102AF0004000200040B402000000000091C1B3007B
:102B00002000200058B402000000000091C1B30072
:102B10004000200058B402000000000091C1B30042
:102B20004000200058B4020000000000EA0020002D
:102B30001800200091C1B3004000200040B4020002
:102B400000000000090064000500320091C1B300DC
:102B50002000200040B40200000000000400370004
:102B600091C1B3002000200058B402000000000012
:102B700091C1B3004000200058B4020000000000E2
:102B800091C1B3002000200058B4020000000000F2
:102B90000A05E9000200320008044400E5FF37009E
:102BA00091C1B3004000200040B4020000000000CA
:102BB00091C1B3002000200058B4020000000000C2
:102BC00091C1B3004000200058B402000000000092
:102BD00091C1B3004000200058B402000000000082
:102BE0002100370091C1B3004000200040B4020032
:102BF00000000000090064000500320091C1B3002C
:102C00002000200040B40200000000000400370053
:102C100091C1B3002000200058B402000000000061
:102C200091C1B3004000200058B402000000000031
:102C300091C1B3002000200058B402000000000041
:102C40000A05E9000800320008044400E5FF3700E7
:102C5000C1002000705F20008ABD0200000000005B
:102C60000000EB0001003700001020004F05780045
:102C70004F04BE0000000600881F78000000E0003E
:102C800003003200E10F500037003A000300370024
:102C9000D1002000306020003500370048A88100B6
:102CA000E80FB200E60F540028003A00B0A68100F9
:102CB0000080A000B0A68900C6FE07000000EB005F
:102CC00038FF0700D4FE07000000EB0035FF0700C7
:102CD000C0FE07006000200032FF07000804E90082
:102CE000FCFF3A00400020002EFF0700CAFE07004C
:102CF000D2FE070000047800B0A681000080A10089
:102D0000B0A68900810020000061200044BD0200BF
:102D1000000000004540DE00CEA5020000000000DB
:102D2000710020008061200044BD0200000000000E
:102D30007F006400FAA502000000000020E52A00E0
:102D4000AEA4020000000000040037005101200082
:102D5000F06120008ABD0200000000000102200096
:102D6000406320000200370041022000E01D2000E7
:102D70008ABD0200000000004F0478000000060039
:102D8000B1002000004521008ABD040000000000C1
:102D9000881F780000E62A00C8A402000000000096
:102DA000404B23001044A00041C6B3006000200047
:102DB00058B40200000000006000200040A8890014
:102DC0002000200050A8890060A60200000000003A
:102DD0000084FB0088007800010CB200020420008F
:102DE000828F50006900320003003C000100E000C7
:102DF00008003200F4FF370000082000808F5000E8
:102E00006B003200000C2000808F5000EEFF3A0073
:102E10007A00370088007800010FB200030032000A
:102E2000F08F500088003A001A0037000080FB0045
:102E30008000EB00E70F5000E08F580082003E005A
:102E400000600100840037000600370009003700E9
:102E50000A0037000C0037000B0037000A0037006B
:102E60000900370000E62A00C8A4020000000000A4
:102E700060003700600020000100370040002000A3
:102E800040A889005B0037006404540058A88900FA
:102E900058003700640064000838A30022003200A4
:102EA0000000E0000500320051C0B3000002200025
:102EB00040B40200000000000400370051C0B3001D
:102EC0000002200058B40200000000000818A3000F
:102ED0000500320051C0B3008000200040B4020061
:102EE000000000000400370051C0B3008000200043
:102EF00058B40200000000000808A30005003200DA
:102F000051C0B3000001200040B4020000000000E6
:102F10003800370051C0B3000001200058B402004F
:102F200000000000330037000000E0000500320020
:102F300040062000E0A3890020032000F0A38900C0
:102F400001003700E0A38900228002000000000099
:102F50000818A30003003200C922A900CB22A80050
:102F600002003700C922A900CB22A9000808A3004B
:102F700003003200E082A800E282A9001D003700B1
:102F8000E282A900E082A9001A00370040A881006F
:102F90000000A00040A8890008007800F003B200FB
:102FA00080FE070040A88100E00FB200B4FF3700A8
:102FB00040A881000000A00040A889000800780017
:102FC000F003B20077FE070040A88100E00FB200D6
:102FD00040A8890060A60200000000004804DD004F
:102FE00060A60200000000000080FB0008007000E6
:102FF0006CFE070010C0B3001400370040A8810029
:103000000000A00040A8890008007800F003B2008A
:1030100064FE070040A88100E00FB20040A88900CC
:1030200010C0B3008CA302000000000003FE0700E4
:10303000000478004840DE008CA30200000000007D
:1030400008407800010037000040EB008CA302002C
:10305000000000005CFF37004F047800000006000D
:10306000807C89000000060050FD2200104078009E
:1030700041FD220042C0B3000004E0000100320024
:1030800002C1B300824878000080FB00B0248800B1
:1030900050FD220000C8EB000000EB00F0FF3700FD
:1030A000C07E81000000E0000D003200E80F5000FB
:1030B00001003600800020008000EB000500370092
:1030C000027C810012019000B37E810063F17800E0
:1030D0008100E800808F5000F9FF390003003700BD
:1030E0000000EB00DEFF07000000EB00017C810028
:1030F00080487800017C81001141900002C1EA0003
:103100000244B20083C8B3000341710092409800AA
:10311000B17E810080804000B17E8900C17E810047
:1031200000805000C07E89000000060001003700CA
:103130009404A8009404AB00FDFF320011C0B3005A
:1031400040FD22000148780094C4AB00FEFF3A0025
:1031500041C0B30040FD2200014878000000060095
:10316000F00F200070248800000006000000EB0033
:10317000507C8900607C8900707C89009624EF0077
:103180009424A8009424A900F00F20007024880043
:1031900020F92200A14A2000020420000001410081
:1031A000050037000008EB008001EB0073B89F00BA
:1031B0008018EB0064004000820F5000F9FF3A00D5
:1031C0000000EB0001002300010140008041EB0002
:1031D0001341980064004000F80F5000F9FF3A00D6
:1031E000D0002000502588000000EB00807E890080
:1031F00042FD22000049EB00907E890050FD220034
:103200000048EB0080C0B3008048780080012300B4
:103210001080890081C8B3001000230001487800A5
:10322000630040000048EB0000022300308089006A
:1032300081C4B3005000230001487800000006005C
:10324000800020005024880041C0B30040FD2200CF
:10325000014878005024800068006000F8FF3A00C0
:10326000907E890051FD220080487800BFFF070052
:1032700094A4A90000000600D0F722001080FB00F3
:103280004400DE004200DD0001F922006100780008
:103290000000E00001003200000001000000060014
:1032A000D0F722001080FB004400DE004200DD0069
:1032B0000080E80001F92200610078000000E000D1
:1032C000010032000000010000000600507C89006F
:1032D00000000600607C890000000600707C890008
:1032E000000006004200DD0002F9220001317800F2
:1032F000000006004200DD0022F9220001307900C2
:1033000000000600107C8900217C8900327C890045
:10331000437C89000000EB00507C8900607C8900C0
:10332000707C89004EFF07006000B800F1FF0700C5
:103330008EFF0700A624EF00A824EF000000230062
:103340004800DE00C02488000008200030248800E7
:103350008804A80094A4A90000000600017C810054
:103360008048780081CCB300007C81001140980037
:103370000000060081C0B30000002300014878006F
:1033800040C8B3005100230080487800E48050001A
:1033900080487800000006001000900090409000E7
:1033A000E1CF50001F00320003003900E3CF50008E
:1033B00042003A0033003700017C81009100900008
:1033C0008048EB00017C8100910090000041EB00FF
:1033D0009240980040409000EF00600081804000E3
:1033E0000080FB004700DE0080804000C208DD0056
:1033F0000000230081004000114090000024A10043
:10340000904098000004E00004003200007C81003D
:103410001000900011C0B300014878002000200087
:10342000250037006400400010417800EF40610043
:103430008180FB0081804000A24A20000281400080
:103440001210A1001081FB004711DE000280FB007A
:1034500080804000C208DD000000230081004000A1
:10346000114090000024A100904098000204E00068
:10347000020032000064A0000D0037000064A100CB
:103480000B00370040409000EF006000818040005A
:103490000080FB004700DE0080804000C208DD00A5
:1034A0000000230081004000114090000024A00093
:1034B000904098000000EB00A8FF3700ADFF3700F8
:1034C00090009000114090000004E00005003200E0
:1034D000EA4F50000B003200EB4F500019003A0049
:1034E00010003700017C8100910090008048780036
:1034F000017C810091009000904098002000200005
:103500000F00370041409000E14F50000D003E0099
:10351000007C8100100090000048EB0010002000AB
:103520000700370041409000E14F500005003E0089
:10353000214090000004E00002003A000000EB008F
:1035400086FF37008BFF370010009000104190007D
:103550000281FB008001EB00E90F5100E08F590070
:10356000A8003E0002600100090037001300370088
:10357000A400370017003700A20037001C003700F6
:10358000260037009F003700880037008D00370085
:10359000007C810010009000817E8100014878004D
:1035A000007C810010009000817E8100C808DE0050
:1035B000114098002000200091003700204090002A
:1035C000E14F50008F003A00807E81000010A10082
:1035D0000500370020409000E14F500089003A007C
:1035E000807E81000010A000807E8900830037006B
:1035F000B04090000104E00082003A0020409000BA
:103600000004E0007F00350051FD22008048780072
:103610004083290092FE070078003700B0409000F8
:10362000E2CF50000D003200E3CF500037003200EF
:10363000E1CF500054003A00117C8100B17E890036
:103640001181FB00C27E8900704190000204E000FD
:1036500050003A0060409000460037008081E8004A
:10366000117C81009150900093CF100046003100F2
:10367000217C8100B17E8900314190004811DD003C
:10368000A14090008180FB0081004100C17E890043
:103690008000EB000A003700C47E81000401410075
:1036A000B27E8900324290004822DD002241900023
:1036B0000281FB0002014200C27E89008100E80015
:1036C0001382FB00B27E8100848F5000F2FF350030
:1036D000F0409000B241900083CF500005003900C7
:1036E0002C003A00E04190002241900082CF51002E
:1036F00028003100C808DD00604090000080FB0019
:1037000080804000C17E8900220037000081E800EF
:103710009281FB00417C8100818F51001A003D00A5
:10372000317C8100B17E89009180FB00C17E8900DF
:103730008000EB0007003700C37E8100B47E81006B
:1037400083014200B37E89009381FB00C37E890020
:103750008100E8009281FB00838F5000F6FF350066
:10376000F04090000104E0000A003A006040900040
:10377000B17E8100914F5000060031000080FB00B7
:10378000C07E89000300370011C0B300A0FD2200F5
:1037900001487800A0FD22001004E00019003A0062
:1037A0003FFE0700008529002DFE3700007C8100C8
:1037B00010009000917E81000148780010002000E8
:1037C0000F003700A0409000E1CF50000D003E00F8
:1037D0008180FB00917E890040FD220005003200BF
:1037E00001C2B30001487800229E020000000000E0
:1037F0000200370001C1B300014878000000EB006F
:10380000D6FE3700DBFE370081C0B300007C8100AC
:103810001140980094A4A900F07B810090009000D2
:103820009180FB00010178000206B2000302200033
:10383000830F51001200320003042000830F510057
:10384000110032000200E00014003A00E380600042
:10385000E18F500006003200E28F50000600320077
:103860000100E0000D003A0037FF07000C003700B0
:1038700013FF07000A003700C7FE070008003700E3
:10388000607C810001003700707C81000000E00056
:10389000030032000000010001003700B5FE070000
:1038A00081C0B300F07B810001487800F27B810089
:1038B0009200900080C8B3001104E00008003500B9
:1038C000E141900080CCB3000304E00004003A0022
:1038D000F14090000104E00001003A0080C8B3000C
:1038E0001041980000000600A0FD22000048EB00F7
:1038F0009124800001407800D2F72200014978002D
:103900008000D100C107B200020023008280400085
:10391000F17B89000034A0000000D100C007B20094
:1039200002004000007C890011409000C003B200FA
:1039300041022000810F500008003200F08040005A
:10394000810F500003003200E40F500004003A00E1
:1039500001003700ACFF370051FE370046FE07007C
:10396000000006008A84AB0004003200C8BF0200D9
:103970000000000000012000502488008A04AB00F1
:10398000030032002EFE07001000200050248800A3
:103990008A24AB0004003200F00F2000702488005D
:1039A00020002000502488008AE4AB00020032008E
:1039B00000082000502488008A44AB000600320032
:1039C000507C81000000E000010032000000010096
:1039D00040002000502488008A64AB0007003200B9
:1039E000902480004400DE006F00600001003A0077
:1039F000BDFF070080002000502488000000060062
:103A00006000B80072990400000000006000B80077
:103A100072990400000000006000B8007299040070
:103A200000000000889FBE008A9FBE00F07B8100DE
:103A30001000900001FE220009000900B058780033
:103A4000A000B1000A7F81001B7F81000A01BE0037
:103A500000402200410F2000182602000000000054
:103A60000004BE000A01BE0000402200410F2000F9
:103A7000382602000000000000014000818148005B
:103A8000820F5500838F5D000200360061045400F0
:103A9000E0845C00481188006000B8007A99020058
:103AA0000000000061D029000000EB0072990200C4
:103AB000000000000000EB00AE99020000000000D2
:103AC00081C0B300F07B81000148780081C8B30059
:103AD000F07B8100114098004F05BE004F04BE00EE
:103AE00000000600881F7800F07B810090009000A5
:103AF0001181FB003206B20010022000800F51003D
:103B00003B003A0011409000E44F500007003E0097
:103B1000E24F5000360031000004E0000C0032009B
:103B2000E14F500032003A0009003700824F500048
:103B30001000320022C2B300824F50001F0032003A
:103B400001C2B300814F500029003A000400370041
:103B50000000EB00AE9902000000000026003700D4
:103B600021D129000000EB007A990200000000003A
:103B70002100370031049000EA0F540001003600A4
:103B8000A8002000007C810010009000080178004F
:103B900001FE2200A42802000000000008007800B6
:103BA000AE99020000000000C1D029000000EB0027
:103BB00072990200000000000F0037009100900091
:103BC000517F890001D029000000EB0072990200AA
:103BD000000000000000EB00AE99020000000000B1
:103BE00011C0B300C0FD2200014878000200370078
:103BF000BA990200000000004F047800000006009F
:103C000000202C0011002000007F8900117F890016
:103C10000000EB00207F8900307F890081C0B30065
:103C200080FE220001487800507F81000000A10042
:103C30000010A100507F890020D729006A99040054
:103C400000000000889FBE008000EB0010002000F4
:103C500072990200000000008000EB0020002000AC
:103C600072990200000000008000EB00200020009C
:103C70007A990200000000005001200060258800B1
:103C8000D0012000702588000044EB00C000230014
:103C900008487800204E23007080890089C4B30052
:103CA000D00023000948780020D729006A99020033
:103CB0000000000090FF2200084878000001230067
:103CC000A07F890064014000B27F890080C0EB00C2
:103CD000E3FE220081497800C3E72200837F890048
:103CE000C4FE2200084A7800B380890008497800A1
:103CF0006501400009497800D2FE22000849780099
:103D0000F2FE220001497800C1EF2200917F890074
:103D100002C4B300024878001100980081C8B300C3
:103D2000114098004F04BE0000000600A07F8100F3
:103D30005004E000FDFF330000000600B07F81006A
:103D40005004E000FDFF330000000600A07F81006A
:103D50001040900000C0EA000080FB004700DE0039
:103D600000000600B07F81001040900000C0EA0013
:103D70000080FB004700DE000000060080FF2200FC
:103D80000048EB00E9FF0700F0FE22009080FB00F6
:103D9000A07F81000108A30004003200C1EF2200CF
:103DA000917F8900C1F3220003003700C1F3220094
:103DB000917F8900C1EF220011009800F0FE2200DF
:103DC00010C8EA00A17F8100D0FE220011487800CF
:103DD00002C4B30082487800A17F810011419000A5
:103DE00002C1EA000244B20083C8B300034171007B
:103DF000924098001040780000000600B17F8100DA
:103E0000114190000204E00016003500C2E72200D4
:103E1000C3EB2200E4FE22001404E00003003200A1
:103E200092009800837F8900020037009300980079
:103E3000827F8900B17F810080487800B07F810057
:103E40009040900081C0EA000144B20082C8B300F3
:103E500082C0700011409800E0FE220010C8EA0005
:103E600000000500FFFF37000040EB00E3FF3700D4
:103E7000889FBE00C8FE2200984478000904E00034
:103E800013003200B7FF07000004E0000F0032000B
:103E900009407800D9FF0700E0FD220001C4B3000B
:103EA00098CF100003003A0011C0B3000148780019
:103EB000010037000048EB00C0FE22000048EB0084
:103EC000D0FD22000048EB0001003700FFFF370063
:103ED0004F04BE0000000600889FBE008A1F7800C5
:103EE000D8FD220018407800E34F50002100360032
:103EF000C9FE2200194578000A04E00015003200CE
:103F0000F0FD22001004E0001B003A0095FF0700BE
:103F10000004E000180032000A407800B7FF0700F4
:103F2000E0FD220001C4B30099CF100003003A0065
:103F300011C0B30001487800010037000048EB00D1
:103F4000C0FE22000048EB00D0FD22000048EB003C
:103F500009003700E9FD22001904E00006003200E4
:103F60000040EB00A5FF0700804CEB00004CEB008D
:103F700001003700004CE8004F0578004F04BE00F8
:103F800000000600889FBE008A1F78001AC0B30098
:103F9000F1FD22008A487800817F81008048780006
:103FA000807F81000000E800807F8900C8FE220039
:103FB0001840E800004C7800E9FD2200804CEB003E
:103FC00001C4B300814F500003003A008BFF07008B
:103FD000004CEB008A4C7800F0FD22000048EB001A
:103FE000D0FD22000048EB004F0578004F04BE00D2
:103FF00000000600D0FE22001004E00005003A0098
:104000005EFF0700D1FE2200804878001104E00026
:10401000FBFF3200917F810031407800917F890061
:10402000D1FE22009148E90000000600889FBE00F2
:1040300080047800D8FE22001804E0000A003A004C
:1040400042FF0700804078000040EB000104E000E0
:104050000C00320049FF0700004C78000040EB00E4
:104060001804E00007003200907F8100904C780037
:10407000907F81000000E800907F8900184CE900E3
:1040800010C0B3004F04BE0000000600889FBE00B1
:1040900080047800D8FE22001804E0000A003A00EC
:1040A0002AFF0700804078000040EB000104E00098
:1040B0000800320031FF0700004C78000040EB00A0
:1040C0001804E00003003200907F8100904C7800DB
:1040D00010C0B3004F04BE0000000600814F500026
:1040E00004003A003100200040CC20008ABD0400CA
:1040F000000000005100200070CC20008ABD0200AA
:1041000000000000805123001048E8000000060075
:10411000881F7800004478004100200070CB200008
:1041200044BD020000000000DA02D50061406000DA
:1041300088407800E9FF070031002000B0CB200064
:1041400044BD020000000000D01680004200DE00E6
:104150006140600088407800E0FF070041002000D7
:10416000E0CB200044BD020000000000D01680001B
:104170004300DE006140600088407800D7FF070000
:104180002100200020CC200044BD020000000000DF
:10419000D01680004400DE00614060008840780056
:1041A000CEFF07004F04780000000600889FBE0085
:1041B0008A1F78000004BE000205780080C2B300A8
:1041C0008CA302000000000008007800D0BA0200B2
:1041D000000000000004780008007800E2A302005C
:1041E0000000000090C2B3008CA302000000000099
:1041F0000000EB00890F540004003600100020007E
:104200008A0F5400010039000000EB0011C0B30018
:10421000B2FF07004F0578004F04BE000000060003
:10422000889FBE008A1F780080447800014478008F
:10423000805123000048EB000904E00004003A002C
:10424000B0A681000080A000B0A689000C00370055
:104250000804E0000A003200E1022000C0BF200094
:104260008ABD02000000000011012000F03321008F
:104270008ABD02000000000060A6020000000000ED
:1042800041002000A0C220008ABD02000000000002
:10429000DAA2A800D8A2A90031002000E0C22000C4
:1042A00044BD020000000000D01680004500DE0082
:1042B0006140600011C0B30088FF0700DAA2A900C6
:1042C000D8A2A800CB02A800C902A9008100200042
:1042D00010C3200044BD0200000000005016800002
:1042E0004800DE006140600011C0B3007BFF0700A2
:1042F000CB02A900E082A800E282A9008100200090
:1043000090C3200044BD0200000000001017800090
:104310004400DE006140600011C0B3006FFF070081
:10432000E282A900E082A9008100200010C42000E0
:1043300044BD020000000000101780004400DE00B1
:10434000614060008040EB0064FF0700C922A900C3
:10435000CB22A80020002000F6BB020000000000D5
:104360004100200090C4200044BD02000000000075
:10437000501680004900DE006140600011C0B300AB
:1043800056FF070061002000904821008ABD02000E
:104390000000000031002000F048210044BD020070
:1043A00000000000D01680004A00DE00614060007E
:1043B00011C0B30049FF070031002000204921004F
:1043C00044BD020000000000D01680004900DE005D
:1043D0006140600011C0B30040FF070021002000D1
:1043E0005049210044BD020000000000D0168000AA
:1043F0004B00DE006140600011C0B30037FF0700D2
:10440000A10020007049210044BD0200000000000E
:10441000DCBE02000000000011C0B3002FFF070047
:10442000E1002000D0C420008ABD0200000000008E
:1044300021E3A80041002000104A210044BD0200F1
:104440000000000072352000712B2000F0002000D9
:1044500056FF070021002000B0C5200044BD020027
:104460000000000072352000712B20002000200089
:104470004EFF0700E882A800EAA2A900E8A2A9006E
:1044800021002000B0C5200044BD02000000000053
:1044900000C2B3008CA30200000000003100200025
:1044A000D0C5200044BD0200000000002000200014
:1044B000F6BB02000000000072352000712B2000C6
:1044C0005000200039FF0700E882A800E8A2A800F9
:1044D0000804E000080032003100200040C620003F
:1044E00044BD02000000000002252000011B200046
:1044F000100020002DFF07004100200000C6200012
:1045000044BD02000000000002252000011B200025
:104510000000EB0025FF0700E8A2A800EA82A9003E
:10452000E882A9004100200000C6200044BD02002E
:104530000000000000C2B3008CA3020000000000D5
:1045400031002000D0C5200044BD02000000000062
:1045500020002000F6BB0200000000000225200021
:10456000011B20005000200010FF0700E8A2A80057
:10457000E882A80021E3A9008100200070C6200085
:104580008ABD0200000000001AFE2F00802D2000CE
:1045900010086500E0168000E001B300E016880016
:1045A00040062000F6BB02000000000010C0B3006F
:1045B000D7FE0700A1002000F0C620008ABD02003F
:1045C00000000000C02D2000100865000804E00075
:1045D00005003200E8A2A800EA82A900E882A9004A
:1045E000E082A800E282A90040062000F6BB02009B
:1045F000000000000040EB00C5FE07000804E000DA
:104600000E003200A100200090C720008ABD0200E9
:1046100000000000C0168000E001B300C016880052
:1046200040062000F6BB02000000000010C0B300EE
:10463000B7FE0700E8A2A800E882A8000904E0008D
:10464000160032000804E00014003200C922A9005C
:10465000CB22A800CD02A800C942A900CD42A800E3
:104660006102200030C820008ABD02000000000066
:10467000F1002000003321008ABD0200000000008C
:1046800060A6020000000000C942A900CD42A900B6
:10469000CD02A900C922A900CB22A90074BA020048
:1046A000000000006100200090CA200044BD02000C
:1046B0000000000088512300184078009AA30200EF
:1046C0000000000081002000F0CA20008ABD020026
:1046D00000000000B0A681000080A100B0A6890003
:1046E000184078004F0578004F04BE000000060017
:1046F000220320001241780032E0B7001180BA0096
:104700009100BA0023032000824978004800DD00B0
:10471000008070000000060001102000624D2300A0
:104720009280600002003A00C29F02000000000078
:1047300000000600889FBE008A9FBE0000447800EB
:104740002AC0B3008041EB0049C6B3008885FB0056
:104750000981FB00110009008285D80080057800DE
:104760000304E00002003A000B04E00007003200FE
:1047700001C3B30001C04500E7FF07000980FB004B
:104780000B80B9000044540013C0B3000A45E9008F
:10479000060032008984FB00A200200011000900FD
:1047A0008284D80080047800E8FF370001C3B3009A
:1047B00001404400D8FF07004F05BE004F04BE0073
:1047C00000000600881F78007D02B900D302200097
:1047D000110009000382D8004206200011000900E0
:1047E0000280D80001047800D2FF0700E0C2B300C5
:1047F000C9FF0700E94F540002003E0000C3B300A8
:10480000C5FF070008407800CAFF07004F04780082
:1048100000000600889FBE008A9FBE0080047800CA
:104820004AC0B3008041EB0008712200110009006A
:104830008884D800800578000304E00002003A0074
:104840000B00E0000600320001C3B30001C04500C8
:10485000B1FF070008D8B9008084540013C0B3002A
:104860000A45E90005003200A200200011000900FD
:104870000284D80000047800ECFF370001C3B300C5
:1048800001C04400A4FF07004F05BE004F04BE0056
:10489000000006000400FA00889FBE008A9FBE0048
:1048A0008C9FBE000004BE008CC0B3008046EB00AD
:1048B0000A102E005B5F20000A01BE000800BE0047
:1048C00018260200000000000002BE000D04E000F7
:1048D00003003A00E00F5000E08F58000E00320055
:1048E00001C3B3000140420084BF9F0095BF9F00F9
:1048F00089FF07000A01BE000FBA97009FBA970010
:104900000400BE003E260200000000000004540027
:1049100081845C001DC0B3000C46E9000700320032
:10492000A2002000030020000A00BE00182602009A
:10493000000000000005BE00DFFF370001C3B30028
:104940000140440074FF07004F06BE004F05BE0043
:104950004F04BE000080FA0000000600881F7800A7
:1049600000047800010037006BFF07003840780032
:104970000004E000FCFF3A00D0C0B30066FF07006F
:10498000A0C0B30064FF07004F04780000000600D9
:10499000881F780000047800010037005EFF0700E0
:1049A000384078000004E000FCFF3A004F04780033
:1049B00000000600889FBE008A1F78008C9FBE0002
:1049C0000004BE00F0232400F1002000800F5400FA
:1049D000818F5C001600360002242400F3002000C2
:1049E0000800BE00182602000000000089FF070032
:1049F000C0C2B30048FF070002242400F3002000D7
:104A00000800BE0038260200000000000004BE00BE
:104A10001A002000703E2000800F5400E08F5C00E0
:104A200008003E0080E12A00D9FF0700240037007B
:104A30000005EB00703E2000800F5400E08F5C000A
:104A40001F003600823E2000030020000800BE0048
:104A500018260200000000000006BE0030062000FC
:104A6000800F5600E08F5E000A003E000A00E00062
:104A700008003200E90F5600E08F5E0003003600A8
:104A800000C3B30024FF070002003700D0E12A0072
:104A9000BFFF07000C0078005EFF0700C0C2B30034
:104AA0001DFF0700823E2000030020000800BE001A
:104AB00038260200000000000004BE001A0020009A
:104AC00030062000800F5400E08F5C000A003E009A
:104AD0000A00E00008003200E90F5400E08F5C009B
:104AE0000300360000C3B3000BFF070002003700CD
:104AF000D0E12A00A6FF07000800780045FF070064
:104B00004F06BE004F0578004F04BE0000000600AF
:104B1000889FBE008A1F78000045780000E22A00C6
:104B20009BFF070089C0B30008C8B3000A406400B7
:104B30000200320010C3B3000100370000C3B3000D
:104B4000F5FE07008944E900030032000884FB00F9
:104B50000804D100F5FF37004F0578004F04BE0070
:104B600000000600889FBE008A1F780001057800BB
:104B7000800478000004EB0003003700394078001F
:104B8000E5FE07000804E8008A0F5400FBFF390027
:104B90004F0578004F04BE0000000600889FBE004D
:104BA000000478002100200030E22A00EDFF070019
:104BB0004C40DE0059E22A0069407800D6FE07002A
:104BC0004840DE006F00600069407800D2FE0700B8
:104BD0004440DE006F00600069407800CEFE0700B0
:104BE0006F04640069407C00CBFE07004F04BE00E8
:104BF00000000600889FBE0000047800210020000D
:104C000030E22A00D7FF07004440DE006F0060005A
:104C100059E22A0069407800BFFE07006F04640073
:104C200069407C00BCFE07004F04BE000000060087
:104C30000000E0000200320010C3B30001003700A2
:104C400000C3B300B4FE3700B3FE3700889FBE0038
:104C50008004780000C3B300FBFF070080C7B300E7
:104C6000F9FF07004448DE006F00600058E22A00A8
:104C700068407800F4FF0700EF84640068C07C009F
:104C8000F1FF07004F04BE00000006009E9E0400D6
:104C9000000000001000050010C0B300D1FE22008B
:104CA0001104E00005003A00A69E0200000000008A
:104CB0000080FB000000EA004F00DE00000006005C
:104CC000FA9F040000000000389F0400000000006C
:104CD00000000500000006000000060000000600BD
:104CE0000000060000000600D862A800D842A90013
:104CF000D822A900D882A900DA62A900DA42A90064
:104D0000DA22A900DA82A90000000600D01680008D
:104D10004300DE006140600000000600D17F81009A
:104D2000C208DE00E1C06000014078000004A2007B
:104D30006100600000014000D0FF2F00C416800019
:104D40008401600083017100C3168800E180600067
:104D500081804000DA02B60000807000D016880022
:104D600040012000CABB040000000000DA22A900B4
:104D7000D822A90040012000CABB040000000000A6
:104D8000D17F8100C208DE00E1C0600001417800EF
:104D90000204A200610161004211DD00B0FF2F009A
:104DA000C41680008401600083017100C31688006E
:104DB000E1806000C208DD00DA02B6000080700009
:104DC000D016880040062000CABB04000000000086
:104DD000DA42A900D842A90040062000CABB04005C
:104DE00000000000889FBE00804478000044EB0073
:104DF00003003700E2FF0700F5FF07000844E80062
:104E0000894F5400FBFF39004F04BE00000006002C
:104E1000881F7800DAFF0700D81680004344DE00C0
:104E200061446400EAFF0700084078004F047800FE
:104E300000000600881F78000004E00002003A002D
:104E4000CAFF070001003700B4FF0700CCFF0700CE
:104E5000D81680004344DE0061446400DCFF070094
:104E6000084078004F04780000000600889FBE00CC
:104E7000D7FF0700A8FF22009840780068C06000B4
:104E800005003200D07F81004400DE0061406000F8
:104E9000E8FF07001834A10089C0B3000044EB000C
:104EA000B7FF07000884FB000804D100DA62AB00FA
:104EB0000200320000C8B30000444400C4FF0700F1
:104EC0008944E900F6FF3A00084078004F04BE002C
:104ED00000000600889FBE008A1F7800004478000A
:104EE000BBFF0700A9FF22009940780068C060005E
:104EF00005003200D07F81004400DE006140600088
:104F0000CCFF07001934A1008044EB00094578006C
:104F10000808A30002003A0094FF070001003700D0
:104F20007EFF070096FF07000884FB000804D100FD
:104F30008984FB008904D100DA62AB0002003200F0
:104F400000C8B30080C44400A1FF0700A0FF2200F6
:104F500010417800E3406100E2CF50000B003A00BE
:104F6000E64F550009003A00824078000130A00069
:104F70000808A30002003A000144A1000100370024
:104F80000144A00001487800030037000A45E8000A
:104F9000E84F5500DEFF3A00094078004F057800E1
:104FA0004F04BE0000000600D17F8100C208DE0071
:104FB000E1C06000014178000204A20061016100CB
:104FC0004411DD00F0FE2F00C41680008401600053
:104FD00083017100C3168800E1806000C408DD0011
:104FE000DA02B60000807000D01688004001200070
:104FF000CABB040000000000DA82A900D882A90020
:1050000040012000CABB040000000000E6FF0700CA
:10501000A0C0B30073FF0700F7FF0700A0FF220046
:10502000C1CFB30010C8600000000600881F7800E0
:1050300000447800E24F540010003200E34F540067
:10504000040032000804E00017003A00EFFF0700F8
:1050500015003700D4FF070010C0B30061FF070040
:10506000E5FF070020C0B3005EFF0700A0FF22009D
:105070009040780063C870000B003700CAFF07003B
:105080000840780057FF0700DBFF07000840780062
:1050900054FF0700A1FF2200114078000000A1008A
:1050A0000014A000804878004F047800000006003B
:1050B000881F7800A8FF2200D07F81006300600075
:1050C000E20F500005003200E30F500019003200DB
:1050D000E10F50001A003A00200037001840780015
:1050E0000038A300070032000048A300020032008D
:1050F0000AFF0700010037001CFF0700A0FF220085
:105100001034A100A8FF070020C0B30035FF07003E
:10511000B9FF070010C0B30032FF0700A1FF220053
:10512000114078000000A0000014A1008048780021
:105130000A0037009CFF070020C0B30029FF0700CA
:10514000ADFF070010C0B30026FF0700184078002D
:105150000000A0000014A100004C78004F0478006B
:1051600000000600881F7800DFFE0700A0FF220075
:10517000104178000224A00071CEB3000148610004
:1051800060A602000000000000447800E0FF22005A
:1051900008487800E24F540006003200E34F540004
:1051A0003D003200E14F5400F5FF3A0097FF070041
:1051B0003700370095FF0700D8FE0700BCFF070047
:1051C0000840780099FF070000C0EB0005FF0700CA
:1051D00000C0EB0003FF0700B5FF070030C0B300BD
:1051E00092FF07000000EB00E07F89000600370017
:1051F000E07F81000000E800E07F8900910F20003F
:10520000810F50000300360001FF07000004E0009A
:10521000F7FF3200A6FF07007CFF0700A4FF07008E
:1052200030C0B30081FF070020002000E17F810033
:105230000008DD008CA3020000000000F0FF220047
:105240000048EB000D00370008FF07008CA30200A8
:105250000000000005FF07008CA302000000000012
:1052600002FF07008CA3020000000000FFFE070001
:105270008CA3020000000000184CE800F8FF220098
:105280009880FB00E07F8100808F5000EEFF3900A6
:1052900087FF0700BAFF3700B4FE0700CCFE070007
:1052A00055FF0700ACC0020000000000607802005B
:1052B00000000000E07F89008CA3020000000000D5
:1052C000AFFF370060E62A00C8A404000000000019
:1052D00060A6040000000000881F780000447800E9
:1052E0000880FB008000D0000102B200C2168000DE
:1052F0000250A10002817000C21688004201DE0047
:1053000062016100C11680000110A10081007100DE
:10531000C116880064016000C11680000120A10050
:1053200081007100C11688004201DD006801610042
:10533000C11680000130A10081007100C1168800F3
:10534000610060004400DD00C11680000140A10042
:1053500081007000C116880050002000CABB020006
:105360000000000000CEB30000406400DAA2AB00F1
:10537000010032000044A000DA22AB00010032003C
:105380000034A000DA42AB00010032000024A0008B
:10539000DA62AB00010032000014A000DA82AB0038
:1053A000010032000004A0004F0478000000060055
:1053B000881F7800004478000880FB000068A30084
:1053C00003003200C922A900CB22A8000200370046
:1053D000C922A900CB22A9000058A3000300320073
:1053E000E082A800E282A90002003700E282A90060
:1053F000E082A9008000D0000102B200D216800035
:105400000250A10002817000D21688004201DE0025
:1054100062016100D11680000110A10081007100BD
:10542000D116880064016000D11680000120A1001F
:1054300081007100D11688004201DD006801610021
:10544000D11680000130A10081007100D1168800C2
:10545000610060004400DD00D11680000140A10021
:1054600081007000D116880050002000CABB0200E5
:105470000000000000CEB30000406400DAA2AB00E0
:10548000010032000044A000DA22AB00010032002B
:105490000034A000DA42AB00010032000024A0007A
:1054A000DA62AB00010032000014A000DA82AB0027
:1054B000010032000004A0004F0478000000060044
:1054C000E8A2A800E882A80000C0EB0082FF070065
:1054D0000040EB00B6FF3700881F7800804078005E
:1054E0000040EB0010A10200000000000044780022
:1054F0000804E00001003200CB02A8000840780058
:105500008CA30200000000004CA602000000000076
:105510000004E0000D00320060A602000000000060
:10552000E14F400004003200084040008CA302001C
:10553000000000000500370010C0B3008CA302007B
:10554000000000004F047800000006000804E0009E
:10555000EDFF3A0000A881000000E0000B003A00D7
:105560000080EB0000A8890051168000C808DE000A
:105570008180EA00E1806000C808DD0050168000EC
:105580000080A100008070005016880000A88100F3
:105590000000E90000A88900DBFF3700889FBE00FB
:1055A000CB02A800C6FF070046FF070048FF070020
:1055B00021502300804878000004E000AB00350053
:1055C000F9FF3200E14F500004003A00BCFF070031
:1055D0000C66020000000000F2FF3700E24F5000AE
:1055E00004003A00B6FF0700087E02000000000039
:1055F000ECFF3700E34F500004003A00B0FF070013
:10560000946E020000000000E6FF3700E44F5000F7
:1056100004003A00AAFF0700769202000000000092
:10562000E0FF3700E54F500004003A00A4FF0700F8
:105630005289020000000000DAFF3700E64F5000F8
:1056400002003A009EFF0700D6FF3700E74F5000E8
:1056500004003A009AFF0700C8960200000000000C
:10566000D0FF3700EF4F500009003A0010C0B300E0
:105670008CA3020000000000CB02A90046A6020095
:10568000000000008EFF07004F04BE00000006006F
:10569000F04F500002003A000040EB0003003700DA
:1056A000F14F500003003A0010C0B3008AFF07001A
:1056B000BEFF3700F24F500020003A001021EF00EB
:1056C0001E21EF00B821EF0000FC2F00D406B60029
:1056D0006001B300A0368800FDFE07000080FB00DB
:1056E0000018A3000100320010A1A8000008A300C8
:1056F000010032001081A800F5FE07004804DD001B
:10570000F3FE07000080FB0008047000F80D88001D
:10571000E80D880060002000C00D8800ECFE070046
:105720004804DD00EAFE07000080FB00080070006E
:105730006008880011E1A80006003700F34F500010
:1057400006003A001021EF00B821EF0000FC2F0006
:10575000D426B60010C0B30045003700F44F500007
:1057600008003A0021E3A80010002000D0BA02008F
:10577000000000000004780021E3A9004840DE009A
:1057800027003700F54F500015003A0021E3A8002C
:1057900010002000D0BA02000000000000047800D1
:1057A00046A60200000000004840DE008CA3020074
:1057B00000000000084078008CA3020000000000F8
:1057C0004CA6020000000000E14F5000F0FF3A003C
:1057D00060A602000000000021E3A90073FF37006B
:1057E000F64F500012003A00BA810200000000009B
:1057F0000004BE004808DE008CA302000000000088
:105800004048DE00010020008CA3020000000000E0
:105810004849DD004840DE0000007100C848DE0055
:105820008CA3020000000000084078001000370040
:10583000F84F500007003A00CB22A800C0E62A002B
:10584000C8A4020000000000B2A80200000000008E
:1058500056FF37000068A300020032009EFE0700DA
:10586000030037000040EB0001003700D0FE0700C6
:105870008CA30200000000004CFF3700A83300009A
:105880005E000000020000000000000000000000B8
:105890000000000000000000000000000000000008
:1058A00000000000000000000000000000000000F8
:1058B00000000000000000000000000000000000E8
:1058C00000000000000000000000000000000000D8
:1058D00000000000000000000000000000000000C8
:1058E00000000000000000000000000000000000B8
:1058F00000000000000000000000000000000000A8
:105900000000F000000000007C34000026000000D1
:105910000000000006340000460000000200000005
:1059200080AB8400AB87AB008CAB9100AB96AB0037
:1059300060AB9C00ABA0AB00A6ABAC00ABB0AB00C7
:10594000B3ABB800ABBDAB00C2ABC900ABCFAB00D3
:10595000D5ABDA00ABDFAB00E7ABEB00ABEFAB00F6
:10596000F7ABFB00AB02AC0006AC0D00AC13AC0017
:1059700017AC1C00AC21AC0027AC000000000000FC
:10598000042800006804000000000000003500004A
:1059900004000000000000001435000002000000B8
:1059A0000200000003000000BC3400000E000000F4
